:1083BD00005EBCE2613FDD83C29C7E20A3FD1F41B8
:1083CD009DC3217FFCA2401E5F01E3BD3E6082DCA8
:1083DD00237D9FC1421CFEA0E1BF5D0380DE3C6298
:1083ED00BEE0025CDF81633D7C22C09E1D43A1FF88
:1083FD004618FAA427799BC584DA3866E5BB590778
:10840D00DB856739BAE406581947A5FB7826C49A67
:10841D00653BD987045AB8E6A7F91B45C6987A2457
:10842D00F8A6441A99C7257B3A6486D85B05E7B947
:10843D008CD2306EEDB3510F4E10F2AC2F7193CD37
:10844D00114FADF3702ECC92D38D6F31B2EC0E5027
:10845D00AFF1134DCE90722C6D33D18F0C52B0EE17
:10846D00326C8ED0530DEFB1F0AE4C1291CF2D7307
:10847D00CA947628ABF517490856B4EA6937D58BF7
:10848D005709EBB536688AD495CB2977F4AA4816E7
:10849D00E9B7550B88D6346A2B7597C94A14F6A8D7
:1084AD00742AC896154BA9F7B6E80A54D7896B35C7
:1084BD00FB04FD82FEC1FF60FF96FFB0FFCBFFE521
:0484CD00FFEEFFF7C8
:03BF5B00016C0A6C
:10C65500901E4D121BCFFFFFFFFF901E4D121B7B3F
:01C6650022B2
:10A1630090FFFE121D77ECF0A3EDF090FFFD121DA2
:0AA1730077121C5090FFFC121D77BC
:10A17D00851283851382A3A3E4F085128385138250
:10A18D00F0A3F0900007121D9BE0FEA3E0FF8512E7
:10A19D0083851382E0FCA3E0C39FEE6480F8EC643A
:10A1AD0080985051900004121D9B121C3085128313
:10A1BD00851382E0FEA3E0F5828E8312171EFF85C4
:10A1CD001283851382A3A3E06FFF900003121D9BE2
:10A1DD00EFF0900003121D9BE09083BD93851283D9
:10A1ED00851382A3A3F0851283851382E475F00194
:0FA1FD0012184F808E851283851382A3A3E0FF73
:07A20C00900009121D7722EA
:0BC2C700901E71EFF0A3ECF0A3EDF06F
:10C2D200901E72E0A3E0FF901E71E0FEEF6E781FE9
:07C2E200F6E69083BD93FF17
:01C2E9002232
:08BAA200901B33EFF0A3EDF05F
:10BAAA00901B33E0703DF584759850F584759115B7
:10BABA00F58475C908A3E025E024BBF582E4348443
:10BACA00F583E493F5CB901B34E025E024BCF582A2
:10BADA00E43484F583E493F5CA75C804E4F584D2A2
:05BAEA00ACC2BCD2AFAC
:01BAEF002234
:10B45700901C85121BCF00000000901C89121BCF87
:10B4670000000000901C7C7464F0E47814F67814F3
:10B47700E6C39402748094805043E625E025E024D7
:10B487007DF582E4341CF583E4F0E625E025E0242D
:10B497007EF582E4341CF583E4F0E625E025E0241C
:10B4A7007FF582E4341CF583E4F0E625E025E0240B
:0DB4B70080F582E4341CF583E4F00680B1DA
:01B4C4002265
:10C3D500D2AFD2A9C2BBE4F584E589540F4401F577
:10C3E50089758E02758CAFE4F58AD28C12B457220A
:10815C00E4901C7BF07402F0E4F0F0901C7BE0C324
:10816C00940274809480400302828EE025E025E026
:10817C002480F582E4341CF583E0D394007480945D
:10818C0080500302825D901C7BE025E025E0247E7C
:10819C00F582E4341CF583E0600302825D901C7B65
:1081AC00E025E025E02480F582E4341CF583E03002
:1081BC00E027901C7BE025E025E02480F582E43468
:1081CC001CF583E0D3940174809480400C7D009066
:1081DC001C7BE0FF12A367800A7D01901C7BE0FFF3
:1081EC0012A367901C7BE025E025E02480F582E457
:1081FC00341CF583E06401700A7D01901C7BE0FF68
:10820C0012A367901C7BE025E025E02480F582E436
:10821C00341CF583E014F0901C7BE025E025E02471
:10822C0080F582E4341CF583E06026901C7BE0250D
:10823C00E025E0247FF582E4341CF583E0FF901CFC
:10824C007BE025E025E0247EF582E4341CF583EF09
:10825C00F0901C7BE025E025E0247EF582E4341CC4
:10826C00F583E06014901C7BE025E025E0247EF58E
:10827C0082E4341CF583E014F0901C7BE004F002E3
:02828C00816708
:01828E0022CD
:03000B0002AE4002
:10AE4000C0E0C0F0C083C082C0D0E8C0E0E9C0E08C
:10AE5000EAC0E0EBC0E0ECC0E0EDC0E0EEC0E0EF47
:10AE6000C0E012C3B4901C85121B7BE47B01FAF98D
:10AE7000F81219AF901C85121BC3901C7CE014F0D3
:10AE8000E07017901C89121B7BE4F81219AF901C1C
:10AE900089121BC3901C7C7464F012815C12B7345D
:10AEA000D0E0FFD0E0FED0E0FDD0E0FCD0E0FBD071
:10AEB000E0FAD0E0F9D0E0F8D0D0D082D083D0F062
:03AEC000D0E032AD
:10B9AD0090FFFF121D77EDF090FFFF121D77EFF066
:10B9BD00851283851382E0C3940274809480502D88
:10B9CD00A3E0FF851283851382E025E025E0247D29
:10B9DD00F582E4341CF583EFF0851283851382A381
:10B9ED00E0FD851283851382E0FF12A367900002AC
:04B9FD00121D77227E
:109E6D0090FFFE121D77EAF0A3EBF090FFFF121D9D
:109E7D0077EDF090FFFF121D77EFF08512838513BC
:109E8D0082E0C39402748094804003029F25E025F4
:109E9D00E025E02480F582E4341CF583E0707985BB
:109EAD001283851382E025E025E0247EF582E434DB
:109EBD001CF583E07062851283851382A3E025E093
:109ECD0004FF851283851382E025E025E02480F5CB
:109EDD0082E4341CF583EFF0851283851382A3A3EE
:109EED00E0FEA3E0FF7C007D0A1218198512838520
:109EFD001382E025E025E0247FF582E4341CF58310
:109F0D00EFF0851283851382E025E025E0247EF5B0
:0F9F1D0082E4341CF583E4F0900004121D7722D7
:10A3670090FFFF121D77EDF090FFFF121D77EFF0C2
:06A3770090FFFF121D77AC
:10A37D00851283851382A3E0C39402748094805068
:10A38D0033851283851382A3E025E025E0247DF536
:10A39D0082E4341CF583E0601B851283851382A350
:10A3AD00A3E070047F0180027F00851283851382F4
:10A3BD00A3A3EFF0851283851382E584F075840FD6
:10A3CD00851283851382A3E0700F85128385138216
:10A3DD00A3A3E024FF92828019851283851382A3A3
:10A3ED00E06401700D851283851382A3A3E024FF21
:0BA3FD009283851283851382E0F584B3
:07A40800900003121D7722F2
:10C57700C2AF901C85121B7B901B31121BC3D2AF1D
:06C58700901B31121B7B2A
:01C58D00228B
:06C2560090FFFC121D77B1
:10C25C00C2AF901C89121B7B851283851382121B23
:0CC26C00C3D2AF851283851382121B7BA6
:07C27800900004121D772263
:10B3E80090FFFF121D77EFF090FFFF121D77851277
:10B3F80083851382A3E07005786DF608F6786CE60D
:10B4080075F064A4FF08E6FC08E6C39FEC95F050CD
:01B4180037FC
:10B41900851283851382E584F075840175D480E4EF
:10B42900F58475D103758401AFD2EF9400748094CB
:10B439008040047F0080027FFF8FD285D2D385129E
:07B4490083851382E0F58406
:07B45000900002121D77229B
:10C51300901B31EFF0D209E4786DF608F6E0600481
:09C52300786CF622786C760A228D
:10C5F700C209E4786DF608F6786C76FF75FFDE758C
:03C60700FFAD2262
:10B7340090FFFF121D77786E06E618700106786C8C
:10B74400E675F064A4FF08E6FC08E6C39FEC95F0F8
:02B7540050376C
:10B75600851283851382E584F075840175D480E4AF
:10B76600F58475D103758401AFD2EF94007480948B
:10B776008040047F0080027FFF8FD285D2D385125E
:07B7860083851382E0F584C6
:07B78D00900001121D77225C
:08BEB000901B36EEF0A3EFF049
:10BEB800E4A3F0A3F0901B36E0FEA3E0FFA3E0FCB0
:10BEC800A3E0C39FEC9E50187FE87E0312ACA77FC7
:10BED8000112B3E8901B38E475F00112184F80D5B1
:01BEE8002237
:08ACA700901B3FEEF0A3EFF05B
:0FACAF00901B3FE0FEA3E0D394FAEE9400502AEE
:10ACBE00901B3FE0A3E0F526D3E526940074809424
:10ACCE00804060752701D3E52794007480948040FE
:0AACDE000500152780F0152680DE22
:10ACE800901B3FE0FEA3E0FFA3EEF0A3EFF0901B64
:10ACF80041E0FEA3E0D394FAEE940040147FFA7E7C
:10AD08000012ACA7901B4174FF75F00612184F8013
:10AD1800DD901B3FE0FEA3E0D39400EE94004009D1
:09AD2800A3E0FEA3E0FF12ACA7BA
:01AD310022FF
:10C470004D53434246464600323032342D30352D3E
:0DC480003037202D2062646362653765004F
:04BF5E00410012008C
:1091BA00E4F584901B31F0A3F0758F04901B31E025
:1091CA00FEA3E0F5828E83742E93FE742F93B4343B
:1091DA0007EEB41203D38001C39202E4F58F200292
:1091EA002F7BFF7AC47970782D7C057D0112200FC0
:1091FA00E4900007F0A37450F0A374C2F0A374467D
:10920A00F0A374DFF0A374FFF0E4900A56F08053E1
:10921A00758F04901B31E0FEA3E0AA06F97BFF7864
:10922A002D7C057D0112200F901B31E0FEA3E02466
:10923A0014FFE43EFAA9077BFF78567C0A7D0112E7
:10924A00200F901B31E0FEA3E02428FFE43EFAA998
:10925A00077BFF78077C007D017E007F061216DF00
:10926A00E4F58FE4900000F0A3F0C207900541F006
:10927A009019B6121C30900541E075F010A4F582E1
:10928A0085F08312171ED39400748094804008904E
:07929A000541E004F080D95A
:0192A10022AA
:06B30600901E74121C50A1
:10B30C00901E74121C3090002E1218A66434700417
:10B31C00E5F0641260037F0022C2AFE4F58412C52D
:10B32C00F7E47871F608F643B701758F0718E6FE57
:10B33C0008E6F5828E83E4F0758F05901E74121C5E
:10B34C0030C00218E6FE08E6AA06F8AC027D01D071
:10B35C00027E007F301216DF53B7FEE4F58FD2AFBA
:0AB36C007F0A12C5131291BA7F0187
:01B3760022B4
:03002300025F9DDC
:0D5F9D00C0E0C0F0C083C082C0D075D00845
:105FAA00309972C299900004E004F0A3E0FF9000D7
:105FBA0004E0C39F5054E0C3940474809480501149
:105FCA00E0240DF582E43400F583E06004D29B807E
:035FDA0002C29B65
:105FDD00752214D3E52294007480948040177523A4
:105FED0001D3E5239400748094804005001523802F
:055FFD00F0152280DE1A
:10600200900004E02449F582E43409F583E0F5992F
:10601200800BC284900005E4F0900004F030982BCD
:10602200300628900002E0FEA3E0C3EE940450196B
:10603200900002E475F001121865FE744925F0F52E
:106042008274053EF583E599F0C2982098030262B6
:1060520010300603026210209A0F20080CC298909A
:106062000002E4F0A3F0026210C29A900002E4750A
:10607200F001121865FE744925F0F58274053EF5AB
:1060820083E599F0C298900002E0FEA3E064014E1D
:10609200700F900549E07009900002F0A3F00262CF
:1060A20010900549E05407FF901B2BE4F0A3EFF09A
:1060B200901B2BE0FEA3E064074E7053900002E0B9
:1060C200FEA3E0D39401EE9400404490054AE024FC
:1060D20003FFE433901B2BF0A3EFF0901B2BE0A304
:1060E200E030E735900002E0FEA3E0D39402EE94A4
:1060F20000402690054AE0547FFEA3E02404FDE41C
:10610200334EFEEDFF901B2BEEF0A3EFF0800A90D2
:106112001B2BE475F00212184F901B2BE0FEA3E03C
:10612200FF901B29EEF0A3EFF0900002E0FEA3E047
:10613200B4000EEEB4040A900002E4F0A3F002628E
:1061420010901B29E0FEA3E0FF900002E0FCA3E018
:10615200C39FEC9E5003026210900002E0FEA3E097
:1061620024FFFDEE34FFFC7B017A05794912A1631D
:10617200900002E0FCA3E02448F58274053CF5831C
:10618200E06F600A900002E4F0A3F0026210900552
:1061920049E064B76005E064BF700BD20090000272
:1061A200E4F0A3F0806830080B7A007B327D017F37
:1061B20000129E6D90052CE004F07B017A0979496A
:1061C20090FFFD121D77121C507B017A057949124E
:1061D2000026901B2BEEF0A3EFF0901B2BE0FEA30A
:1061E200E0D39400EE940040157A007B327D017F6B
:1061F20001129E6D901B2BE0A3E0FF12B5A03005AB
:0E6202000675840075EF10900002E4F0A3F022
:0B621000D0D0D082D083D0F0D0E0329C
:01C6F1002226
:06C6DB0090052CE0FF2297
:10C17C0012B734900546E0FEA3E0D39400EE940091
:10C18C00400A90054674FFF5F012184F900546E0F2
:0DC19C00FEA3E04E7006900000F0A3F0221C
:1054DC007BFF7AC47978901B31121C50901B3112CF
:1054EC001C30121705FF3395E04F600C901B32E413
:1054FC0075F00112184F80E47BFF7AC47978C003F1
:10550C00C002C001901B31121C30D3D082D083D08A
:10551C00E0E99582EA95834019901B31121C3012F8
:10552C001705642D600C901B3274FFF5F012184FA8
:10553C0080C6901B31121C30EB8A8389827BFF7AE8
:10554C00C47978F4700A74786582700474C46583C5
:10555C0070030257CA901B32E475F00212184F9078
:10556C001B31121C3090000112171EFF3395E0FE08
:10557C00C3EF9430EE64809480402D901B31121C4C
:10558C003090000112171EFF3395E0FED3EF9439D3
:10559C00EE648094805011901B31121C30900001ED
:1055AC0012171E24D0FF804B901B31121C30900020
:1055BC000112171EFF3395E0FEC3EF9461EE648079
:1055CC009480402D901B31121C3090000112171E3C
:1055DC00FF3395E0FED3EF9466EE64809480501117
:1055EC00901B31121C3090000112171E24A9FF8051
:1055FC00027F00EF7D00FC901B31121C301217054E
:10560C00FF3395E0FEC3EF9430EE64809480402726
:10561C00901B31121C30121705FF3395E0FED3EFAF
:10562C009439EE64809480500E901B31121C301211
:10563C00170524D0FF8042901B31121C3012170525
:10564C00FF3395E0FEC3EF9461EE648094804027B5
:10565C00901B31121C30121705FF3395E0FED3EF6F
:10566C009466EE64809480500E901B31121C3012A4
:10567C00170524A9FF80027F00EFC454F04CFCED09
:10568C00901B31121C3090000212171EFF3395E054
:10569C00FEC3EF9430EE64809480402D901B311249
:1056AC001C3090000212171EFF3395E0FED3EF94CE
:1056BC0039EE648094805011901B31121C30900094
:1056CC000212171E24D0FF804B901B31121C3090FD
:1056DC00000212171EFF3395E0FEC3EF9461EE64D7
:1056EC00809480402D901B31121C309000021217B8
:1056FC001EFF3395E0FED3EF9466EE6480948050E9
:10570C0011901B31121C3090000212171E24A9FF9D
:10571C0080027F00EF75F010A4FFE5F04CFEEF4D1A
:10572C00FF901B31121C3090000312171EFD339595
:10573C00E0FCC3ED9430EC64809480402D901B31E0
:10574C00121C3090000312171EFD3395E0FCD3EDB4
:10575C009439EC648094805011901B31121C309061
:10576C00000312171E24D0FD804B901B31121C30ED
:10577C0090000312171EFD3395E0FCC3ED9461EC11
:10578C0064809480402D901B31121C3090000312C9
:10579C00171EFD3395E0FCD3ED9466EC6480948089
:1057AC005011901B31121C3090000312171E24A9AB
:0E57BC00FD80027D00EEEF4D786FA60608F628
:0157CA0022BC
:09621B00901CF2EFF0A3121C50DC
:10622400901CF3121C3012170564207004D205FF71
:1062340022901CF3121C3012170564616003026380
:106244002A901CF6121C30747812177E901CF612D9
:106254001C309000017405121790786FE6FE08E672
:10626400EEFF901CF6121C30900002EF121790788B
:106274006FE608E6FF901CF6121C30900003EF1244
:10628400179012C256901CF9121BC3901CF9121BD2
:106294007BEFE4901CF6121C30900007EF1217906D
:1062A400901CF9121B7B7808121AE7901CF9121B38
:1062B400C3901CF9121B7BEFE4901CF6121C309067
:1062C4000006EF121790901CF9121B7B7808121A23
:1062D400E7901CF9121BC3901CF9121B7BEFE4908E
:1062E4001CF6121C30900005EF121790901CF91246
:1062F4001B7B7808121AE7901CF9121BC3901CF937
:10630400121B7BEFE4901CF6121C30900004EF1279
:106314001790901CF9121B7B7808121AE7901CF94D
:10632400121BC37F0822901CF3121C301217056441
:10633400687055900A56E0FF3395E0FEEF4E602DED
:106344007B017A0A7956C003C002C001901CF31283
:106354001C30E92401F9E43AA801FCAD03D001D0D2
:1063640002D003121F26EF3395E04F700D901CF6F8
:10637400121C30747812177E800B901CF6121C309D
:1063840074FF12177E7F0122901CF3121C30121727
:10639400056498703E901CF3121C30E92401F9E462
:1063A4003AFA12B306EF601D901CF6121C30747892
:1063B40012177E901CF6121C30900001E412179004
:1063C400D2057F0222901CF6121C3074FF12177E35
:1063D4007F0122901CF3121C3012170564416003E4
:0363E40002646EE2
:1063E700901CF2E0FF3395E0FE7C007D3D1217B272
:1063F700747B2FF974123EFA7B01901CFD121C501E
:10640700901CF3121C3090000112171E6401703C9F
:10641700901CFD121C30E92404F9E43AFA78427C16
:10642700057D017E007F041216DF901CFD121C30D3
:106437009000021218A6FF900000E5F0F0A3EFF01D
:106447009005467403F0A374E8F0800DE490000013
:10645700F0A3F0900546F0A3F0901CF6121C3074E0
:076467007812177E7F01226D
:02646E007F00AD
:016470002209
:08955200901E51EFF0A3EDF0B3
:10955A00E4900002F0A3F0F584FE7F04FD7B017A1B
:10956A0000790D1221D6901E52E030E02FE4A3F0CC
:10957A00901E51E0FF901E53E0C39F501FE0C3941A
:10958A0004748094805015E0240DF582E43400F5CB
:10959A00837401F0901E53E004F080D4901E52E0D0
:1095AA0030E53D900949E064107008901E54740239
:1095BA00F08006901E547404F0E4901E53F0901E3E
:1095CA0054E0FF901E53E0C39F5015E0240DF5822E
:1095DA00E43400F5837401F0901E53E004F080DE59
:1095EA0090000DE024FF929B901E51E0900005F040
:1095FA00751014D3E5109400748094804017751187
:10960A0001D3E511940074809480400500151180FF
:05961A00F0151080DED8
:0F961F00D284900949E0F599E4900004F07F01AE
:01962E002219
:05B5A000901B2DEFF0EF
:10B5A500E4F584C29BE0900005F0E4900004F0907F
:10B5B5001B2EF0901B2DE0FFA3E0C39F5014E02449
:10B5C5000DF582E43400F583E4F0901B2EE004F0E1
:02B5D50080E113
:10B5D700752414D3E524940074809480401775254E
:10B5E70001D3E525940074809480400500152580DB
:05B5F700F0152480DEC8
:0AB5FC00D284900949E0F5997F011F
:01B606002221
:05B60700901B33EFF081
:10B60C00E4F584C29BE0900005F0E4900004F09017
:10B61C001B34F0901B33E0FFA3E0C39F5014E024D5
:10B62C000DF582E43400F583E4F0901B34E004F073
:02B63C0080E1AB
:10B63E00752614D3E52694007480948040177527E0
:10B64E0001D3E5279400748094804005001527806F
:05B65E00F0152680DE5E
:0AB66300D284900949E0F5997F01B7
:01B66D0022BA
:095A7900901D44EFF0A3121C5033
:105A8200901D44E030E104E4FEFF22901D44E0302A
:105A9200E20B901D4CE4F0A37432F0801D901D4483
:105AA200E030E30C901D4C7475F0A37430F0800A62
:105AB200901D4C7401F0A374F4F0E4901D48F0A31F
:105AC200F0901D4EF0A3F0901D4AF0A3F0901D4CF3
:105AD200E0FEA3E0FF901D4AE0FCA3E0C39FEC9E22
:105AE2004003025CF1901D4EE0FEA3E0FF90000235
:105AF200E0FCA3E09FEC9E4017E4901D4AF0A3F067
:105B0200900002E0FEA3E0FF901D4EEEF0A3EFF046
:105B1200900949E0641A703E900002E0FEA3E0643E
:105B2200014E7032900549E06478702A7B017A0553
:105B32007949C003C002C001901D45121C30A80162
:105B4200AC02AD03D001D002D0037E007F01121659
:105B5200DF7E007F0122900949E064A1600DE064CC
:105B62000A704690094DE064A1703E900002E0FE8A
:105B7200A3E064014E7032900549E06478702A7B9C
:105B8200017A057949C003C002C001901D45121C6B
:105B920030A801AC02AD03D001D002D0037E007F59
:105BA200011216DF7E007F0122900949E064A260A3
:105BB2000DE0640A704690094DE064A2703E9000C8
:105BC20002E0FEA3E064014E7032900549E0647881
:105BD200702A7B017A057949C003C002C001901D79
:105BE20045121C30A801AC02AD03D001D002D00393
:105BF2007E007F011216DF7E007F0122900002E00C
:105C0200FEA3E0D39400EE94005003025CD890050A
:105C120049E0547864786003025CD8E05407FF904E
:105C22001D48E4F0A3EFF0901D48E0FEA3E06407F6
:105C32004E7053900002E0FEA3E0D39401EE940074
:105C4200404490054AE02403FFE433901D48F0A34A
:105C5200EFF0901D48E0A3E030E735900002E0FE4F
:105C6200A3E0D39402EE9400402690054AE0547FCC
:105C7200FEA3E02404FDE4334EFEEDFF901D48EE4A
:105C8200F0A3EFF0800A901D48E475F00212184F5D
:105C9200901D48E0FEA3E0FF900002E0FCA3E0B507
:105CA2000734ECB50630901D48E0A3E07B017A058D
:105CB2007949C003C002C001901D45121C30A801E1
:105CC200AC02AD03D001D002D0031216DF901D4802
:105CD200E0FEA3E0FF227F0012B3E87F647E0012A1
:105CE200ACA7901D4AE475F00112184F025ACF90EA
:105CF2001D4CE0FEA3E0FF901D4AE0FCA3E0B507C7
:105D020014ECB50610901D45121C3074FF12177E5C
:085D12007E007F0122E4FEFF88
:015D1A002266
:10AF46007B017A1A79D0C002C001E4901CE7F0A315
:10AF5600F0A37402F0A37411F0E4A3F07A0079135D
:10AF6600A3121C50901CEF7401F0A37413F0D001CF
:10AF7600D0027D997C0412A748901E55EFF0E0FFA1
:10AF86003395E0FE7C007D3D1217B2747B2FF97479
:10AF9600123EFA7B01A3121C507A017926C003C027
:10AFA60002C001901E56121C3090000E121CF89022
:10AFB6001E56121C30900011740475F00512198289
:01AFC6002268
:067B1800901CD2121C506B
:107B1E0090165DE0901CE1F0E070057EFF7F9D22E7
:107B2E00901CE1E0640A6005E0640B700990164D4C
:107B3E00121B7B128FE212C0F2901CD8EFF0E020E5
:107B4E00E103027C66E490127DF0A3F0FE7F04FD5B
:107B5E007B017A12797F1221D67E007F107D007B09
:107B6E00017A0079131221D67B017A1C79D912473A
:107B7E008D901CDFEEF0A3EFF07B007A007900C051
:107B8E0003C002C001901CD9121C30D082D083D009
:107B9E00E06B7008E965827003EA65837003FEFF8F
:107BAE0022901CD9121C30900013121CC8901CDCA1
:107BBE00121C50901CDC121C3012187B2406FFE4A1
:107BCE0035F0FE901CDFE0FCA3E06F7002EE6C60FF
:107BDE0004E4FEFF22901CDC121C309000051217EC
:107BEE001E64056014901CDC121C309000061217E7
:107BFE001E64616004E4FEFF22901CDC121C3090B7
:107C0E0000021218A6FF901CD9121C3090002CE511
:107C1E00F08FF0121982901CD9121C3090001312A2
:107C2E001CC8C003C002C001901CD2121C30121C12
:107C3E0079901CD9121C3090001C12171EFF901C3C
:107C4E00D5121C30EF12177E901CD9121C309000EA
:0B7C5E00191218A6FFAEF022E4FEFF92
:017C690022F8
:0B8DFB00901D74EFF0A3ECF0A3EDF06E
:108E0600901D74E0C3748094804009E094107480CF
:108E160094804004E4FEFF22901D75E0FEA3E0D39B
:108E26009406EE648094844004E4FEFF22901D7450
:108E3600E075F03DA4247BF9741235F0FA7B0190BD
:108E46001D77121C507A017926901D7A121C5090BB
:108E56001D7A121C309000057405121790901D752E
:108E6600E0FEA3E0FF901D7A121C30EE8FF012197F
:108E760063901D77121C3090002C1218A6FF901DCF
:108E86007A121C30900002E5F08FF0121982901DC4
:108E96007A121C30900004E4121790901D75E0FEC3
:108EA600A3E02406FFE43EFEA3121C30900011EE60
:108EB6008FF0121982901D77121C30127324901DA8
:108EC6007DEEF0A3EFF0901D7DE0FEA3E0C39406D7
:108ED600EE94005008901D7DE0A3E0FF22901D7DDA
:0B8EE600E0FEA3E024FAFFEE34FFFEE4
:018EF100225E
:10C52C00C208C203C205C206E4900002F0A3F012D6
:09C53C0054DC1291BA12C32F2243
:062AB700901B33121C50BD
:102ABD00901B33121C301217055407FF901B3FE477
:102ACD00F0A3EFF0901B3FE0FEA3E064074E7057BC
:102ADD00901B33121C3090000112171E30E72C9002
:102AED001B33121C3090000112171E547FFE901BD9
:102AFD0033121C3090000212171EFDEEED2404FF60
:102B0D00E43E901B3FF0A3EFF08026901B33121C88
:102B1D003090000112171E547F2403FFE433901BE5
:102B2D003FF0A3EFF0800A901B3FE475F0021218FE
:102B3D004F901B3FE0FEA3E024FFFDEE34FFFC9021
:102B4D001B33121C3012A163901B33121C30901BCF
:102B5D003FE0FCA3E024FFFDEC34FF8D82F58312F2
:102B6D00171E6F6004E4FEFF22E4901B3DF0A3F0FE
:102B7D00901B33121C3012170564B76003022DF839
:102B8D00901B3FE0FEA3E024F7FFEE34FFFEE4FCD4
:102B9D00FD901B45121BC3901B33121C309000037C
:102BAD0012171E901B49F0901B33121C309000041D
:102BBD0012171EFFE4FCFDFE901B41121BC3901B60
:102BCD0033121C3090000512171EFFE4FCFDFEC0F1
:102BDD0004C005C006C007901B41121B7B7808126C
:102BED001AFAA804A905AA06AB07D007D006D00586
:102BFD00D004121A98901B41121BC3901B33121C48
:102C0D003090000612171EFFE4FCFDFEC004C00547
:102C1D00C006C007901B41121B7B7808121AFAA838
:102C2D0004A905AA06AB07D007D006D005D004121B
:102C3D001A98901B41121BC3901B33121C3090002D
:102C4D000712171EFFE4FCFDFEC004C005C006C040
:102C5D0007901B41121B7B7808121AFAA804A905CC
:102C6D00AA06AB07D007D006D005D004121A98904B
:102C7D001B41121BC3901B41121B7B781C121AE7C0
:102C8D00E4FBFAF9F8C3121AD66003022DF4901B77
:102C9D0041121B7BEFEEEDEC540FFC901B41121B10
:102CAD00C3E4FF12C693901B49E0FF12BF93901B24
:102CBD0041121B7B7810121AE7EFEE540FFEE4FD64
:102CCD00FCFBFAF9F8C3121AD650427F1412AA5E11
:102CDD00901B41121B7B7818121AE7EFE412AA5EC3
:102CED00901B41121B7B7810121AE7EFE412AA5EBB
:102CFD00901B41121B7B7808121AE7EFE412AA5EB3
:102D0D00901B41121B7BEFE412AA5E804C901B417D
:102D1D00121B7B7808121AE7EFE4FEFDFCFBFAF9B3
:102D2D00F8C3121AD650227F1212AA5E901B4112BE
:102D3D001B7B7808121AE7EFE412AA5E901B411272
:102D4D001B7BEFE412AA5E80107F1112AA5E901B0E
:102D5D0041121B7BEFE412AA5EE4901B3BF0A3F043
:102D6D00901B3BE0FEA3E0FFE4FCFD901B45121B16
:102D7D0087D3121AD64029901B33121C30901B3B5F
:102D8D00E0FEA3E02408FFE43E8F82F58312171EB8
:102D9D00FF12AA5E901B3BE475F00112184F80C024
:102DAD007FFF12BF937F0112C693901B36121C300A
:102DBD00747812177E901B45121B7BAD07AC0690E5
:102DCD001B33121C30E92408F9E43AFA12A163907E
:102DDD001B36121C30900001EF121790901B3DE432
:102DED00F0A37402F08004E4FEFF22901B33121C4A
:102DFD003012170564BF6003023122901B33121C81
:102E0D003090000212171EFE901B33121C309000E2
:102E1D000312171EFDEEEDFFEE3395E0FDFC901B4A
:102E2D0045121BC3901B33121C3090000412171E49
:102E3D00901B49F0901B33121C3090000512171E89
:102E4D00FFE4FCFDFE901B41121BC3901B33121CB3
:102E5D003090000612171EFFE4FCFDFEC004C005F5
:102E6D00C006C007901B41121B7B7808121AFAA8E6
:102E7D0004A905AA06AB07D007D006D005D00412C9
:102E8D001A98901B41121BC3901B33121C309000DB
:102E9D000712171EFFE4FCFDFEC004C005C006C0EE
:102EAD0007901B41121B7B7808121AFAA804A9057A
:102EBD00AA06AB07D007D006D005D004121A9890F9
:102ECD001B41121BC3901B33121C309000081217AC
:102EDD001EFFE4FCFDFEC004C005C006C007901B2C
:102EED0041121B7B7808121AFAA804A905AA06AB91
:102EFD0007D007D006D005D004121A98901B4112A6
:102F0D001BC3901B45121B7BEF2404FBE43EFAE42C
:102F1D003DF9E43CF8901B39E0FEA3E0FFEE33955C
:102F2D00E0FDFCD3121AD64004E4FEFF22901B45AF
:102F3D00121B7B7D00901B36121C30E92403F9E433
:102F4D003AFA1221D6901B41121B7B781C121AE7FC
:102F5D00E4FBFAF9F8C3121AD6600302311E901B76
:102F6D0041121B7BEFEEEDEC540FFC901B41121B3D
:102F7D00C3E4FF12C693901B49E0FF12BF93901B51
:102F8D0041121B7B7810121AE7EFEE540FFEE4FD91
:102F9D00FCFBFAF9F8C3121AD650427F2412AA5E2E
:102FAD00901B41121B7B7818121AE7EFE412AA5EF0
:102FBD00901B41121B7B7810121AE7EFE412AA5EE8
:102FCD00901B41121B7B7808121AE7EFE412AA5EE0
:102FDD00901B41121B7BEFE412AA5E804C901B41AB
:102FED00121B7B7808121AE7EFE4FEFDFCFBFAF9E1
:102FFD00F8C3121AD650227F2212AA5E901B4112DC
:10300D001B7B7808121AE7EFE412AA5E901B41129F
:10301D001B7BEFE412AA5E80107F2112AA5E901B2B
:10302D0041121B7BEFE412AA5E901B45121B7BEF36
:10303D00E412AA5EE4901B3BF0A3F0901B3BE0FE74
:10304D00A3E0FFE4FCFD901B45121B87D3121AD69B
:10305D00402912A6A5901B36121C30901B3BE0FC9C
:10306D00A3E02403FDE43C8D82F583EF12179090CD
:10307D001B3BE475F00112184F80C07FFF12BF9308
:10308D007F0112C693901B36121C30747F12177E6F
:10309D00901B45121B7B7808121AE7EF547FFFE453
:1030AD00EF4480FFE4901B36121C30900001EF12AC
:1030BD001790901B45121B7BEFE4901B36121C30B2
:1030CD00900002EF121790901B45121B7BEF24030B
:1030DD00FDE43EFC901B36121C3012A163C007901C
:1030ED001B45121B7BEF2403FFE43EFE901B3612A3
:1030FD001C308F828E83D007EF121790901B4512D4
:10310D001B7BEF2404FFE43E901B3DF0A3EFF0800A
:0D311D0004E4FEFF22901B3DE0FEA3E0FF56
:01312A002282
:10BA01007B017A057949C002C0017A097949901B05
:10BA110036121C50901B397401F0A3740DF0D00143
:10BA2100D002122AB7901B31EEF0A3EFF0901B3138
:10BA3100E0FEA3E0D39400EE940040157A007B323F
:10BA41007D017F01129E6D901B31E0A3E0FF12B6D4
:01BA510007ED
:01BA520022D1
:0F00260090FFFD121D77121C5090FFF2121D77F4
:1000350090000E121D9B121C301217055407FF7EEF
:1000450000900005121D9BEEF0A3EFF09000051245
:100055001D9BE0FEA3E064074E707090000E121D1C
:100065009B121C3090000112171E30E73A90000ECB
:10007500121D9B121C3090000112171E547F7F0029
:10008500FE90000E121D9B121C3090000212171ECE
:10009500FDEEEF4D2404FFE43EFE900005121D9B8E
:1000A500EEF0A3EFF0803190000E121D9B121C3074
:1000B50090000112171E547F2403FFE433FE9000C5
:1000C50005121D9BEEF0A3EFF0800D900005121DAB
:1000D5009BE475F00212184F900005121D9BE0FE7F
:1000E500A3E024FFFDEE34FFFC90000E121D9B12D1
:1000F5001C3012A16390000E121D9B121C30900043
:1001050005121D9BE0FCA3E024FFFDEC34FF8D826E
:10011500F58312171E6F6006E4FEFF02123290008F
:1001250003121D9BE4F090000E121D9B121C301251
:100135001705121D5101650A023B1001E712016501
:100145001A025120025628042A2907113307D537E8
:1001550008475008E561064A7008E1980000093C27
:1001650090000E121D9B121C3090000112171E7F6D
:1001750000FE90000E121D9B121C309000021217FB
:100185001EFDEEEF4DFF9019BDE0FCA3E06F700280
:10019500EE6C7044D20890000604F07A007B32FDC4
:1001A5007F00129E6D90000E121D9B121C301217BF
:1001B50005641A600302093C900011121D9B121C74
:1001C50030900003121D9BE0FF04F08F82758300C1
:1001D500747812179002093CC208E4900006F002F8
:1001E500093C90000E121D9B121C30900001121745
:1001F5001E7F00FE90000E121D9B121C3090000207
:1002050012171EFDEEEF4DFF9019BFE0FCA3E0B500
:10021500071AEEB50416D2089000067402F07A00AB
:100225007B327D017F00129E6D02093CC208E4907D
:100235000006F002093CD2089000067403F07A002B
:100245007B327D017F00129E6D02093CD2050209B9
:100255003C900011121D9B121C30900003121D9B37
:10026500E0FF04F08F82758300747F121790900071
:1002750011121D9B121C30900003121D9BE0FF0400
:10028500F08F827583007418121790900011121D5B
:100295009B121C30900003121D9BE0FF04F08F821F
:1002A5007583007405121790900541E0FF900011C9
:1002B500121D9B121C30900003121D9BE0FE04F0E2
:1002C5008E82758300EF1217909019BDE0FEA3E0B2
:1002D500EEFF900011121D9B121C30900003121DA1
:1002E5009BE0FE04F08E82758300EF121790901943
:1002F500BDE0A3E0FF900011121D9B121C30900081
:1003050003121D9BE0FE04F08E82758300EF121729
:10031500909019BFE0FEA3E0EEFF900011121D9B27
:10032500121C30900003121D9BE0FE04F08E8275B6
:100335008300EF1217909019BFE0A3E0FF90001122
:10034500121D9B121C30900003121D9BE0FE04F051
:100355008E82758300EF121790786FE6FE08E6EE41
:10036500FF900011121D9B121C30900003121D9B63
:10037500E0FE04F08E82758300EF121790786FE629
:1003850008E6FF900011121D9B121C30900003120D
:100395001D9BE0FE04F08E82758300EF1217908599
:1003A5001283851382E4F0851283851382E0C3945A
:1003B50010748094805033E024C1F582E43419F53B
:1003C50083E0FF900011121D9B121C309000031258
:1003D5001D9BE0FE04F08E82758300EF1217908559
:1003E5001283851382E004F080BD900003121D9BEB
:1003F500E0FD7C00900011121D9B121C3012A163C0
:10040500900011121D9B121C30900003121D9BE0E1
:10041500F582758300EF121790900003121D9BE083
:1004250004F002093C90000E121D9B121C30900036
:100435000112171EFF900541E0FEEFC39E40030227
:0204450006208F
:1004470090000E121D9B121C3090000112171E7592
:10045700F010A4FF9019B6121C30E92FF9EA35F015
:10046700FA90000B121D9B121C50900011121D9B3D
:10047700121C30900003121D9BE0FF04F08F827561
:100487008300747F121790900011121D9B121C306D
:10049700900003121D9BE0FF04F08F8275830074A8
:1004A7000D12179090000B121D9B121C301217058E
:1004B700FF900011121D9B121C30900003121D9B10
:1004C700E0FE04F08E82758300EF12179090000B08
:1004D700121D9B121C3090000112171EFF90001175
:1004E700121D9B121C30900003121D9BE0FE04F0AE
:1004F7008E82758300EF12179090000B121D9B12CE
:100507001C3090000212171EFF900011121D9B1243
:100517001C30900003121D9BE0FE04F08E82758351
:1005270000EF12179090000B121D9B121C309000C9
:100537000312171EFF900011121D9B121C30900012
:1005470003121D9BE0FE04F08E82758300EF1217E5
:100557009090000B121D9B121C3090000412171E66
:10056700FF900011121D9B121C30900003121D9B5F
:10057700E0FE04F08E82758300EF121790851283D8
:10058700851382E4F0851283851382E0C39408748F
:10059700809480504990000B121D9B121C30E92457
:1005A70005F9E43AFA851283851382E07E0029F97A
:1005B700EE3AFA121705FF900011121D9B121C301C
:1005C700900003121D9BE0FE04F08E82758300EFFE
:1005D700121790851283851382E004F080A790009C
:1005E70003121D9BE0FD7C00900011121D9B121C45
:1005F7003012A163900011121D9B121C3090000352
:10060700121D9BE0F582758300EF1217909000038F
:06061700121D9BE004F03F
:10061D0002093C900011121D9B121C3074781217A8
:10062D007E900011121D9B121C30900001E41217D8
:10063D0090900003121D9B7402F002093C12C256E9
:10064D00900007121D9B121BC3900011121D9B12CF
:10065D001C30747C12177E900007121D9BE0FF90DA
:10066D000011121D9B121C30900001EF1217907B90
:10067D0001900007121D9BA982AA839000011217F9
:10068D001EFF900011121D9B121C30900002EF12E4
:10069D0017907B01900007121D9BA982AA839000E1
:1006AD000212171EFF900011121D9B121C3090009C
:1006BD0003EF1217907B01900007121D9BA982AAD0
:1006CD008390000312171EFF900011121D9B121C28
:1006DD0030900004EF1217907C007D0590001112F0
:1006ED001D9B121C3012A163900011121D9B121C38
:1006FD0030900005EF121790900003121D9B7406A9
:10070D00F002093C90000E121D9B121C309000014E
:10071D0012171E6401703090000E121D9B121C30BA
:10072D0090000212171E7F00FE90000E121D9B12EC
:10073D001C3090000312171EFDEEEF4DFF9019BDFA
:10074D00EEF0A3EFF0807C90000E121D9B121C307A
:10075D0090000112171E6402702890000E121D9B4E
:10076D00121C3090000212171EFF7F0090000E1217
:10077D001D9B121C3090000312171E4F9019BDF0D7
:10078D00804190000E121D9B121C3090000112171B
:10079D001E6403702E90000E121D9B121C309000D3
:1007AD000212171E7F00FE90000E121D9B121C30B0
:1007BD0090000312171EFDEEEF4DFF9019BFEEF0E6
:1007CD00A3EFF0D20402093C851283851382E4F075
:1007DD00851283851382E0C39410748094805050E9
:1007ED0090000E121D9B121C3090000112171EFF5F
:1007FD00851283851382E0C39F5035E02402FFE408
:10080D0033FE90000E121D9B121C308F828E8312B0
:10081D00171EFF851283851382E024C1F582E4340F
:10082D0019F583EFF0851283851382E004F080A023
:10083D00E49019D0F0D20402093C20064D9000112D
:10084D00121D9B121C30747912177E900011121D0F
:10085D009B121C3090000174011217907C007D02D8
:10086D00900011121D9B121C3012A16390001112E9
:10087D001D9B121C30900002EF1217909000031276
:10088D001D9B7403F0D20302093C900011121D9BB5
:10089D00121C30747912177E900011121D9B121CC0
:1008AD003090000174021217907C007D02900011AF
:1008BD00121D9B121C3012A163900011121D9B1270
:1008CD001C30900002EF121790900003121D9B74C4
:1008DD0003F0805BD2048057900011121D9B121CF7
:1008ED0030747912177E90000E121D9B121C3090E1
:1008FD00000112171EFF900011121D9B121C30904B
:10090D000001EF1217907C007D02900011121D9BCB
:10091D00121C3012A163900011121D9B121C3090FD
:10092D000002EF121790900003121D9B7403F090BC
:10093D00000E121D9B121C3012170554F864A06096
:10094D0003020EE190000E121D9B121C30121705B2
:10095D0064A16003020C0590000E121D9B121C3049
:10096D0090000112171EFF900004121D9BEFF090D6
:10097D000541E0FF900004121D9BE0C39F40030260
:10098D000BEB9019B6121C30900004121D9BE075F4
:10099D00F010A4F58285F08312171EFF900003124C
:1009AD001D9BEFF0900004121D9BE075F010A4FF4D
:1009BD009019B6121C30E92FF9EA35F0FA900004BF
:1009CD0012171E20E203020A64900011121D9B12E1
:1009DD001C30747F12177E900011121D9B121C305B
:1009ED00E92402F9E43AFA900004121D9BE0FF128B
:1009FD009A6F900003121D9BEFF0900003121D9B48
:100A0D00E0FF900011121D9B121C30900001EF129F
:100A1D001790900003121D9BE02402F0900003122A
:100A2D001D9BE0FD7C00900011121D9B121C3012CD
:100A3D00A163900011121D9B121C30900003121D1A
:100A4D009BE0F582758300EF121790900003121D45
:100A5D009BE004F0020EE1900003121D9BE0D39485
:100A6D0006748094805003020B1D900011121D9B83
:100A7D00121C30747F12177E900003121D9BE0FF35
:100A8D00900011121D9B121C30900001EF12179057
:100A9D00851283851382E4F0900003121D9BE0FF05
:100AAD00851283851382E0C39F5058900004121D58
:100ABD009BE075F010A4FF9019B6121C30E92FF9C8
:100ACD00EA35F0FA90000D121CC885128385138249
:100ADD00E0F58275830012171EFF85128385138240
:100AED00E02402FDE433FC900011121D9B121C301A
:100AFD008D828C83EF121790851283851382E0040B
:100B0D00F08095900003121D9BE02402F0020BB0C3
:100B1D00900003121D9BE02478FF900011121D9B85
:100B2D00121C30EF12177E851283851382E4F0902C
:100B3D000003121D9BE0FF851283851382E0C39F86
:100B4D005058900004121D9BE075F010A4FF9019F1
:100B5D00B6121C30E92FF9EA35F0FA90000D121C8F
:100B6D00C8851283851382E0F58275830012171EE6
:100B7D00FF851283851382E02401FDE433FC900090
:100B8D0011121D9B121C308D828C83EF12179085D4
:100B9D001283851382E004F08095900003121D9B53
:100BAD00E004F0900003121D9BE0FD7C009000110D
:100BBD00121D9B121C3012A163900011121D9B126D
:100BCD001C30900003121D9BE0F582758300EF121F
:100BDD001790900003121D9BE004F0020EE19000AF
:100BED0011121D9B121C30747812177E9000031287
:100BFD001D9B7401F0020EE190000E121D9B121C44
:100C0D003012170564A26003020EE190000E121D52
:100C1D009B121C3090000112171EFF900541E0FE43
:100C2D00EFC39E4003020ECA90000E121D9B121CB4
:100C3D003090000212171EFF900541E0FEEFC39E9B
:100C4D004003020ECA90000E121D9B121C30900024
:100C5D000212171EFF90000E121D9B121C309000E9
:100C6D000112171ED39F4003020ECA90000E121DD3
:100C7D009B121C3090000112171E85128385138262
:100C8D00F0A3A3E4F090000E121D9B121C309000F7
:100C9D000212171EFF851283851382E0D39F5030F9
:100CAD009019B6121C30851283851382E075F010F1
:100CBD00A4F58285F08312171EFF8512838513829A
:100CCD00A3A3E02FF0851283851382E004F080B595
:100CDD00900003121D9BE4F0900011121D9B121C3D
:100CED0030900003121D9BE0FF04F08F827583008E
:100CFD00747F121790851283851382A3A3E0C3948A
:100D0D0080748094805028851283851382A3A3E07C
:100D1D00FF900011121D9B121C30900003121D9BA1
:100D2D00E0FE04F08E82758300EF121790804F85E0
:100D3D001283851382A3A3E0E47480FF9000111247
:100D4D001D9B121C30900003121D9BE0FE04F08EC3
:100D5D0082758300EF121790851283851382A3A3EA
:100D6D00E0FF900011121D9B121C30900003121D0C
:100D7D009BE0FE04F08E82758300EF1217909000B9
:100D8D000E121D9B121C3090000112171E8512832E
:100D9D00851382F090000E121D9B121C30900002E4
:100DAD0012171EFF851283851382E0D39F40030225
:100DBD000E90A3E4F09019B6121C308512838513A2
:100DCD0082E075F010A4F58285F08312171EFF8561
:100DDD001283851382A3E0C39F4003020E84851204
:100DED0083851382E075F010A4FF9019B6121C30A4
:100DFD00E92FF9EA35F0FA90000412171E30E21EC1
:100E0D00900011121D9B121C30900003121D9BE0CF
:100E1D00FF04F08F82758300E4121790804C8512C9
:100E2D0083851382E075F010A4FF9019B6121C3063
:100E3D00E92FF9EA35F0FA90000D121CC8851283DE
:100E4D00851382A3E0F58275830012171EFF9000B3
:100E5D0011121D9B121C30900003121D9BE0FE040D
:100E6D00F08E82758300EF121790851283851382A1
:100E7D00A3E004F0020DC2851283851382E004F015
:100E8D00020DA1900003121D9BE0FD7C009000114E
:100E9D00121D9B121C3012A163900011121D9B128A
:100EAD001C30900003121D9BE0F582758300EF123C
:100EBD001790900003121D9BE004F0801790001115
:100ECD00121D9B121C30747812177E900003121D98
:100EDD009B7401F090000E121D9B121C3012170511
:100EED0054F86480601590000E121D9B121C301278
:100EFD00170554F86488600302122890000E121D25
:100F0D009B121C301217055407FF900003121D9BF6
:100F1D00EFF0900003121D9BE06407703B85128378
:100F2D00851382A304F090000E121D9B121C3090AD
:100F3D00000112171EFF900003121D9BEFF0900091
:100F4D000E121D9B121C3090000212171EFF9000F6
:100F5D0004121D9BEFF08021851283851382A3E47B
:100F6D00F090000E121D9B121C3090000112171EE6
:100F7D00FF900004121D9BEFF0900003121D9BE0EB
:100F8D0014F0900541E0FF900004121D9BE0C39FFB
:100F9D0040030212289019B6121C30900004121D45
:100FAD009BE075F010A4F58285F08312171EFF905B
:100FBD000003121D9BE0D39F40229019B6121C30E6
:100FCD00900004121D9BE075F010A4F58285F0834E
:100FDD0012171EFF900003121D9BEFF085128385E3
:100FED001382E4F0900003121D9BE0FF85128385B0
:100FFD001382E0C39F40030211BA900004121D9B9F
:10100D00E075F010A4FF9019B6121C30E92FF9EA23
:10101D0035F0FA90000412171E30E2030211AE9063
:10102D000004121D9BE075F010A4FF9019B6121C60
:10103D0030E92FF9EA35F0FA90000112171E6438E5
:10104D006003021125900003121D9BE0D3940474DC
:10105D00809480405F851283851382A3E02402FF74
:10106D00E433FE851283851382E07C002FFFEC3E76
:10107D00FE90000E121D9B121C308F828E83121754
:10108D001EFD900004121D9BE075F010A4FF901939
:10109D00B6121C30E92FF9EA35F0FA90000D121C4A
:1010AD00C8851283851382E0F582758300ED1217D2
:1010BD00900211AE900005121D9BE0FEA3E024FEF0
:1010CD00FFEE34FFFE851283851382E0FDC3EF9D95
:1010DD00FFEE9400FE90000E121D9B121C308F82AD
:1010ED008E8312171EFD900004121D9BE075F010EB
:1010FD00A4FF9019B6121C30E92FF9EA35F0FA90D9
:10110D00000D121CC8851283851382E0F58275834C
:10111D0000ED1217900211AE9019B6121C3090000E
:10112D0004121D9BE075F010A4F58285F083121753
:10113D001EFF7E00900005121D9BE0FCA3E024FF26
:10114D00FDEC34FFFCC3ED9FFFEC9EFE8512838505
:10115D001382E07C002FFFEC3EFEA3E02FFFEC3E60
:10116D00FE90000E121D9B121C308F828E83121763
:10117D001EFD900004121D9BE075F010A4FF901948
:10118D00B6121C30E92FF9EA35F0FA90000D121C59
:10119D00C8851283851382E0F582758300ED1217E1
:1011AD0090851283851382E004F0020FF190000EFA
:1011BD00121D9B121C30900004121D9BE0FF129C0F
:1011CD001A90000E121D9B121C3012170554F86454
:1011DD00887048900011121D9B121C3074781217E4
:1011ED007E90000E121D9B121C30900005121D9B4F
:1011FD00E0FEA3E024FFFFEE34FF8F82F58312178C
:10120D001EFF900011121D9B121C30900001EF1259
:10121D001790900003121D9B7402F0900003121D95
:05122D009BE0FF7E00C4
:07123200900014121D772249
:10312B0012C6E1EF4E60142007117B007A00790084
:10313B007F807EF47DFF7CFF12BFC890165DE0643C
:10314B0009700B12C6E1EF4E6004D2078002C20772
:10315B00300719900012E070137D01FF12B9AD7D9D
:10316B00017F0012A3679000127401F020071990E1
:10317B000012E060137D007F0012B9AD7D017F006E
:10318B0012A367E4900012F07B017A1C7940C00215
:10319B00C0017A1C7950901CD5121C50D001D00262
:1031AB00127B18901C4CEEF0A3EFF0D39400EE942E
:1031BB00005003023660901C40121C30901C5112C0
:1031CB001C507B017A01792C901C43121C509000EF
:1031DB0000E0FEA3E04E605D901C50E0FF3395E0F5
:1031EB00FE90127D75F03DEF121C24EE75F03DA4A0
:1031FB002583F583E0FEA3E0FF900000E0FCA3E055
:10320B006F7002EC6E6003023670901C50E0FF335F
:10321B0095E0FE7C007D3D1217B2747F2FF974127E
:10322B003EFA78427C057D017E007F041221B2EFCD
:10323B006003023670900000E0FEA3E04E606790E2
:10324B001C50E0FF3395E0FE90127D75F03DEF12C0
:10325B001C24EE75F03DA42583F583E0FEA3E0FF6F
:10326B00900000E0FCA3E06F7002EC6E7038901CD5
:10327B0050E0FF3395E0FE7C007D3D1217B2747F6A
:10328B002FF974123EFA7B0178427C057D017E009A
:10329B007F041221B2EF3395E04F700A900546740C
:1032AB0003F0A374E8F0901C4CE0FEA3E0D394135E
:1032BB00EE94014003023670901C51121C30E9242D
:1032CB0006F9E43AFA901C48121C50901C51121C3F
:1032DB003090000412171E5410D394007480948005
:1032EB0040047F0180027F00901C47EFF0901C513F
:1032FB00121C3012187BFF901C4EE5F0F0A3EFF080
:10330B00901C51121C3090000412171E901C46F09A
:10331B00901C4EE0FEA3E02406FFE43EFE901C4C06
:10332B00E0FCA3E06F7002EE6C6003023670901C41
:10333B0051121C3090000512171E64056010901C72
:10334B0048121C30121705646160030236707A0054
:10335B007B327D017F00129E6D901C47E060539085
:10336B001C50E0FF901C48121C30C003C002C0016F
:10337B00901C43121C30901CF6121C50D001D00232
:10338B00D00312621B901C4CE4F0A3EFF0901C4C8A
:10339B00E0FEA3E0D39400EE94005003023660905D
:1033AB001C50E0FF901C4CE0FCA3E0FD128DFB02D7
:1033BB003660901C48121C3012170564B7600D90D4
:1033CB001C48121C3012170564BF7055901C481214
:1033DB001C30C003C002C001901C43121C30901B58
:1033EB0036121C50901B397404F0A3E4F0D001D0BA
:1033FB0002D003122AB7901C4CEEF0A3EFF0901CF6
:10340B004CE0FEA3E0D39400EE9400500302367020
:10341B00901C50E0FF901C4CE0FCA3E0FD128DFBD8
:10342B0022901C43121C3090FFFD121D77121C5072
:10343B00901C48121C30120026901C4CEEF0A3EF8F
:10344B00F0901C4CE0FEA3E0D39400EE94004010EF
:10345B00901C50E0FF901C4CE0FCA3E0FD128DFB98
:10346B00200803023553901C48121C3012170554C8
:10347B00072402901C4BF0E0FF901C4EE0FCA3E0F5
:10348B00D39FEC94005003023553901C4BE0901CDF
:10349B0049E48FF012184FD206901C48121C3012C0
:1034AB00170564B7600D901C48121C301217056489
:1034BB00BF7054901C48121C30C003C002C0019056
:1034CB001C43121C30901B36121C50901B39740479
:1034DB00F0A3E4F0D001D002D003122AB7901C4C19
:1034EB00EEF0A3EFF0901C4CE0FEA3E0D39400EEC3
:1034FB0094004010901C50E0FF901C4CE0FCA3E0AB
:10350B00FD128DFBC20622901C43121C3090FFFD56
:10351B00121D77121C50901C48121C301200269062
:10352B001C4CEEF0A3EFF0901C4CE0FEA3E0D39408
:10353B0000EE94004010901C50E0FF901C4CE0FCFF
:10354B00A3E0FD128DFBC206300803023604901C6B
:10355B004EE0FEA3E0FF901C48121C3078497C091A
:10356B007D011216DFD206901C4EE0A3E0FF901CEB
:10357B0046E0FD129552EF607C900005E060077FFE
:10358B000012B3E880F3901C46E0FF901C43121C22
:10359B0030125A79901C4CEEF0A3EFF0901C4CE0DB
:1035AB00FEA3E0D39400EE94004032901C4CE0A3B9
:1035BB00E064014E700C901C43121C30121705F482
:1035CB00600B7A007B327D017F01129E6D901C5047
:1035DB00E0FF901C4CE0FCA3E0FD128DFB90094931
:1035EB00E06410701090094BE064397008A3E0FDA3
:1035FB00E4FF12BAA2C206805C900006E06402608F
:10360B0005E06403704F901C4EE0FEA3E0FF901C9E
:10361B0048121C3078497C097D011216DFD20690C6
:10362B001C4EE0A3E0FF901C46E0FD12955290006B
:10363B0005E060077F0012B3E880F3900949E0646E
:10364B0010701090094BE064397008A3E0FDE4FFA3
:10365B0012BAA2C20630050D7F647E0012BEB0E422
:05366B00F58475EF106D
:013670002237
:10C58E0075840FC2E8C2E9C2EAD2DBD2D9D2DAC2CE
:06C59E00ECC2EED2EB221C
:10C03000901B53EFF0A3EDF075840FE0701BC2D995
:10C04000901B53E01392E8E0FFC313F0E01392E972
:10C05000E0FFC313F0E01392EA901B54E024FF9238
:02C06000DA22E2
:05BC6A00901EA4EFF0A4
:10BC6F0075840FE4A3F0901EA5E0C394087480942C
:10BC7F0080502A901EA4E054019400748094804058
:10BC8F0003D38001C392D9901EA4E0FFC313F0D257
:0FBC9F00DBD2DBD2DBC2DBA3E004F080C9C2D969
:01BCAE002273
:05A9C600901B53EFF0AF
:10A9CB0075840FE0F526E5263392D9E52625E0F5CB
:10A9DB0026D2DBD2DBD2DBC2DB3392D9E52625E0F4
:10A9EB00F526D2DBD2DBD2DBC2DB3392D9E52625CF
:10A9FB00E0F526D2DBD2DBD2DBC2DB3392D9E52604
:10AA0B0025E0F526D2DBD2DBD2DBC2DB3392D9E5F4
:10AA1B002625E0F526D2DBD2DBD2DBC2DB3392D9A3
:10AA2B00E52625E0F526D2DBD2DBD2DBC2DB339287
:10AA3B00D9E52625E0F526D2DBD2DBD2DBC2DB3330
:10AA4B0092D9E52625E0F526D2DBD2DBD2DBC2DBC1
:02AA5B00C2D95E
:01AA5D0022D6
:10A6020075840FE4901B3FF0E0FF25E0FFA2D8E441
:10A61200334FF0D2DBD2DBD2DBC2DBE0FF25E0FF3F
:10A62200A2D8E4334FF0D2DBD2DBD2DBC2DBE0FFD5
:10A6320025E0FFA2D8E4334FF0D2DBD2DBD2DBC27B
:10A64200DBE0FF25E0FFA2D8E4334FF0D2DBD2DB20
:10A65200D2DBC2DBE0FF25E0FFA2D8E4334FF0D229
:10A66200DBD2DBD2DBC2DBE0FF25E0FFA2D8E433A2
:10A672004FF0D2DBD2DBD2DBC2DBE0FF25E0FFA270
:10A68200D8E4334FF0D2DBD2DBD2DBC2DBE0FF25F2
:10A69200E0FFA2D8E4334FF0D2DBD2DBD2DBC2DB65
:02A6A200E0FFD7
:01A6A4002293
:10C35100901EA6EFF0A3EDF0901EA6E0FFE4FD1203
:10C36100C030901EA7E0FF12BC6A0DE4FF12C0307E
:01C3710022A9
:10C37200901EA8EFF0A3EDF0901EA8E0FFE4FD12DE
:10C38200C030901EA9E0FF12A9C60DE4FF12C03012
:01C392002288
:0EC69300901B4AEFF075840FE024FF92EB221B
:05BCAF00901EAAEFF059
:10BCB40075840FE4A3F0901EABE0C39408748094E1
:10BCC40080502A901EAAE05401940074809480400D
:10BCD40003D38001C392EE901EAAE0FFC313F0D2F7
:0FBCE400ECD2ECD2ECC2ECA3E004F080C9C2EECB
:01BCF300222E
:05AA5E00901B4AEFF01F
:10AA630075840FE0F526E5263392EEE52625E0F51D
:10AA730026D2ECD2ECD2ECC2EC3392EEE52625E002
:10AA8300F526D2ECD2ECD2ECC2EC3392EEE52625DD
:10AA9300E0F526D2ECD2ECD2ECC2EC3392EEE52612
:10AAA30025E0F526D2ECD2ECD2ECC2EC3392EEE503
:10AAB3002625E0F526D2ECD2ECD2ECC2EC3392EEB2
:10AAC300E52625E0F526D2ECD2ECD2ECC2EC3392AB
:10AAD300EEE52625E0F526D2ECD2ECD2ECC2EC333F
:10AAE30092EEE52625E0F526D2ECD2ECD2ECC2ECD0
:02AAF300C2EEB1
:01AAF500223E
:10A6A50075840FE4901B4AF0E0FF25E0FFA2EFE47C
:10A6B500334FF0D2ECD2ECD2ECC2ECE0FF25E0FF58
:10A6C500A2EFE4334FF0D2ECD2ECD2ECC2ECE0FFD7
:10A6D50025E0FFA2EFE4334FF0D2ECD2ECD2ECC28E
:10A6E500ECE0FF25E0FFA2EFE4334FF0D2ECD2EC33
:10A6F500D2ECC2ECE0FF25E0FFA2EFE4334FF0D24D
:10A70500ECD2ECD2ECC2ECE0FF25E0FFA2EFE433A3
:10A715004FF0D2ECD2ECD2ECC2ECE0FF25E0FFA288
:10A72500EFE4334FF0D2ECD2ECD2ECC2ECE0FF25F3
:10A73500E0FFA2EFE4334FF0D2ECD2ECD2ECC2EC66
:02A74500E0FF33
:01A7470022EF
:0BBF6200481DCCFFFFFFFFFFFFFFFFAB
:10B66E00E4901B33F0901B33E0C3940474809480F9
:10B67E005028E0FF7B087D0A12BEE9901B33E0FFE5
:10B68E00E4FBFD12BEE9901B33E0FFE4FB7D0112EB
:10B69E00BEE9901B33E004F080CB7FFF12BF937B9B
:10B6AE00017D017F0312970C7B017D027F031297B0
:10B6BE000C7B017D037F0312970CE4FF12C30DE494
:04B6CE00FF12C0C4E3
:01B6D2002255
:10BEE900901B50EFF0A3EDF0A3EBF0E4FD7F0112FE
:10BEF900C030901B50E05407FF25E04440FF12A9D1
:10BF0900C6901B51E0FF12A9C6901B52E0FF12A96F
:09BF1900C67D01E4FF12C03022D4
:08BE7500901E77EFF0A3EDF041
:10BE7D00E4FD7F0112C030901E77E05407FF25E0EE
:10BE8D004441FF12A9C6901E78E0FF12A9C612A662
:10BE9D0002901E79EFF07D01E4FF12C030901E7903
:02BEAD00E0FFB4
:01BEAF002270
:0B970C00901B4CEFF0A3EDF0A3EBF07E
:10971700901B4DE0C39408748094805007E4901B1D
:109727004FF0800D901B4F7401F0901B4DE024F813
:10973700F0901B4EE06039A3E0FF901B4CE025E062
:1097470024CCF582E4341DF583E5822FF582E435D8
:1097570083F583C083C082E0FF901B4DE0FEF87461
:1097670001088002C333D8FC4FD082D083F0803AFF
:10977700901B4FE0FF901B4CE025E024CCF582E4E2
:10978700341DF583E5822FF582E43583F583C083A5
:10979700C082E0FF901B4DE0FEF87401088002C311
:1097A70033D8FCF45FD082D083F0901B4FE0FF905A
:1097B7001B4CE025E024CCF582E4341DF583E582DB
:1097C7002FF582E43583F583E0FB901B4CE0FF9097
:0E97D7001B4FE070047D1480027D1512BEE968
:0197E5002261
:10C4AA00901EACEFF0A3EDF0901EACE0FFA3E0709D
:0BC4BA00047D1280027D1312BE75226B
:06BD3800901B33121C50A9
:10BD3E00E4901B36F0901B36E0C394107480948010
:10BD4E00502AE0FD901B33121C30901B36E0F5821A
:10BD5E0075830012171E20E0047B0180027B007F9A
:0CBD6E000212970C901B36E004F080C914
:01BD7A0022A6
:05BF9300901B4AEFF0D5
:10BF9800E4A3F0901B4BE0C3941074809480501F6E
:10BFA800E0FD901B4AE0FFA3E06F60047B01800284
:0FBFB8007B00E4FF12970C901B4BE004F080D449
:01BFC7002257
:0FC66600901B32EFF0E0FBE4FD7F0312970C22F4
:10C60A00E4FB7D017F0312970C7B017D017F0312FE
:03C61A00970C2258
:10C61D00E4FB7D027F0312970C7B017D027F0312E9
:03C62D00970C2245
:10C63000E4FB7D037F0312970C7B017D037F0312D4
:03C64000970C2232
:10C30D00901B34EFF0E05401FB7D047F0312970C7A
:10C31D00901B34E0FFC3135401FB7D057F0312977F
:02C32D000C22E0
:10C0C400901B34EFF0E020E0047B0180027B007DD4
:10C0D4000A7F0312970C901B34E0FFC31320E00483
:0EC0E4007B0180027B007D0B7F0312970C22F4
:0CB8AE00901B38EFF0A3EDF0A3121C502B
:10B8BA00E4FDFF12C030901B38E0FFC454F0FFA330
:10B8CA00E0540F4FFF12A9C6E4901B3EF0901B3DB7
:10B8DA00E0FFA3E0C39F501912A602901B3AE47539
:10B8EA00F001121C39EF12177E901B3EE004F08023
:08B8FA00DC7D01E4FF12C03007
:01B902002222
:10C39300901B33EFF0A3EDF0E4FDFF12C030901BD0
:10C3A30033E0FFC454F0FFA3E0540F4FFF12A9C6BC
:01C3B3002267
:080003007D01E4FF12C0302270
:0BC6BC00901B33EFF0E0FF12A9C62234
:10C1D500E4FD7F0712C393E4FD7F0D12C3937FFF38
:10C1E50012C6BC7FFF12C6BCE4FF12C6BCE4FF1238
:0BC1F500C6BC7F1512C6BC120003225E
:057DAA00901B31EFF019
:107DAF00E0FD7B017A1B7932901B3D7402F0FF12CC
:107DBF00B8AE901B32E0FEA3E0FFEEC4F854F0C85B
:107DCF0068FCEFC4540F48FDE41214DCE4FBFA79AD
:107DDF00207840121331E4FBFA7980784512143A77
:107DEF00901B34121BC3901B31E0121D517E0F00EC
:107DFF007E54017E6B037E84047E9D0500007EB45D
:107E0F00901B34121B7B7BCD7ACC794C78431213A9
:107E1F0031901B34121BC3E4FFFE7D207C41901B6D
:107E2F0034121B87121331E4FBFAF9783F12124018
:107E3F00128EF2E4FBFA7920784112143A901B3437
:107E4F00121BC38060901B34121B7BE4FBFAF97882
:107E5F0040121331901B34121BC38049901B3412F4
:107E6F001B7B7BCD7ACC79CC783D12143A901B34A6
:107E7F00121BC38030901B34121B7B7B8B7A2E79A5
:107E8F003A783F12143A901B34121BC38017901B81
:107E9F0034121B7B7B907AC279F5783E12143A909C
:107EAF001B34121BC3E4FFFE7DC87C42901B3412AF
:107EBF001B87121331E4FBFAF9783F121240128E2E
:107ECF00F2E4FBFA79C8784212143A901B34121B71
:077EDF00C3901B34121B7B52
:017EE6002279
:10F00000C2AF7584015398FC75FFDE75FFADE478DF
:10F0100015F618F6E4F584209848E47819F608F611
:0FF0200020983BC3781AE6948818E69413502F73
:10F02F0075260AD3E52694007480948040177527BF
:10F03F0001D3E52794007480948040050015278044
:05F04F00F0152680DE33
:10F05400781A06E61870C50680C2B28280B57814A4
:10F06400A699C298E6FF7E00641A600302F1BB7899
:10F0740019F608F620983BC3781AE6948818E694A3
:03F0840013502FF7
:10F0870075280AD3E5289400748094804017752961
:10F0970001D3E529940074809480400500152980E8
:05F0A700F0152880DED9
:10F0AC00781A06E61870C50680C220980302F01480
:10F0BC007815A699C298E47819F608F620983BC3FF
:0BF0CC00781AE6948818E69413502F81
:10F0D700752A0AD3E52A9400748094804017752B0B
:10F0E70001D3E52B940074809480400500152B8094
:05F0F700F0152A80DE87
:10F0FC00781A06E61870C50680C220980302F01430
:10F10C007815A699C298E47819F608F620983BC3AE
:0BF11C00781AE6948818E69413502F30
:10F12700752C0AD3E52C9400748094804017752DB4
:10F1370001D3E52D940074809480400500152D803F
:05F14700F0152C80DE34
:10F14C00781A06E61870C50680C220980302F014DF
:0AF15C007815A699C298D284C299D2
:10F16600752E14D3E52E9400748094804017752F65
:10F1760001D3E52F940074809480400500152F80FC
:05F18600F0152E80DEF3
:06F18B007599783099FD32
:10F1910075300AD3E530940074809480401775313E
:10F1A10001D3E531940074809480400500153180CD
:05F1B100F0153080DEC6
:10F1B600C28402F976EF64504E600302F2C67819F3
:10F1C600F608F620983BC3781AE6948818E6941356
:02F1D600502FB8
:10F1D80075320AD3E53294007480948040177533F1
:10F1E80001D3E53394007480948040050015338082
:05F1F800F0153280DE7D
:10F1FD00781A06E61870C50680C220980302F0142E
:0AF20D007815A699C298D284C29920
:10F21700753414D3E53494007480948040177535A1
:10F2270001D3E5359400748094804005001535803E
:05F23700F0153480DE3B
:08F23C007599793099FDC29922
:10F24400753614D3E536940074809480401775376E
:10F2540001D3E5379400748094804005001537800D
:05F26400F0153680DE0C
:08F269007599013099FDC2996D
:10F27100753814D3E538940074809480401775393B
:10F2810001D3E539940074809480400500153980DC
:05F29100F0153880DEDD
:06F29600E4F5993099FD3A
:10F29C00753A0AD3E53A9400748094804017753B14
:10F2AC0001D3E53B940074809480400500153B80AD
:05F2BC00F0153A80DEB0
:10F2C100C28402F9767814E6FF7E006401600302CD
:06F2D100F359D284C2993A
:10F2D700753C14D3E53C9400748094804017753DC9
:10F2E70001D3E53D940074809480400500153D806E
:05F2F700F0153C80DE73
:08F2FC007599783099FDC29963
:10F30400753E14D3E53E9400748094804017753F95
:10F3140001D3E53F940074809480400500153F803C
:05F32400F0153E80DE43
:06F32900E4F5993099FDA6
:10F32F0075400AD3E540940074809480401775416E
:10F33F0001D3E5419400748094804005001541800D
:05F34F00F0154080DE16
:10F35400C28402F976EF64024E600302F4837819E2
:10F36400F608F620983BC3781AE6948818E69413B6
:02F37400502F18
:10F3760075420AD3E5429400748094804017754321
:10F3860001D3E543940074809480400500154380C2
:05F39600F0154280DECD
:10F39B00781A06E61870C50680C220980302F0148E
:10F3AB007815A699C298E408F618E6FF13B3928273
:10F3BB00EF25E0FEC3E49400EE94F0502CE6FD7FC5
:10F3CB000025E0FEC394E05020ED20E023E4F5841B
:10F3DB0043B701758F03781BEEF608EFF6F5828EB7
:10F3EB0083F053B7F0F58F8004781676FFE4F5843D
:04F3FB00D284C2995D
:10F3FF00754414D3E5449400748094804017754588
:10F40F0001D3E54594007480948040050015458034
:05F41F00F0154480DE41
:08F424007599783099FDC29939
:10F42C00754614D3E5469400748094804017754754
:10F43C0001D3E54794007480948040050015478003
:05F44C00F0154680DE12
:08F451007816E6F5993099FDEB
:10F4590075480AD3E548940074809480401775492B
:10F4690001D3E549940074809480400500154980D2
:05F47900F0154880DEE3
:10F47E00C28402F9767814E66403600302F67078AB
:10F48E0019F608F620983BC3781AE6948818E69485
:03F49E0013502FD9
:10F4A100754A0AD3E54A9400748094804017754BDD
:10F4B10001D3E54B940074809480400500154B8086
:05F4C100F0154A80DE99
:10F4C600781A06E61870C50680C220980302F01462
:10F4D6007815A699C298E47819F608F620983BC3E1
:0BF4E600781AE6948818E69413502F63
:10F4F100754C0AD3E54C9400748094804017754D87
:10F5010001D3E54D940074809480400500154D8031
:05F51100F0154C80DE46
:10F51600781A06E61870C50680C220980302F01411
:10F526007817A699C2987815E6FF139282EF25E020
:10F53600FEC3E49400EE94F0400302F014E625E0E6
:10F54600FCC394E0400302F014E4F58443B701756C
:10F556008F017817E675F020A42400FFE5F03C78CB
:10F566001BF608A607E4F5847818F67818E6C3941F
:10F5760020748094805063E408F608F620983BC314
:0BF58600781AE6948818E69413502FC2
:10F59100754E0AD3E54E9400748094804017754FE0
:10F5A10001D3E54F940074809480400500154F808D
:05F5B100F0154E80DEA4
:10F5B600781A06E61870C50680C220980302F01471
:10F5C600781B0806E618860670010614F5828E83F7
:10F5D600E599F0C2987818068091E4F58453B7F05F
:08F5E600F58FF584D284C2996F
:10F5EE00755014D3E5509400748094804017755173
:10F5FE0001D3E5519400748094804005001551802C
:05F60E00F0155080DE44
:08F613007599783099FDC29948
:10F61B00755214D3E552940074809480401775533F
:10F62B0001D3E553940074809480400500155380FA
:05F63B00F0155280DE15
:06F64000E4F5993099FD8C
:10F6460075540AD3E5549400748094804017755518
:10F6560001D3E555940074809480400500155580CB
:05F66600F0155480DEE8
:10F66B00C28402F9767814E6FD7C00640460030220
:10F67B00F78F7819F608F620983BC3781AE694882A
:06F68B0018E69413502F55
:10F6910075560AD3E55694007480948040177557C7
:10F6A10001D3E5579400748094804005001557807C
:05F6B100F0155680DE9B
:10F6B600781A06E61870C50680C220980302F01470
:10F6C6007815A699C298E625E0781DF6087600E436
:10F6D6007816F67819F608F6781D0806E6188606EE
:10F6E60070010614F5828E83E493781626F6781A4E
:10F6F60006E618700106781AE6B400DC18E6B402CD
:05F70600D7D284C29976
:10F70B00755814D3E558940074809480401775593C
:10F71B0001D3E559940074809480400500155980FD
:05F72B00F0155880DE1E
:08F730007599783099FDC2992A
:10F73800755A14D3E55A9400748094804017755B09
:10F7480001D3E55B940074809480400500155B80CC
:05F75800F0155A80DEEF
:08F75D007816E6F5993099FDDC
:10F76500755C0AD3E55C9400748094804017755DE0
:10F7750001D3E55D940074809480400500155D809B
:05F78500F0155C80DEC0
:10F78A00C28402F976ED64054C600302F96A7819BD
:10F79A00F608F620983BC3781AE6948818E694137C
:02F7AA00502FDE
:10F7AC00755E0AD3E55E9400748094804017755F93
:10F7BC0001D3E55F940074809480400500155F8050
:05F7CC00F0155E80DE77
:10F7D100781A06E61870C50680C220980302F01454
:10F7E1007815A699C298E47819F608F620983BC3D3
:0BF7F100781AE6948818E69413502F55
:10F7FC0075600AD3E560940074809480401775613D
:10F80C0001D3E561940074809480400500156180FB
:05F81C00F0156080DE24
:10F82100781A06E61870C50680C220980302F01403
:0AF831007817A699C298D284C299F4
:10F83B00756214D3E56294007480948040177563ED
:10F84B0001D3E563940074809480400500156380B8
:05F85B00F0156280DEE3
:08F8600075997F3099FDC299F2
:10F86800756414D3E56494007480948040177565BA
:10F8780001D3E56594007480948040050015658087
:05F88800F0156480DEB4
:10F88D007599203099FD7815E625E0FC7817E67519
:10F89D00F020A42400FFE5F03C781DF608A607E44F
:10F8AD007816F67818F67818E6C39420748094804C
:04F8BD005053C29949
:10F8C100756614D3E566940074809480401775675B
:10F8D10001D3E5679400748094804005001567802A
:05F8E100F0156680DE59
:10F8E600781DE6FE08E6F5828E83E493F599309955
:10F8F600FD781D0806E618860670010614F5828E48
:0EF9060083E493781626F678180680A1C2993D
:10F91400756814D3E5689400748094804017756901
:10F9240001D3E569940074809480400500156980D2
:05F93400F0156880DE03
:08F939007816E6F5993099FDFE
:10F94100756A0AD3E56A9400748094804017756BD8
:10F9510001D3E56B940074809480400500156B80A1
:05F96100F0156A80DED4
:10F96600C284800C7814E664067005F58475EF1081
:0CF976007814E66407600302F014D2AFBE
:01F982002262
:1051E60046455F4343000134000000537461747503
:1051F60073000001195004180000015532340000F4
:10520600000000011951041800000155332E330027
:10521600000000011955041800000155352E300014
:10522600000000011959040800000154656D700062
:1052360000000001195D0132000000464542303091
:10524600000000011961013200000046454230317C
:10525600000000011962013200000046454230326A
:105266000000000119630132000000464542303358
:105276000000000119640132000000464542303446
:105286000000000119650132000000464542303534
:105296000000000119660132000000464542303622
:1052A6000000000119670132000000464542303710
:1052B60000000001196801320000004645423038FE
:1052C60000000001196901320000004645423039EC
:1052D60000000001196A01320000004645423130E3
:1052E60000000001196B01320000004645423131D1
:1052F60000000001196C01320000004645423132BF
:1053060000000001196D01320000004645423133AC
:1053160000000001196E013200000046454231349A
:1053260000000001196F0132000000464542313588
:1053360000000001197001320000004D61786366BB
:10534600670000011971013200000452737446505F
:1053560047410000000001320000045273744350BC
:1053660055000000000001320000045273744D41E4
:10537600580000000000013400000042504D6F64E8
:1053860065000001197201340000004174746E005A
:105396000000000119730137000004535049000052
:1053A60000000000000001340000005350495F5324
:1053B6004C540001197401340000004E31575465F5
:1053C6006D70000119750408000001315754656DB0
:1053D6007030300119760408000001315754656DAC
:1053E60070303101197A0408000001315754656D97
:1053F60070303201197E0408000001315754656D82
:105406007030330119820408000001315754656D6C
:105416007030340119860408000001315754656D57
:1054260070303501198A0408000001315754656D42
:1054360070303601198E0408000001315754656D2D
:105446007030370119920408000001315754656D18
:105456007030380119960408000001315754656D03
:1054660070303901199A0408000001315754656DEE
:1054760070313001199E0408000001315754656DE2
:105486007031310119A20408000001315754656DCD
:105496007031320119A60408000001315754656DB8
:1054A6007031330119AA0408000001315754656DA3
:1054B6007031340119AE0408000001315754656D8E
:1054C6007031350119B20000000000000000000034
:0654D600000000000000D0
:0DBF6D004319B6FF51EC4418880000000095
:1099990012C5F775840F75E104E4F5E275E34075C6
:1099A900A4FF75A5FF75A6FF75A7FF759DDE759EBA
:1099B9007F7580E0F590F5A075B0FF75D8FF75E863
:1099C900FF758A83F597F589F58475B71075840F46
:1099D900438901758D01758F01758E02901B31F0D8
:1099E900A3F0901B31E0FEA3E0C3EE9401500C906C
:1099F9001B31E475F00112184F80E7438902E490A6
:109A09001B31F0A3F0901B31E0FEA3E0FFE4FCFD65
:109A19007B507AC3F9F8D3121AC04011E589541062
:109A2900700B901B3175F00112184F80D875970291
:109A3900E4F58475A3D775A1B7C2847F0AFE12BE67
:109A4900B0C2857D08E4FF12BAA2D2BC12B4577A1B
:109A5900007B967D037F00129E6D7A007B967D03C5
:059A69007F01129E6D5B
:019A6E0022D5
:05A21300901B31EFF08B
:10A21800E0602DE4A3F0901B32E0C3941B7480949B
:10A22800805014E02461F582E43419F583E4F09059
:10A238001B32E004F080DFE4901971F0A3F0A3F082
:10A248009019507401F0E4901974F012C58E12B68A
:10A258006E12C1D57B017A19796112BD38E4FF12FB
:10A26800C693E4901B32F0901B32E0C394107480C4
:10A278009480501DE025E025E02476F582E4341929
:10A28800F583121BCFC479C000901B32E004F08024
:10A29800D612890B901975EFF090188C121BCF000D
:10A2A8000000007B007A0079007F00129C1AE4907D
:05A2B80019D3F0A3F032
:01A2BD00227E
:109C1A0090FFFD121D77121C5090FFFF121D77EF67
:079C2A00F090FFFE121D7710
:109C3100851283851382A3A3E07008901950E02454
:109C4100FF92DC851283851382A3A3E0641B7077E6
:109C5100900003121D9B121C301217055407851228
:109C610083851382F0A37402F0851283851382E049
:109C71006407701A900003121D9B121C30900001A2
:109C810012171E851283851382F0A37403F08512C7
:109C910083851382E014F0E0FF7E00900003121D23
:109CA1009B121C30851283851382A3E07C0029F965
:109CB100EC3AFA78107C197D011216DF8512838542
:109CC1001382E09019D5F0851283851382A3A3E056
:0C9CD1002490F582E43418F5837401F04F
:079CDD00900006121D772222
:109A6F0090FFFD121D77121C5090FFFF121D77EF14
:079A7F00F090FFFE121D77BD
:109A8600851283851382A3A3E06416601A85128368
:109A9600851382A3A3E06417600D85128385138264
:109AA600A3A3E064187012900003121D9B121C30D1
:109AB600E412177E7F01029B3E851283851382A3E3
:109AC600A3E0641B7070851283851382F0A3F08572
:109AD6001283851382E0FEA3E0C3EE9401504B90FF
:109AE60019D3E0FFA3E06F60419019D3E024D0F5CD
:109AF60082E43418F583E0FF900003121D9B121CCC
:109B060030851283851382E0FCA3E0F5828C83EF17
:109B16001217909019D3E004543FF08512838513F1
:109B260082E475F00112184F80A585128385138291
:089B3600E0A3E0FF80027F00C4
:079B3E00900006121D7722C2
:10938A00E4901B31F0901B31E0C3941074809480F8
:10939A00502DE02495F582E43418F583E060187BBB
:1093AA00017A19796112BD38901B31E02495F58252
:1093BA00E43418F583E4F0901B31E004F080C690A1
:1093CA0018A5E0600D901971E0FF12C666E49018C6
:1093DA00A5F09018A6E0600812C60AE49018A6F054
:1093EA009018A7E0600812C61DE49018A7F090181C
:1093FA00A8E0600812C630E49018A8F09018A9E016
:10940A00600D901972E0FF12C30DE49018A9F09054
:10941A0018AAE0600D901973E0FF12C0C4E4901816
:10942A00AAF09018ABE0603B901974E0FF12BF936A
:10943A00E4901B31F09019D5E0FF901B31E0C39FF7
:10944A005017E02410F582E43419F583E0FF12AADC
:10945A005E901B31E004F080DC7FFF12BF93E49042
:03946A0018ABF04C
:01946D0022DC
:10C2EA009019D4E0FF9019D3E0B50716A3E024D043
:10C2FA00F582E43418F5837458F09019D4E00454A4
:03C30A003FF022DF
:10A4B7007E007F167D007B017A1979BD1221D67E39
:10A4C700007F667D007B017A1979501221D6E4F569
:10A4D70084901B31F0A37480F0758F04901B31E0DA
:10A4E700FEA3E0AA06F97BFF78BD7C197D017E00FB
:10A4F7007F161216DF901B31E4F0A37496F0901BC1
:10A5070031E0FEA3E0AA06F97BFF78507C197D01B4
:10A517007E007F661216DFE4F58F9019D1E0FEA367
:10A52700E064347003EE6412602774FF9019BDF085
:10A53700A3F0A3F0A3F0FB7A5179E678C17C197DEB
:10A547000112200F9019D17412F0A37434F07F0117
:05A5570022D2017F008B
:01A55C0022DC
:10B0C20012C5F7C2AFE4F5847814F608768043B768
:10B0D20001758F0718E6FE08E6F5828E83E4F075A7
:10B0E2008F0518F60876807B017A1979BDC002189F
:10B0F200E6FE08E6AA06F8AC027D01D0027E007FD9
:10B10200161216DF781476000876967B017A197982
:10B1120050C00218E6FE08E6AA06F8AC027D01D08D
:10B12200027E007F6A1216DF53B7FEE4F58FD2AFBC
:05B132007F0A12C513A5
:01B1370022F5
:10BAF00012C577901888121B871219BCE47B0AFACA
:10BB0000F9F8D3121AD6503512C577901888121B3F
:10BB1000C37F03127DAA901951121BC37F04127DAB
:10BB2000AA901955121BC37F05127DAA90195912AC
:0DBB30001BC3E4FF127DAA90195D121BC318
:01BB3D0022E5
:108C0A00E4F58475EF02901B2F7464F0901B2FE03B
:108C1A00D39400748094804005E014F080EE129999
:108C2A0099C204C203C20012A4B7901B2FEFF0E04E
:108C3A00FF12A21312C52C7F0A12C513901B30749F
:108C4A0001F0FD7F0012B9AD7D017F0012A36720FC
:108C5A00010B7A007B327D017F00129E6D30040A7F
:108C6A00C20412B0C2D20112A4B730030CC2037FED
:108C7A000A7E0012BEB012F00030000512BA01C21C
:108C8A0000901B30E0601C12C256E47B05FAF9F82A
:108C9A00D3121AD6500DE4901B30F090189004F0BD
:108CAA0012938A7F0012B3E812BAF012938A12C2A0
:108CBA00EA12C577A804A905AA06AB0790188C1270
:108CCA001B7BEF2464FFE43EFEE43DFDE43CFCD361
:108CDA00121AD65003028C5912C57790188C121B9F
:108CEA00C37B017A197976127EE77A007B647D016B
:088CFA007F00129E6D028C59EF
:018D0200224E
:10C0620075840FD2DE7FF47E0112ACA7C2DE7F4B55
:10C072007E0012ACA720DD047F0180027F00901BAE
:10C082003EEFF07FF47E0112ACA7C2DE901B3EE0D1
:01C09200FFAE
:01C09300228A
:0CA2BE00901B40EFF0C2DED2DEE0602515
:10A2CA0075260FD3E526940074809480403C752748
:10A2DA0001D3E527940074809480400500152780F7
:05A2EA00F0152680DEE6
:10A2EF00752869D3E52894007480948040177529E8
:10A2FF0001D3E529940074809480400500152980CE
:05A30F00F0152880DEBE
:08A31400C2DE901B40E0602551
:10A31C00752A69D3E52A940074809480403C752B8F
:10A32C0001D3E52B940074809480400500152B809C
:05A33C00F0152A80DE8F
:10A34100752C0FD3E52C9400748094804017752DE3
:10A3510001D3E52D940074809480400500152D8073
:05A36100F0152C80DE68
:01A3660022D4
:05BBD600901B3EEFF0A2
:10BBDB00E4A3F0901B3FE0C394087480948050352D
:10BBEB00E0FF7E007401A807088005C333CE33CE77
:10BBFB00D8F9FF901B3EE0FDE4EF5DD39400748019
:10BC0B00948040047F0180027F0012A2BE901B3FF4
:05BC1B00E004F080BE12
:01BC20002201
:04AEC300C2DED2DE3B
:10AEC70075260AD3E5269400748094804017752769
:10AED70001D3E527940074809480400500152780EE
:05AEE700F0152680DEDD
:02AEEC00C2DEC4
:10AEEE0075280AD3E528940074809480401775293C
:10AEFE0001D3E529940074809480400500152980C3
:05AF0E00F0152880DEB3
:08AF1300A2DDE433901B40F0C5
:10AF1B00752A50D3E52A9400748094804017752BC2
:10AF2B0001D3E52B940074809480400500152B8091
:05AF3B00F0152A80DE84
:05AF4000901B40E0FF42
:01AF450022E9
:10BB3E00E4901B3FF0901B3EF0901B3EE0C3940838
:10BB4E0074809480503012AEC3EF6018901B3EE0AC
:10BB5E00FF7E007401A807088005C333CE33CED80C
:10BB6E00F9FF80047E007F00901B3FE04FF0901B9A
:0BBB7E003EE004F080C3901B3FE0FF9E
:01BB89002299
:10890B007F0012B3E8C2AF12C062901B33EFF0E0EE
:10891B007002FF227FCC12BBD67F9912BBD67F5A37
:10892B0012BBD67FA512BBD612BB3E901B34EFF009
:10893B007FF47E0112ACA7E49019D6F09019D6E023
:10894B00C394107480948040030289E07F0012B3BB
:10895B00E812C0627F0F12BBD6E4901B33F0901B62
:10896B0033E0C3940874809480502D12BB3E901B4F
:10897B0033E0FE9019D6E075F008A424D7F582E415
:10898B003419F583E5822EF582E43583F583EFF018
:10899B00901B33E004F080C69019D7E0901B35F0A4
:1089AB009019D6E075F008A424D7F582E43419F5B4
:1089BB0083E0F460207F9912BBD67F9612BBD67FE3
:1089CB006912BBD612BB3E901B34EFF09019D6E068
:1089DB0004F00289477F0A7E0012BEB012C0627F8C
:1089EB00CC12BBD67F9912BBD67F3C12BBD67FC3B2
:1089FB0012BBD612BB3E901B34EFF0D2AF7F0012EE
:078A0B00B3E89019D6E0FF6B
:018A12002241
:067EE700901B31121C503B
:107EED0012C6DB901B39EFF0E4901B36F09019D6DB
:107EFD00E0FF901B36E0C39F40030280077F001216
:107F0D00B3E812C062901B35EFF0E0701D901B318D
:107F1D00121C30901B36E075F004A4F58285F083B9
:107F2D00121C00C479C000027FFE7F5512BBD6E43F
:107F3D00901B34F0901B34E0C394087480948050EF
:107F4D002AE0FF901B36E075F008A424D7F582E4F3
:107F5D003419F583E5822FF582E43583F583E0FF4F
:107F6D0012BBD6901B34E004F080C97FBE12BBD685
:107F7D0012BB3E901B37EFF012BB3E901B38EFF05B
:107F8D0012C6DB901B39E06F7070901B38E0FE90CD
:107F9D001B37E0FDEEFCEDEC1214DCE4FBFA79AAE4
:107FAD007842121331E4FBFA79AA784412143A900C
:107FBD001B3A121BC3E4FFFE7D207C41901B3A123D
:107FCD001B87121331E4FBFAF9783F121240128E1F
:107FDD00F2E4FBFA7920784112143A901B31121C0D
:107FED0030901B36E075F004A4F58285F083121BEA
:107FFD0057901B36E004F0027EFA7F0012B3E812B0
:10800D00C062C2AF7FCC12BBD67F4412BBD6D2AFFB
:05801D007F0012B3E832
:01802200223B
:0300000002AAF65B
:10AAF600787FE4F6D8FD7512207513007581720211
:02AB0600AB435F
:05BF7A0042164B00001F
:10C27F0090166374FFF07E027F247D007B017A1697
:10C28F0079641221D67E007F167D007B017A1679A4
:04C29F004D0221D655
:0FBFC800901DDCEBF0A3EAF0A3E9F0A3121BC37A
:10BFD7007E007F047D007B017A1C792A1221D6908E
:10BFE700165D7401F0901DDCE0FBA3E0FAA3E0F915
:04BFF700A31243B698
:01BFFB002223
:10C41500E4FFFE90165DE060157407F07B007A007E
:0EC4250079007D007C001243C1E490165DF0AA
:01C4330022E6
:068FE200901DFF121BC3ED
:108FE80090165EE060030290BE90165DE0C394099F
:108FF80050030290BE7B007A007900901DFF124357
:10900800B6901E03EEF0A3EFF064014E70030290D9
:10901800B690165DE0B40A47E47B02FAF9F89016B8
:109028004DE0FCA3E0FDA3E0FEA3E0FF121A0690CA
:109038001655E0F8A3E0F9A3E0FAA3E0FBC3121A7F
:10904800D6701C901655E0FCA3E0FDA3E0FEA3E05B
:10905800FFE47B02FAF9F8121A06901655804C9034
:10906800165DE0B40B48E47B08FAF9F890164DE079
:10907800FCA3E0FDA3E0FEA3E0FF121A0690165938
:10908800E0F8A3E0F9A3E0FAA3E0FBC3121AD67054
:109098001D901659E0FCA3E0FDA3E0FEA3E0FFE469
:1090A8007B02FAF9F8121A06901659121BC3901689
:1090B8005D7409F08008901E03E4F0A304F0901E8C
:0690C80003E0FEA3E0FF3F
:0190CE00227F
:10946E0090165EE0600302955190165DE0C394097C
:10947E00500302955190164CE004F0700690164B76
:10948E00E004F090164BE07004A3E0646470289042
:10949E00164BF0A3F0901651E0FCA3E0FDA3E0FE06
:1094AE00A3E024FFFFEE34FFFEED34FFFDEC34FFAE
:1094BE00FC901651121BC3901655E0FCA3E0FDA3C1
:1094CE00E0FEA3E0FF901651E0F8A3E0F9A3E0FA66
:1094DE00A3E0FBD3121AD6506AE4FFFEFDFC9016F1
:1094EE0051E0F8A3A3A3E0C3121AD6700590165D3F
:1094FE00F022901659E0FCA3E0FDA3E0FEA3E0FFEE
:10950E00901651E0F8A3E0F9A3E0FAA3E0FBD31222
:10951E001AD6500790165D740BF022901655E0FC8B
:10952E00A3E0FDA3E0FEA3E0FF901651E0F8A3E058
:10953E00F9A3E0FAA3E0FBD3121AD6500690165DFB
:03954E00740AF0AC
:0195510022F7
:0B43B600E0FCA3E0FDA3E0FEA3E0FF9D
:0F43C100901B98EBF0A3EAF0A3E9F0A3121BC343
:1043D000E4901B9FF0A3F0A3F0A3F0901BAEF0A31A
:1043E000F090165DE07003024784E064076004E02B
:1043F000B40A10901BB07401F0A37416F0A3745F9C
:10440000F0800E901BB07401F0A3741AF0A374CC6A
:10441000F0901C92E4F0A37443F0A37411F0E4A3B1
:10442000F0A304F0A37416F0A37464F0A37402F074
:10443000A37424F0901BB0E0FBA3E0FAA3E0F97DA5
:10444000447C00124EB3901BA3EFF0C364809480B1
:104450005003024775E0FF3395E0FE7C007D3D127E
:1044600017B2747B2FF974123EFA901BA57401F0F9
:10447000A3EAF0A3E9F0901B9FE07002A3E06003C1
:10448000024765901BA4F0901B98E0FBA3E0FAA301
:10449000E0F9A3E0FCA3E0FDA3E0FEA3E0FF123FF0
:1044A000C8901BA8121BC3901BAEE0FCA3E0FDEC60
:1044B00090166CF0EDA3F0901BB0E0FBA3E0FAA324
:1044C000E0F97401901ACC6B7008E965827003EA18
:1044D0006583700790166304F08005E4901663F01E
:1044E0007B017A167964C003C002C001901BA5E06D
:1044F000FBA3E0FAA3E0F990000E121CF8901BA5B4
:10450000E0FBA3E0FAA3E0F9900011740275F02437
:10451000121982127324901BA1EEF0A3EFF09016F3
:104520005DE0B4070B901B9FE4F0A304F002474842
:10453000901BA4E02401FEE433901BACF0A3CEF06A
:10454000C3901BA1E0648094805015901BACE0FEEA
:10455000A3E0FF7C007D641217B212C4F902473950
:104560009016637401F07B017A167964901C1874BC
:1045700002F0A37424F0901BACE0FEA3E0FF7C00EB
:104580007D641217B2901C1AEEF0A3EFF0901BA3FB
:10459000E0FF127148901BA1EEF0A3EFF0D394005E
:1045A000EE64809480500302471B90166BE0FFE49A
:1045B000FCFDFE7808121AFAA804A905AA06AB07A2
:1045C00090166AE0FFEB4FFFEAFEE9FDE8FC780891
:1045D000121AFAA804A905AA06AB07901669E0FF0B
:1045E000EB4FFFEAFEE9FDE8FC7808121AFAA8048E
:1045F000A905AA06AB07901668E0FFEB4FFFEAFE9D
:10460000E9FDE8FC901BA8E0F8A3E0F9A3E0FAA319
:10461000E0FBC3121AD6600302471B901664E064E5
:1046200002600302471B90165DE024FD602324F91D
:10463000601F14601C240A600302470F12000EBFA3
:10464000020C90165D7403F012C43402472F024727
:104650000F12000EEF64056003024704782A7C1CE9
:104660007D017B017A167974FE7F041216DF12C475
:104670005212C48D127C6A901651121BC3901651AF
:10468000E0FCA3E0FDA3E0FEA3E0FF90164D121BAB
:10469000C312C43474FFFFFEFDFC901651E0F8A372
:1046A000E0F9A3E0FAA3E0FBC3121AD67007901654
:1046B0005E04F0803FE47B02FAF9F8901651E0FCCA
:1046C000A3E0FDA3E0FEA3E0FF121A069016551228
:1046D0001BC3E47B08FAF9F8901651E0FCA3E0FD57
:1046E000A3E0FEA3E0FF121A06901659121BC3E4C2
:1046F00090165EF090165D7409F0901B9FE4F0A395
:1047000004F0802B12000EBF020302456680009069
:104710001B9F74FFF0A3749CF08014901BACE0FE10
:10472000A3E0FF901BAFE02FF0901BAEE03EF090B7
:104730001B9FE07002A3E0700F901BA4E004F0E068
:10474000C394035003024487901BA1E0FEA3E0FF43
:10475000D39400EE648094804003024476901B9FC3
:10476000EEF0A3EFF090166374FFF0901BA3E0FF50
:1047700012A40F800F901BA3E0FE3395E0901B9FC7
:0C478000F0A3CEF0901B9FE0FEA3E0FF32
:01478C00220A
:0F3FC800901D00EBF0A3EAF0A3E9F0A3121BC3D6
:103FD70090165DE024FD700302409024FC601424D9
:103FE700FD7003024090147003024090240A60039E
:103FF70002412E12C6AFEF2401FFE43EFEE433FD7B
:10400700E433FC7810121AFAC004C005C006C007D2
:1040170012C6AFEF2401FFE43EFED003D002D00169
:10402700D000EB4FFFEA4EFEE9FDE8FC901D0712BA
:104037001BC3901D07E0FCA3E0FDA3E0FEA3E0FF88
:10404700901668EFF0901D07A3A3A3E07808121A53
:10405700E7901669EFF0901D07E0FCA3E0FDA3E0F1
:10406700FEA3E0FF7810121AE790166AEFF0901D92
:1040770007E0FCA3E0FDA3E0FEA3E0FF7818121A17
:10408700E790166BEFF002413890166BE0FFE4FC07
:10409700FDFE901D07121BC3901D07E0FCA3E0FD6A
:1040A700A3E0FEA3E0FF7808121AFAA804A905AA5C
:1040B70006AB0790166AE0FFEB4FFFEAFEE9FDE863
:1040C700FC901D07121BC3901D07E0FCA3E0FDA396
:1040D700E0FEA3E0FF7808121AFAA804A905AA06C9
:1040E700AB07901669E0FFEB4FFFEAFEE9FDE8FC3E
:1040F700901D07121BC3901D07E0FCA3E0FDA3E082
:10410700FEA3E0FF7808121AFAA804A905AA06ABCD
:1041170007901668E0FFEB4FFFEAFEE9FDE8FC9029
:104127001D07121BC3800A901D07121BCF0000003A
:10413700009016647401F0A3F0A37406F07E007F6C
:10414700047D007B017A1679781221D67E007F04E0
:104157007D007B017A16797C1221D678807C167DCA
:10416700017B017A0079077E007F061216DF901D1A
:1041770000A3E0FAA3E04A601478D07C167D019092
:104187001D00E0FBA3A3E0F912200F8005E49016C1
:10419700D0F0901D0B7401F0A37417F0A37450F0C6
:1041A700901D0BE0FBA3E475F001121865A9F0FA66
:1041B700746312177E901D0BE0FBA3E475F00112E8
:1041C7001865A9F0FA748212177E901D0BE0FBA305
:1041D700E475F001121865A9F0FA745312177E906E
:1041E7001D0BE0FBA3E475F001121865A9F0FA7442
:1041F7006312177E901D0BE0FBA3E475F001121804
:1042070065A9F0FA743512177E901D0BE0FBA3E445
:1042170075F001121865A9F0FA740112177E90164D
:104227005DE024FD605A24FC700302436224FD70A4
:104237000302432F14700302432F240A600302432F
:104247009790166E7480F07E007F047D007B017A64
:104257001679741221D67E007F047D007B017A16C1
:1042670079701221D6901D0BE0FBA3E475F00112C3
:104277001865A9F0FA740112A93B1284D102435DB3
:1042870090166E7480F07E007F047D007B017A16A5
:1042970079701221D612A92912B1AE901D0BEBF03D
:1042A700A3EAF0A3E9F0901D0BE0FBA3E475F0018E
:1042B700121865A9F0FA743212177E901D0BE0FBF5
:1042C700A3E475F001121865A9F0FA740412177EB9
:1042D700E4FF74742FF582E43416F583E0FE901D35
:1042E7000BE0FBA3E475F001121865A9F0FAEE12D2
:1042F700177E0FEFB404DB901D0BE0FBA3E0FAA3DE
:10430700E0F91284DC12AFC712B138901D0BEBF045
:10431700A3EAF0A3E9F07E007F047D007B017A1613
:1043270079741221D6024397E490166EF0FE7F044B
:10433700FD7B017A1679741221D678707C167D017F
:104347007B017A1C792A7E007F041216DF12A929C5
:104357001284D112AFC712B138802AE490166EF0DA
:10436700FE7F04FD7B017A1679741221D6901D0B0E
:10437700E0FBA3E475F001121865A9F0FA740712BF
:10438700A93B12B1AE901D0BEBF0A3EAF0A3E9F045
:10439700901D0BE0FBA3E0FAA3E0F974FF12177E70
:0E43A700901D07E0FCA3E0FDA3E0FEA3E0FFF5
:0143B50022E5
:109F2C007B017A177954901E05EBF0A3EAF0A3E9B4
:109F3C00F02437F9EA3401FAA3EBF0A3EAF0A3E931
:109F4C00F0901E05E0FBA3E0FAA3E0F9121705FE62
:109F5C00B50702807EEEF46029901E08E0FBA3E0BA
:109F6C00FAA3E0F9C003C002C001901E05A3E0FAF9
:109F7C00A3E0F9D3D082D083D0E0E99582EA95832F
:109F8C00400B901E05E4F0A3F0A3F08046EE701C8D
:109F9C00901E06E475F00112184F901E05E0FBA30D
:109FAC00E0FAA3E0F912170560E68095901E06E42E
:109FBC0075F00112184F901E05E0FBA3E0FAA3E028
:109FCC00F912170504FEFD901E06E48DF012184FD1
:0E9FDC00029F4D901E05E0FBA3E0FAA3E0F902
:019FEA002254
:10000E00E4FC7F35129F2CE94A600790000212171C
:04001E001EFCAF0411
:0100220022BB
:107C6A00901DE3121BCF000000007F33129F2C905F
:107C7A001DE7EBF0A3EAF0A3E9F0AE024E700302AF
:107C8A007D9B901DE8E475F00212184F901DE7E005
:107C9A00FBA3E0FAA3E0F9121705FFE4FCFDFE7866
:107CAA0018121AFA901DE3121BC3901DE8E475F02E
:107CBA000112184F901DE3E0F8A3E0F9A3E0FAA33C
:107CCA00E0FBC000C001C002C003A3E0FBA3E0FACE
:107CDA00A3E0F9121705FFE4FCFDFE7810121AFA68
:107CEA00D003D002D001D000EB2FFFEA3EFEE93DDF
:107CFA00FDE83CFC901DE3121BC3901DE8E475F0FF
:107D0A000112184F901DE3E0F8A3E0F9A3E0FAA3EB
:107D1A00E0FBC000C001C002C003A3E0FBA3E0FA7D
:107D2A00A3E0F9121705FFE4FCFDFE7808121AFA1F
:107D3A00D003D002D001D000EB2FFFEA3EFEE93D8E
:107D4A00FDE83CFC901DE3121BC3901DE8E475F0AE
:107D5A000112184F901DE3E0F8A3E0F9A3E0FAA39B
:107D6A00E0FBC001C002C003A3E0FBA3E0FAA3E06A
:107D7A00F9121705FFE4FCFDFED003D002D001EB97
:107D8A002FFFEE3AFEED39FDEC38FC901DE3121B95
:0F7D9A00C3901DE3E0FCA3E0FDA3E0FEA3E0FF28
:017DA90022B7
:10C434007F36129F2CE94A6014740229F9E43AFA0F
:0DC44400785F7C167D017E007F041216DFFC
:01C4510022C8
:10A92900901D0BE0FBA3E475F001121865A9F0FA7C
:10A93900740312177E901D0BE0FBA3E0FAA3E0F964
:0BA94900901E7AEBF0A3EAF0A3E9F007
:10A95400901E7AE0FBA3E475F001121865A9F0FAE1
:10A96400743D12177E901E7AE0FBA3E475F0011289
:10A974001865A9F0FA740712177E901E7AE0FBA3FB
:10A98400E475F001121865A9F0FA740112177EE457
:10A99400FF74072FF582E43400F583E0FE901E7AFD
:10A9A400E0FBA3E475F001121865A9F0FAEE1217A2
:10A9B4007E0FEFB406DB901E7AE0FBA3E0FAA3E07F
:01A9C400F999
:01A9C500226F
:0BB1AE00901D0BEBF0A3EAF0A3E9F00A
:0BB1B900901E7DEBF0A3EAF0A3E9F08C
:10B1C400901E7DE0FBA3E475F001121865A9F0FA66
:10B1D400743612177E901E7DE0FBA3E475F0011215
:10B1E4001865A9F0FA740412177EE4FF745F2FF552
:10B1F40082E43416F583E0FE901E7DE0FBA3E47543
:10B20400F001121865A9F0FAEE12177E0FEFB404DC
:0CB21400DB901E7DE0FBA3E0FAA3E0F954
:01B22000220B
:0BAFC700901D0BEBF0A3EAF0A3E9F0F3
:0BAFD200901E80EBF0A3EAF0A3E9F072
:10AFDD00901E80E0FBA3E475F001121865A9F0FA4C
:10AFED00740C12177E7B017A05792D12C5BA901E4D
:10AFFD0080E0FBA3E475F001121865A9F0FAEF12D9
:10B00D00177EE4FEEEC39F5023742D2EF582E4349B
:10B01D0005F583E0FD901E80E0FBA3E475F00112C1
:10B02D001865A9F0FAED12177E0E80D8901E80E0FB
:07B03D00FBA3E0FAA3E0F918
:01B0440022E9
:1084D100901D0BEBF0A3EAF0A3E9F0901D03E0FC83
:0984E100A3E0FDA3E0FEA3E0FF0F
:1084EA00901DEAEBF0A3EAF0A3E9F0A3121BC3E4A0
:1084FA00FFFEFDFC901DEDE0F8A3E0F9A3E0FAA36E
:10850A00E0FBC3121AD6700A901DED121BCF0000B1
:10851A008CA0901DEAE0FBA3E475F001121865A98E
:10852A00F0FA743312177E901DEAE0FBA3E475F0AB
:10853A0001121865A9F0FA740412177E901DEDE075
:10854A00FCA3E0FDA3E0FEA3E0FF7818121AE7906F
:10855A001DEAE0FBA3E475F001121865A9F0FAEF31
:10856A0012177E901DEDE0FCA3E0FDA3E0FEA3E060
:10857A00FF7810121AE7901DEAE0FBA3E475F001F8
:10858A00121865A9F0FAEF12177E901DEDE0FCA310
:10859A00E0FDA3E0FEA3E0FF7808121AE7901DEAC7
:1085AA00E0FBA3E475F001121865A9F0FAEF1217BF
:1085BA007E901DEDA3A3A3E0FF901DEAE0FBA3E4D8
:1085CA0075F001121865A9F0FAEF12177E901DEAEC
:0985DA00E0FBA3E0FAA3E0F922A2
:0BB13800901D0BEBF0A3EAF0A3E9F080
:10B14300901E83EBF0A3EAF0A3E9F0901E83E0FBEB
:10B15300A3E475F001121865A9F0FA743712177E8B
:10B16300901E83E0FBA3E475F001121865A9F0FAC1
:10B17300740212177E901E83E0FBA3E475F00112A4
:10B183001865A9F0FA740112177E901E83E0FBA3E1
:10B19300E475F001121865A9F0FA740312177E9092
:0BB1A3001E83E0FBA3E0FAA3E0F9220A
:10C452007F01129F2CE94A6014740229F9E43AFA26
:0DC4620078347C1C7D017E007F041216DF03
:01C46F0022AA
:10C48D007F03129F2CE94A6013740229F9E43AFAEA
:0CC49D0078387C1C7D017E000F1216DF39
:01C4A9002270
:05BF7F00421AC500009C
:10B53300E4901AC7F0A3F0F9A3C9F0A3F0A3E9F0CC
:10B543007E007F047D007B017A1B79251221D67E44
:10B55300007F047D007B017A1A79D41221D67E0004
:10B563007F047D007B017A1A79D01221D67E007F79
:10B57300497D007B017A1A79D81221D6901ACF74AB
:10B58300FFF0901ACEF0901ACDF0901ACCF0901BE9
:0DB593002174E0F0E4A3F0A3F0A304F02283
:10C0F2001286F1901EB0EFF030E210127834C3EFE6
:10C10200648094804012128D03800D901EB0E03046
:0DC11200E6061276951292A2901EB0E0FF94
:01C11F0022FD
:1086F100E4901AC7F0A3F0126D68D3EF9400EE6412
:1087010080948050037F002212BA53EF901E0CF028
:10871100A3E4F012BA53901E0DE02FF0901E0CE06E
:108721003EF0E0FEA3E0FFD394EEEE94055004EF9B
:108731004E700612C5A47F0022900A73E0FBA3E0ED
:10874100FAA3E0F9901E0CE0FEA3E0FFE92FF9EA9D
:108751003EFAA3EBF0A3EAF0A3E9F0901E0EA3E02A
:10876100FAA3E0D39012779582EA9583500E901E7A
:108771000EE0F9A3A3E0901AC9C9802C900A73A353
:10878100E0FAA3E0FFC374779FFF74129AFEC390CF
:108791001E0DE09FFF901E0CE09EFE74772FF97472
:1087A1000E3EFA901AC97401F0A3EAF0A3E9F0129F
:1087B100AD32EF1460090470037F20227F00221282
:1087C1006471901E0BEFF06004E030E3051292A299
:1087D1008025901E0BE0FF20E00620E10330E21728
:1087E100901DAB7401F0A3741CF0A3742EF07B01F7
:0C87F1007A1B7925129CE4901E0BE0FF1F
:0187FD002259
:10691600901CA2EDF0901C9FEBF0A3EAF0A3E9F027
:106926004A70037F8522901663E0FEF46017901C80
:106936009FE0FBA3E0FAA3E0F912187B644445F05C
:1069460060037FA422EE6401601D782A7C1C7D0111
:106956007B017A1A79D07E007F041221B2EF33953B
:10696600E04F70037F8522901CA4E02414F0901C55
:10697600A3E03400F0901AC6E004F07006901AC541
:10698600E004F0901AC5E0FFA3E0901CABCFF0A3A3
:10699600EFF0901C9FE0FBA3E0FAA3E0F990001D46
:1069A60012171E901CA230E406E0FF74048004E077
:1069B600FF7440901CADF0A3EFF0901CA3E0FCA385
:1069C600E0FDE4901BD3F0A3F0901CADE0FFA3E044
:1069D600901BD5CFF0A3EFF0A37401F0A3741CF0C5
:1069E600A3742AF0901C9FE0FBA3E0FAA3E0240422
:1069F600F9E43AFA901BDAEBF0A3EAF0A3E9F0E443
:106A0600A3F0901CABE0FAA3E0FB7F007E45125D8D
:106A16001B901CA5121BC3901CA5E0FCA3E0FDA3C4
:106A2600E0FEA3E0FF7808121AE7A3EFF0901CA59A
:106A3600A3A3E0FEA3E0FF901CAAEFF0901CA2E047
:106A4600B40107E4901CAFF08012901663E0B40125
:106A5600047F0180027F00901CAFEFF0901C9FE046
:106A6600FBA3E0FAA3E0F9901CAFE0901D99F07D3E
:106A7600007C081279C1EF64016001227F4512C5CE
:106A86005EE4FF12C55E901CA3E0FF12C55E901C7B
:106A9600A3A3E0FF12C55E901CABE0FF12C55E909B
:106AA6001CABA3E0FF12C55EE4FF12C55EE4FF1255
:106AB600C55E901C9FE0FBA3E0FAA3E0F990001DE1
:106AC60012171E30E4047F0480027F4012C55E90D8
:106AD6001CA2E0FF12C55E901CA9E0FF12C55E90E5
:106AE6001CAAE0FF12C55E901C2AE0FF12C55E904C
:106AF6001C2BE0FF12C55E901C2CE0FF12C55E90B9
:106B06001C2DE0FF12C55E901C9FE0FBA3E0FAA3DC
:106B1600E0F990000412171EFF12C55E901C9FE05C
:106B2600FBA3E0FAA3E0F990000512171EFF12C5B9
:106B36005E901C9FE0FBA3E0FAA3E0F9900006122A
:106B4600171EFF12C55E901C9FE0FBA3E0FAA3E0B0
:0D6B5600F990000712171EFF12C55E7F01A7
:016B6300220F
:1092A200901AC9E0FBA3E0FAA3E0F9C003C002C030
:1092B20001900A73E0FBA3E0FAA3E0F9D082D08325
:1092C200D0E06B7008E965827003EA65837003027F
:1092D2009389901AC9E0FBA3E0FAA3E0F9C003C0A6
:1092E20002C001900A73A3E0FAA3E0F9C3D082D0CE
:1092F20083D0E0E99582EA9583501F900A73A3A375
:10930200E0AE02FF901AC9A3E0FAA3E0C39FFFEA0E
:109312009E901EAEF0A3EFF08027901AC9A3E0FA48
:10932200A3E0AE02FF900A73A3E0FAA3E0C39FFF9B
:10933200EA9EFEC3E49F901EAFF074049E901EAEA0
:10934200F0901278E0FEA3E0FFD3901EAFE09F9072
:109352001EAEE09E400302C5A4C2AF901EAEE0FE68
:10936200A3E0FFC3901279E09FF0901278E09EF0A4
:10937200901AC9E0F9A3E0FAA3E0900A73C9F0A336
:07938200EAF0A3E9F0D2AF0D
:0193890022C1
:10647100E4901CB8F012BA53901CB5EFF0E0FE5452
:106481000FA3F0EEC4540F640460030266C4E0FF7E
:10649100C3940550030266C4EF25E025E0F0C394E0
:1064A10014A3F012BA53901CB0EFF012BA53EF904C
:1064B1001AC7F0A3E4F012BA53901AC8E02FF09073
:1064C1001AC7E03EF0C3A3E09414901AC7E0940009
:1064D10050037F002212BA53EF901CB9F0A3E4F0ED
:1064E10012BA53901CBAE02FF0901CB9E03EF012A2
:1064F100BA53EF901CBBF0A3E4F012BA53901CBC4A
:10650100E02FF0901CBBE03EF0A3E030E507901CCB
:10651100B8E04410F012BA53901CB1EFF012BA5324
:10652100901CB2EFF014601D14602324F1600D245F
:106531000B7024901CB8E04401F08022901CB8E05C
:106541004402F08019901CB8E04404F08010901CC3
:10655100B8E04440F08007901CB8E04408F012BA5B
:1065610053901CB3EFF012BA53901CB4EFF012BA6F
:1065710053901B25EFF012BA53901B26EFF012BA7D
:1065810053901B27EFF012BA53901B28EFF0901B8A
:1065910025E0FFC394E04009EFD394EF50037F005F
:1065A1002212BA53901AD4EFF012BA53901AD5EFBF
:1065B100F012BA53901AD6EFF012BA53901AD7EFDD
:1065C100F012B903EF7047901C2AE0FF901AD4E053
:1065D100FE6F6004EEF47033901C2BE0FF901AD52F
:1065E100E0FE6F6004EEB4FF22901C2CE0FF901AD5
:1065F100D6E0FE6F6004EEB4FF11901C2DE0FF9019
:106601001AD7E0FE6F6007EEF460037F0022901C52
:10661100B5E0FE901CB0E0FDEDFFC006C007901A8A
:10662100C7E0FCA3E0FD901CBBE0FFA3E0901BD3FF
:10663100CFF0A3EFF0901CB1E0FEA3E0FBEBFF90E5
:106641001BD5EEF0A3EFF0A37401F0A3741AF0A32D
:1066510074D4F0A37401F0A3741BF0A37425F0901B
:106661001CB7E0901BDDF0901CB9E0FAA3E0FBD071
:1066710007D006125D1B901CBD121BC3901CBDE010
:10668100FCA3E0FDA3E0FEA3E0FF7808121AE79067
:106691001CB3E0B50711901CBDA3A3A3E0FF901CA0
:1066A100B4E0FEEF6E60037F0022901CB6E0FFC3F2
:1066B100901AC8E09FF0901AC7E09400F0901CB8BF
:0566C100E0FF227F0054
:0166C60022B1
:10B90300E4901EB1F078D47C1A7D017B017A1B7917
:10B9130021FE7F041221B2EF7005901EB104F09056
:10B923001EB1E0702A7B017A1A79D412AC22E94A5B
:10B93300601D90000612171E601590000712171E57
:10B94300FF64016004EFB40206901EB17401F0902D
:04B953001EB1E0FF42
:01B9570022CD
:0E5D1B00901BCFECF0A3EDF0A3EAF0A3EBF0A9
:105D2900E4FCFD901BDE121BC3901BDEE0F8A3E030
:105D3900F9A3E0FAA3E0FBC000C001C002C00390D0
:105D49001BD7E0FBA3E0FAA3E0F990000112171EAC
:105D5900FD121705FEEDFFE4FCFDD003D002D001D2
:105D6900D000EB2FFFEA3EFEED39FDEC38FC901B2D
:105D7900DE121BC3901BDEE0F8A3E0F9A3E0FAA34F
:105D8900E0FBC000C001C002C003901BD7E0FBA329
:105D9900E0FAA3E0F990000212171EFE9000031228
:105DA900171EFDEDFFE4FCFDD003D002D001D000A9
:105DB900EB2FFFEA3EFEED39FDEC38FC901BDE12BD
:105DC9001BC3901BDEE0F8A3E0F9A3E0FAA3E0FB14
:105DD900901BCFE0FEA3E0FFE4FCFDEB2FFFEA3EC2
:105DE900FEED39FDEC38FC901BDE121BC3901BDE67
:105DF900E0F8A3E0F9A3E0FAA3E0FB901BD1E0FEF1
:105E0900A3E0FFE4FCFDEB2FFFEA3EFEED39FDECDC
:105E190038FC901BDE121BC3901BDEE0F8A3E0F9EF
:105E2900A3E0FAA3E0FB901BD3E0FEA3E0FFE4FCB0
:105E3900FDEB2FFFEA3EFEED39FDEC38FC901BDE51
:105E4900121BC3901BDEE0F8A3E0F9A3E0FAA3E07C
:105E5900FB901BD5E0FEA3E0FFE4FCFDEB2FFFEA7E
:105E69003EFEED39FDEC38FC901BDE121BC3901B86
:105E7900DEE0F8A3E0F9A3E0FAA3E0FBC000C0016B
:105E8900C002C003901BDAE0FBA3E0FAA3E0F9909B
:105E9900000112171EFD121705FEEDFFE4FCFDD0EF
:105EA90003D002D001D000EB2FFFEA3EFEED39FD11
:105EB900EC38FC901BDE121BC3901BDEE0F8A3E05C
:105EC900F9A3E0FAA3E0FBC000C001C002C003903F
:105ED9001BDAE0FBA3E0FAA3E0F990000212171E17
:105EE900FE90000312171EFDEDFFE4FCFDD003D068
:105EF90002D001D000EB2FFFEA3EFEED39FDEC3870
:105F0900FC901BDE121BC3901BDDE0606120E05E8C
:105F1900E4901BE4F0901BDDE0FF901BE4E0C39FDD
:105F2900504C12BA53EF901BE2F0A3E4F012BA53AB
:105F3900901BE3E02FF0901BE2E03EF0901BDEE0C7
:105F4900F8A3E0F9A3E0FAA3E0FBA3E0FEA3E0FFD6
:105F5900E4FCFDEB2FFFEA3EFEED39FDEC38FC9049
:105F69001BDE121BC3901BE4E02402F080A7901BE8
:105F7900DEE0FCA3E0FDA3E0FEA3E0FF12B377900F
:105F89001BDE121BC3901BDEE0FCA3E0FDA3E0FEB9
:035F9900A3E0FF83
:015F9C0022E2
:10783400901D8B74FFF012BA53901D8AEFF0640808
:1078440060030279B8901AC7E0FEA3E0FFD394481E
:10785400EE940040030279B8C3EF9404EE94005010
:10786400030279B8E4901C92F0A3F0A304F0E4A31B
:10787400F0F9A3C9F0A3F0A3E9F0E4A3F0A3F07B2B
:10788400017A1B7925FDFC124EB3901D8BEFF0C3DA
:107894006480948050030279B812BA53901D8AEF21
:1078A400F0901AC8E024FEFE901AC7E034FF901D41
:1078B4008DF0A3CEF0901D8BE0901AD8F0901D8D22
:1078C400E0FCA3E0FDEC901AD9F0EDA3F0901D8E3E
:1078D40024FEF0901D8DE034FFF012BA53901D8CFD
:1078E400EFF012BA53901D8CE02408F0C3940850B2
:1078F400010F901D8CE0901ADBF0A3EFF0901D8F28
:107904007401F0A3741AF0A374DDF0900A73A3E079
:10791400FAA3E0FFC374779FFF74129ACF2401CFB8
:107924003400901D92F0FCA3EFF0FD901D8DE0FE5D
:10793400A3E0FFD39DEE9C501AA3E0FBA3E0FAA3BF
:10794400E0F8AC02AD03900A73E0FBA3E0FAA3E015
:10795400F9805E901D92E0FEA3E0FF901D8FE0FB96
:10796400A3E0FAA3E0F8AC02AD03900A73E0FBA332
:10797400E0FAA3E0F91216DF901D92E0FEA3E0FF07
:10798400C3901D8EE09FF0901D8DE09EF0E0FCA35F
:10799400E0FDC004C005A3E0FBA3E0FAA3E02FF9D7
:1079A400EA3EA801FCAD037B017A0E7978D007D0BA
:0C79B400061216DF1292A2901D8BE0FF5D
:0179C00022A4
:108D0300901AD8E0901E13F0C3648094805003023D
:108D13008DFAE0FFFD3395E0FC90129975F03DED7F
:108D2300121C24EC75F03DA42583F583E020E003B9
:108D3300028DFAEF3395E0FE7C007D3D1217B2748D
:108D43007B2FF974123EFA7B01901E14EBF0A3EA19
:108D5300F0A3E9F090001B12171E64016003028D5B
:108D6300FA901AD9E0901E11F0A3E4F0901ADAE019
:108D7300FF901E12E02FF0901E11E03400F0E0FE91
:108D8300A3E0FFD39446EE940050647A1A79DBC0D3
:108D930003C002C001901E14E0FBA3E0FAA3E0F9B4
:108DA30090000E121CF8901E14E0FBA3E0FAA3E05F
:108DB300F9900011EE8FF0121982EF2402FFE43EC6
:108DC300901CA3F0A3EFF07D01126916EF6020E47D
:108DD300FF12C55EE4FF12C55E901E14E0FBA3E024
:108DE300FAA3E0F9901E11E0FCA3E0FD12BE399056
:078DF3001E13E0FF12A40FA4
:018DFA002256
:10C5A400C2AF12C2A3901AC97401F0A3740EF0A30F
:06C5B4007478F0D2AF2202
:10C3F500901B31EFF07B017A0A7978900A6AEBF0AD
:10C40500A3EAF0A3E9F0A3EBF0A3EAF0A3E9F02295
:10C2A3007B017A0E7978900A73EBF0A3EAF0A3E9A5
:10C2B300F0900A70EBF0A3EAF0A3E9F0E4901278AF
:04C2C300F0A3F022D2
:0EC6A10012C2A3E4FF12C3F5E490127AF02255
:10BDFC0090127AE0601F7B017A1E792F7D587C02AD
:10BE0C0012AB887B017A1E792F12B794EF700690D3
:10BE1C00127AE070EE90127AE070057F0112C3F591
:0CBE2C0090127AE070047F0180027F0019
:01BE380022E7
:10C54500C2AF438901758C60758A7FD28CD2A9E40C
:09C55500900A76F0A3F0D2AF22A7
:10C3B400C28C758C60758A7FD28C900A77E004F009
:10C3C4007006900A76E004F012C17C12946E02BDED
:01C3D4007BED
:10C32F007E037FD07D007B017A12797B1221D6129A
:10C33F00B53312C54512C68412C27F12C67512C616
:01C34F00C726
:01C3500022CA
:10A74800C003C002C001901CE7E0FFA3E0901C9288
:10A75800CFF0A3EFF0901CEAE0901C94F0901CEB73
:10A76800E0901C95F0901CECE0F9A3E0FAA3E090CF
:10A778001C96C9F0A3EAF0A3E9F0901CEFE0FFA350
:10A78800E0901C99CFF0A3EFF0D001D002D00312D3
:10A798004EB3901CF1EFF0901CEAE06406703D9017
:10A7A8001CF1E0FFC3648094804031EF3395E0FEF4
:10A7B8007C007D3D1217B2747B2FF974123EFA7B30
:10A7C80001901CE9E0FF128A13D3EF648094805053
:10A7D8000B901CF1E0FF12A40F7F8422901CF1E083
:01A7E800FF71
:01A7E900224D
:104EB300901C8DEBF0A3EAF0A3E9F0A3ECF0A3EDD3
:014EC300F0FE
:104EC400901C9B7482F0901C94E0FE146018146093
:104ED4001524FC601124F5600D240D700E901C95B2
:104EE400E0B420078000E4901C9BF0901C9BE0FF42
:104EF400B4820122901C8DE0FBA3E0FAA3E0F91236
:104F04001705FFC394E0400DEFD394EF5007901CB6
:104F140095E04410F0901C90E07002A3E0700EEE57
:104F240064066036901C94E0B41102802D901C94A9
:104F3400E0B40607A3E030E402801F12170564E022
:104F4400702190000112171E701990000212171E92
:104F5400701190000312171E7009901C9B7485F049
:104F64000251E0901C92E0FCA3E0FD901C8DE0FB5C
:104F7400A3E0FAA3E0F9901C94E0901D3EF0901C8D
:104F840090E0FEA3E0FF128023901C9CEBF0A3EAC8
:104F9400F0A3E9F04A602C901C9CE0FBA3E0FAA388
:104FA400E0F990001C12171E75F03DA42499F582B7
:104FB400E5F03412F583E030E009901C9B7481F035
:104FC4000251E012C200901C9BEFF0648070030257
:104FD40051E07E007F3DC006C0077F00C007E0FFB0
:104FE4003395E0FE7C007D3D1217B2747B2FF9747B
:104FF400123EFA7B01D005D007D0061221D6901CB0
:105004009BE0FF3395E0FE7C007D3D1217B2747B7C
:105014002FF974123EFA7B01A3EBF0A3EAF0A3E9A3
:10502400F0901C9BE090001C121790901C90E0FFE5
:10503400A3E0CF8FF0121963901C92E0FEA3E0FF6F
:10504400901C9CE0FBA3E0FAA3E0F9900002EE8F31
:10505400F0121982901C8DE0FBA3E0FAA3E0F91290
:105064001705FF901C9CE0FBA3E0FAA3E0F9900075
:1050740004EF121790901C8DE0FBA3E0FAA3E0F973
:1050840090000112171EFF901C9CE0FBA3E0FAA302
:10509400E0F9900005EF121790901C8DE0FBA3E05F
:1050A400FAA3E0F990000212171EFF901C9CE0FB8B
:1050B400A3E0FAA3E0F9900006EF121790901C8D7C
:1050C400E0FBA3E0FAA3E0F990000312171EFF909F
:1050D4001C9CE0FBA3E0FAA3E0F9900007EF121791
:1050E40090901C95E0FF64207044901C94E064044C
:1050F400703C901C2EE0900008121790901C2FE03A
:10510400900009121790901C30E090000A1217903A
:10511400901C31E090000B121790901C32E090002C
:105124000C121790901C33E090000D121790901CF5
:1051340094E0FE901C9CE0FBA3E0FAA3E0F990004D
:105144001BEE12179090001DEF121790901C96E022
:10515400FBA3E0FAA3E0F9EA494B604EA3E0FCA309
:10516400E0FD4C6045C003C002C001901C9CE0FB04
:10517400A3E0FAA3E0F9900013121CF8901C96E047
:10518400FBA3E0FAA3E02DF9EA3CFAE924FFF9EAEB
:1051940034FFFAC003C002C001901C9CE0FBA3E0F2
:1051A400FAA3E0F9900016121CF8EEB4060E901C57
:1051B4009CE0FBA3E0FAA3E0F91290CF901C9BE0E3
:1051C400FF3395E0FE90129975F03DEF121C24EE2A
:1051D40075F03DA42583F583E04401F0901C9BE029
:0151E400FFCB
:0151E50022A7
:1074E800901D2BEBF0A3EAF0A3E9F0901D2AEFF032
:1074F800901D3374FFF0A37489F0E4A3F0A3F0C3E4
:10750800EF64809480400B901D2AE0FD6480949085
:1075180040057EFF7F8522EDFF3395E0FE901299AE
:1075280075F03DEF121C24EE75F03DA42583F5831C
:10753800E020E0057EFF7F862290165DE0FF700563
:107548007EFF7F9D22901663E0B4FF1AEF640A6005
:1075580004EFB40B1190164DE0FCA3E0FDA3E0FE90
:10756800A3E0FF128FE212B045901D2AE0FF339589
:10757800E0FE7C007D3D1217B2747B2FF974123E39
:10758800FA901D307401F0A3EAF0A3E9F0901D2BE6
:10759800E0FBA3E0FAA3E0F9EA494B6034A3E0FE7C
:1075A800A3E0FF4E602BC003C002C001901D30E075
:1075B800FBA3E0FAA3E0F990000E121CF8901D302E
:1075C800E0FBA3E0FAA3E0F9900011EE8FF01219A6
:1075D80082901D30E0FBA3E0FAA3E0F990001B12B3
:1075E800171E6406600302767A901D30E0FBA3E064
:1075F800FAA3E0F9126F59901D35EEF0A3EFF0D31E
:107608009400EE648094804060901D33E0B4FF23C2
:10761800A3E0B4891E901D2AE0FF7B007A00790060
:10762800E4901C18F0A312713F901D33EEF0A3EF05
:10763800F080D6901D33E0FEA3E0FFC3EE64809493
:10764800805011EF64877002EEF46008A3EEF0A397
:10765800EFF08015901D30E0FBA3E0FAA3E0F9906D
:1076680000241218A645F07080901D35E0FEA3E0B6
:10767800FF22901D30E0FBA3E0FAA3E0F990001B85
:0C76880012171EB41103027324E4FEFF6D
:0176940022D3
:10C64300901E1BE0FDA3E0901C18CDF0A3ED12712A
:02C653003F2284
:09713F00F0A37402F0A37458F0EF
:0D714800901C15EBF0A3EAF0A3E9F0AD07F1
:10715500E4901C1CF0A3F0C3ED648094804007ED1F
:10716500648094904003027236EDFB3395E0FA900B
:10717500129975F03DEB121C24EA75F03DA42583A8
:10718500F583E020E0057EFF7F862290165DE070A6
:10719500057EFF7F9D227C007D3DAF03AE02121769
:1071A500B2747B2FF974123EFA901C1E7401F0A381
:1071B500EAF0A3E9F0901C15E0FBA3E0FAA3E0F9DF
:1071C500EA494B604EA3E0FEA3E0FF4E6045C003D5
:1071D500C002C001901C1EE0FBA3E0FAA3E0F990F9
:1071E5000013121CF8901C15E0FBA3E0FAA3E02F96
:1071F500F9EA3EFAE924FFF9EA34FFFAC003C002CE
:10720500C001901C1EE0FBA3E0FAA3E0F990001674
:10721500121CF8901C1EE0FBA3E0FAA3E0F9900015
:107225001B12171EB4110F900013121CC8E94A70E7
:10723500057EFF7F8522901C1EE0F9A3E0FAA3E0FE
:10724500A3C9F0A3EAF0A3E9F0901C1AE0FCA3E0BF
:10725500FD4C60097B017A1C792412AB8812C0F2BF
:10726500901C29EFF054077029901C1AE07002A3B6
:10727500E0600C7B017A1C792412B794EF60057EDF
:10728500FF7F872212B04512C6EBBF9AD07EFF7FE3
:107295009A22901C29E0FF20E2C3EF30E0197B0120
:1072A5007A1C791E1222CE901C1CEEF0A3EFF0BEC4
:1072B500FF1DBFFA1A805F901C29E030E1117B01A8
:1072C5007A1C791E12478D901C1CEEF0A3EFF090EE
:1072D5001C21E0FBA3E0FAA3E0F9C003C002C00152
:1072E500901C1EE0FBA3E0FAA3E0F9D082D083D086
:1072F500E06B7008E965827003EA65836018901C8D
:1073050021E0F9A3E0FAA3E0901C1EC9F0A3EAF07E
:0E731500A3E9F0027262901C1CE0FEA3E0FFF0
:017323002247
:05A0A800901E59EFF0CD
:10A0AD00C3648094804008E0FD6480949040057EF8
:10A0BD00FF7F8522EDFF3395E0FE90129975F03DFF
:10A0CD00EF121C24EE75F03DA42583F583E020E00E
:10A0DD00057EFF7F862290165DE0700D901E59E083
:10A0ED00FF12A40F7EFF7F9D22901E59E0FF339536
:10A0FD00E0FE7C007D3D1217B2747B2FF974123E89
:10A10D00FA7B01A3EBF0A3EAF0A3E9F090001B1298
:10A11D00171EB4060E901E5AE0FBA3E0FAA3E0F959
:10A12D0012BDBD901E59E0FF3395E0FE901299755A
:10A13D00F03DEF121C24EE75F03DA42583F583E46C
:10A14D00F0901E5AE0FBA3E0FAA3E0F9E4F5F0125B
:05A15D001963E4FEFFA0
:01A1620022DA
:05A40F00901E5DEFF05E
:10A41400C3648094804008E0FD6480949040057E8D
:10A42400FF7F8522EDFF3395E0FE90129975F03D94
:10A43400EF121C24EE75F03DA42583F583E020E0A3
:10A44400057EFF7F8622901E5DE0FF3395E0FE7C53
:10A45400007D3D1217B2747B2FF974123EFA7B0112
:10A46400A3EBF0A3EAF0A3E9F090001B12171EB4CB
:10A47400060E901E5EE0FBA3E0FAA3E0F912B6D349
:10A48400901E5DE0FF3395E0FE90129975F03DEF6C
:10A49400121C24EE75F03DA42583F583E4F0901E90
:10A4A4005EE0FBA3E0FAA3E0F9E4F5F0121963E43B
:02A4B400FEFFA9
:01A4B6002283
:10BE390090165DE06033E94A601390001B12171EEB
:10BE4900B4060A90002074FF12174B800090127AF2
:10BE59007401F01257CBE490127AF0D3EF9400EE0C
:0BBE69006480948040057F01227F9DD3
:01BE740022AB
:10C1A900EE7024EF24EC601314601024FC6010245A
:10C1B900D4601024F570107D81800E7D02800A7D87
:0BC1C9000480067D088002E4FDAF0545
:01C1D4002248
:10802300901D37EEF0A3EFF0A3ECF0A3EDF0A3EB7C
:07803300F0A3EAF0A3E9F05D
:10803A00901663E0901D43F0901D40E4F0A3F0A376
:10804A00F0901D3BA3E0FAA3E04A7003028150E4DA
:10805A00901D3FF0901D3FE0FFC394104003028142
:10806A005075F03DEFA4247BF582E5F03412F583D8
:10807A00E0FEA3E0FF901D37E0FCA3E0FDEF6D708A
:10808A0002EE6C6003028147901D3FE0FF75F03DF0
:10809A00A4247DF582E5F03412F583E0FCA3E0FD2B
:1080AA00901D39E0FAA3E0FBED6B7002EC6A600305
:1080BA0002814775F03DEFA42496F582E5F034126B
:1080CA00F583E0FF901D3EE0FEEF6E7070901D4359
:1080DA00E0B40124901D3FE075F03DA4247FF974BB
:1080EA001235F0A801FC7D017B017A1A79CC7E0059
:1080FA007F041221B2EF6029901D3FE075F03DA484
:10810A00247FF9741235F0A801FC7D01901D3BE033
:10811A00FBA3E0FAA3E0F97E007F041221B2EF701C
:10812A001C901D3FE075F03DA4247BF9741235F0D4
:10813A00FAA37401F0A3EAF0A3E9F08009901D3FC5
:10814A00E004F002805E901D40E0FBA3E0FAA3E0A9
:01815A00F92B
:01815B002201
:10C200007F80E4FEEEFD3395E0FC90129975F03DE1
:10C21000ED121C24EC75F03DA42583F583E020E0AD
:0AC2200004AF0680050EEEB410DA3C
:01C22A0022F1
:04C6E10012C5E32279
:0B478D00901BE5EBF0A3EAF0A3E9F0BD
:1047980012BA53EF901BEEF0A3E4F012BA53901B39
:1047A800EFE02FF0901BEEE03EF012BA53EF901BB3
:1047B800ECF0A3E4F012BA53901BEDE02FF0901B3D
:1047C800ECE03EF0E0FEA3E0FFA3E0FCA3E0FD7B0D
:1047D800017A1B7925901D3E7411F0128023901BDD
:1047E800F8EBF0A3EAF0A3E9F04A600302488590E9
:1047F8001BECE0FEA3E0FF7B017A1B7925901D3EB0
:104808007411F0E4FDFC128023901BF8EBF0A3EA8E
:10481800F0A3E9F04A7025901BECE0FEA3E0FF7BD3
:10482800017A1A79D0901D3E7411F0E4FDFC1280D3
:1048380023901BF8EBF0A3EAF0A3E9F0901BF8E053
:10484800FBA3E0FAA3E0F94A6012901BEEE0FFA395
:10485800E0900002CF8FF012198280217B007A004D
:104868007900C003C002C001901BE5E0FBA3E0FA99
:10487800A3E0F9121C791292A2E4FEFF22901BF821
:10488800E0FBA3E0FAA3E0F9C003C002C001901B5B
:10489800E5E0FBA3E0FAA3E0F9121C79901BF8E02D
:1048A800FBA3E0FAA3E0F990000412171E705490DD
:1048B800001D12171E30E423901AD4E09000041251
:1048C8001790901AD5E0900005121790901AD6E02C
:1048D800900006121790901AD78021901B25E0901F
:1048E8000004121790901B26E09000051217909074
:1048F8001B27E0900006121790901B28E0900007F5
:1049080012179012BA53EF901BF2F0A3E4F012BA08
:1049180053901BF3E02FF0901BF2E03EF0C3A3E0AE
:104928009408901BF2E0940050227B007A007900F2
:10493800C003C002C001901BE5E0FBA3E0FAA3E0BE
:10494800F9121C791292A27EFF7FFF2212BA53EF4E
:10495800901BEAF0A3E4F012BA53901BEBE02FF09F
:10496800901BEAE03EF0901BF4121BCF0000000001
:10497800E4901BFBF0A3F0901BEAE07002A3E06058
:1049880042901BF2E0FCA3E0FD901BEEE0FFA3E0E9
:10499800901CC6CFF0A3EFF0A37401F0A3741AF033
:1049A800A374D4F0A37401F0A3741BF0A37425F0CE
:1049B800901BECE0FAA3E0FB7F11126B64901BF4F0
:1049C800121BC3901BF3E024F8F0901BF2E034FFB5
:1049D800F0E0FEA3E0FF901BF0EEF0A3EFF04E70C6
:1049E80003024AD1E4901BE9F0901BF0E0FEA3E03B
:1049F800FF901BF8E0FBA3E0FAA3E0F912C6D2127D
:104A0800BA53901BE8EFF0901BEAE07002A3E06055
:104A180057901BE9E0901BE8700FE0901BFBF0A398
:104A2800E4F0901BE904F0803FE0FF901BFCE02FCE
:104A3800F0901BFBE03400F0901BF4E0F8A3E0F9E1
:104A4800A3E0FAA3E0FB901BFBE0FEA3E0FFE4FC7D
:104A5800FDEB2FFFEA3EFEED39FDEC38FC901BF430
:104A6800121BC3E4901BE9F0901BE8E0FF901BF8D1
:104A7800E0FBA3E0FAA3E0F912A55D901BF074FF38
:104A8800F5F012184F45F06003024A07901BEAE060
:104A98007002A3E06047901BE9E06041901BF4E0DE
:104AA800F8A3E0F9A3E0FAA3E0FB901BFBE0FEA368
:104AB800E0FFE4FCFDEB2FFFEA3EFEED39FDEC38AC
:104AC800FC901BF4121BC38014901BF8E0FBA3E0BE
:104AD800FAA3E0F9900019E4F5F0121982901BEAA4
:104AE800E07002A3E0603E901BF4E0FCA3E0FDA3AD
:104AF800E0FEA3E0FF12B377901BF4121BC3901BD8
:104B0800EAE0FEA3E0FFE4FCFD901BF4E0F8A3E07C
:104B1800F9A3E0FAA3E0FBC3121AD660081292A226
:104B28007EFF7FFC22901BF8E0FBA3E0FAA3E0F9EC
:104B380012C6E51292A2901BF8E0FBA3E0FAA3E0EC
:0A4B4800F99000191218A6FFAEF054
:014B52002240
:0B732400901D50EBF0A3EAF0A3E9F08D
:10732F004A70057EFF7F8522901D50E0FBA3E0FA97
:10733F00A3E0F912C120901D53EEF0A3EFF04E70B1
:10734F0003FEFF22901D50E0FBA3E0FAA3E0F990AB
:10735F00000E121CC8901D57EBF0A3EAF0A3E9F042
:10736F00901D54E02408FF901D53E03400FE901D43
:10737F0055F0FCA3EFF0FD901D50E0FBA3E0FAA346
:10738F00E0F912187BFBAAF0C002C003901D50E079
:10739F00FBA3E0FA9000021218A6FF901CC6E5F0BE
:1073AF00F0A3EFF0A37401F0A3741CF0A3742AF000
:1073BF00901D50A3A3E02404F9E43AFA901CCBEB00
:1073CF00F0A3EAF0A3E9F0D003D0027F11126B64AF
:1073DF00C007901D57E0FBA3E0FAA3E0F9901D53FF
:1073EF00E0FFA3E0901D6FCFF0A3EFF0D007128561
:1073FF00E312B377901D5AEEF0A3EFF0901D50E01B
:10740F00FBA3E0FAA3E0F990001B12171EFD901DDD
:10741F0055E0FFA3E0901CA3CFF0A3EFF0901D5019
:10742F00A3A3E0126916EF640160030274CD901DEF
:10743F0050E0FBA3E0FAA3E0F912187BE5F0FF128E
:10744F00C55E901D50E0FBA3E0FAA3E0F912187B94
:10745F00FF12C55E901D50E0FBA3E0FAA3E0F99088
:10746F0000021218A6E5F0FF12C55E901D50E0FB5A
:10747F00A3E0FAA3E0F99000021218A6FF12C55E6E
:10748F00901D55E0FF12C55E901D55A3E0FF12C57C
:10749F005E901D5AE0FF12C55E901D5AA3E0FF12C9
:1074AF00C55E901D50E0FBA3E0FAA3E0F9A3E0FC5A
:1074BF00A3E0FD12BE39D3EF648094805006EF3302
:1074CF0095E0FE22901D50E0FBA3E0FAA3E0F990B7
:0874DF0000111218A6FFAEF027
:0174E7002282
:104B5300901C6374FFF012BA53EF4E6003024EAD24
:104B630012BA53EF64014E6003024EAD12BA53EF13
:104B730064084E6003024EAD12BA53EF4E60030257
:104B83004EAD12BA53EF64064E6003024EAD12BA35
:104B930053EF64044E6003024EAD12BA53EF4E60FE
:104BA30003024EAD12BA53EF24FE7003024DE40428
:104BB3006003024EADE4901C54F012BA53901C549F
:104BC300E0245DF582E4341CF583EFF0901C54E09F
:104BD30004F0E0C3940640E2E4901C54F012BA538C
:104BE300901C54E02459F582E4341CF583EFF090D3
:104BF3001C54E004F0E0C3940440E2E4901C54F03D
:104C030012BA53901C54E004F0E0C3940640F1E45C
:104C1300901C54F012BA53901C54E02455F582E4CE
:104C2300341CF583EFF0901C54E004F0E0C39404CB
:104C330040E2901C2AE0FF901C55E06F6003024E97
:104C4300AD901C2BE0FF901C56E06F6003024EAD4D
:104C5300901C2CE0FF901C57E06F6003024EAD9058
:104C63001C2DE0FF901C58E06F6003024EAD7B01EA
:104C7300901DAB04F0A3741CF0A3745DF07A1C794F
:104C830059129CE474FF901C92F0A3F0A37404F0F7
:104C9300A37420F0A3E4F0A3F0A3F0A3F0A3F07BAC
:104CA300017A1C795974FFFDFC124EB3901C64EF1A
:104CB300F0C3648094805003024EAD901663E0F419
:104CC3006003024DD912BDFCEF7003024DD9901C55
:104CD30064E0FF3395E0FE7C007D3D1217B2747BE8
:104CE3002FF974123EFA7B01A3EBF0A3EAF0A3E9D8
:104CF300F0E4FD12C094E4FF12C55E7F0212C55EAC
:104D0300E4901C54F0901C54E0FFC39406501774B5
:104D1300072FF582E43400F583E0FF12C55E901C93
:104D230054E004F080DFE4901C54F0901C54E0FF46
:104D3300C39404501774552FF582E4341CF583E0B3
:104D4300FF12C55E901C54E004F080DFE4901C5415
:104D5300F0901C54E0FFC394065027901C65E0FBC1
:104D6300A3E0FAA3E02408F9E43AFA7E00E92FF974
:104D7300EE3AFA121705FF12C55E901C54E004F0D8
:104D830080CFE4901C54F0901C54E0FFC394045073
:104D930027901C65E0FBA3E0FAA3E02404F9E43ABE
:104DA300FA7E00E92FF9EE3AFA121705FF12C55EF3
:104DB300901C54E004F080CF901C65E0FBA3E0FA64
:104DC300A3E0F9E4FDFC12BE39D3EF648094804084
:104DD30005E4901C63F0901C64E0FF12A40F024EE4
:104DE300ADE4901C54F012BA53901C54E0245DF5CA
:104DF30082E4341CF583EFF0901C54E004F0E0C32C
:104E0300940640E2E4901C54F012BA53901C54E010
:104E13002459F582E4341CF583EFF0901C54E0042C
:104E2300F0E0C3940440E2E4901C54F012BA5390AF
:104E33001C54E004F0E0C3940640F1E4901C54F0E9
:104E430012BA53901C54E02455F582E4341CF583C4
:104E5300EFF0901C54E004F0E0C3940440E2901C93
:104E63002AE0FF901C55E06F7040901C2BE0FF90F0
:104E73001C56E06F7034901C2CE0FF901C57E0B57B
:104E83000728901C2DE0FF901C58E0B5071C901DCF
:104E9300AB7401F0A3741CF0A3745DF07B017A1C66
:0F4EA3007959129CE4E4901C63F0901C63E0FFCB
:014EB20022DD
:0FC675007E007F6E7D007B017A1A79570221D6F5
:039CE400901DA828
:109CE70012B294901DAEEBF0A3EAF0A3E9F04A702C
:109CF7000E12B221901DAEEBF0A3EAF0A3E9F090AB
:109D07001DAEE0FBA3E0FAA3E0F990000A12171ECC
:109D170030E003029DAAE9240AF9E43AFA1217058A
:109D2700440112177EE4FF901DA8E0FBA3E0FAA30D
:109D3700E0F98F8275830012171EFE901DAEE0FBBF
:109D4700A3E0FAA3E0F98F82758300EE1217900F54
:109D5700EFB404D3E4FF901DABE0FBA3E0FAA3E06C
:109D6700F98F8275830012171EFE901DAEE0FBA3CC
:109D7700E0FAA3E02404F9E43AFAEF7C0029F9ECCD
:109D87003AFAEE12177E0FEFB406CB901DAEE0FB4A
:109D9700A3E0FAA3E0240AF9E43AFA12170554FEFD
:039DA70012177E12
:019DAA002296
:03962F00901D7F0C
:1096320012B294901D82EBF0A3EAF0A3E9F04A6023
:1096420003029700F9901D82C9F0A3F0A3E9F07418
:10965200FF901C92F0A3F0A37404F0A37420F0A373
:10966200E4F0A3F0A3F0A3F0A3F0901D7FE0FBA32E
:10967200E0FAA3E0F974FFFDFC124EB3901D86EFF1
:10968200F0C3648094804076E0FF3395E0FE7C0076
:109692007D3D1217B2747B2FF974123EFAA3740146
:1096A200F0A3EAF0A3E9F0E4901D85F0901D87E0B5
:1096B200FBA3E0FAA3E0F9128B0FEF6039901D874C
:1096C200E0FBA3E0FAA3E0F912BCF4EF601C901DEA
:1096D2007FE0FBA3E0FAA3E0F912B29C901D82EBBB
:1096E200F0A3EAF0A3E9F04A700C901D85E004F0C3
:1096F200E0C3940640B6901D86E0FF12A40F901DB1
:0997020082E0FBA3E0FAA3E0F908
:01970B00223B
:08B29400EBF0A3EAF0A3E9F0DE
:0BB29C00901E61EBF0A3EAF0A3E9F0C4
:10B2A700E4A3F0901E64E0FFC3940A504BEF75F0DF
:10B2B7000BA42457F9741A35F0FA7B01C003C002B6
:10B2C700901E61E0FBA3E0FAA3E0F8AC02AD03D067
:10B2D70002D0037E007F041221B2EF7013901E6428
:10B2E700E075F00BA42457F9741A35F0FA7B0122A4
:0EB2F700901E64E004F080AB7B007A007900CA
:01B305002225
:10B22100E4901EB2F0901EB2E0FFC3940A501FEFEB
:10B2310075F00BA42457F582E4341AF583E0700607
:10B24100901EB2E0803E901EB2E004F080D712C69C
:10B25100AF7C007D0A1217C4901EB2EDF0901EB2B1
:10B26100E0FF75F00BA42461F582E4341AF583E064
:10B2710030E010901EB2E004F0E075F00A84E5F0D1
:10B28100F080DAEF75F00BA42457F9741A35F0FA4F
:02B291007B013F
:01B293002298
:0B8B0F00901E34EBF0A3EAF0A3E9F0A5
:108B1A00E4901E38F0901663E064017003028C043E
:108B2A0012BDFCEF7003028C04901E34E0FBA3E03C
:108B3A00FAA3E0F97D0112C094E4FF12C55E7F0139
:108B4A0012C55EE4901E37F0901E37E0FFC394060C
:108B5A00501774072FF582E43400F583E0FF12C53D
:108B6A005E901E37E004F080DFE4901E37F0901E1E
:108B7A0037E0FFC394045017742A2FF582E4341C9B
:108B8A00F583E0FF12C55E901E37E004F080DFE453
:108B9A00901E37F0E4FF12C55E901E37E004F0E045
:108BAA00C3940640EFE4901E37F0901E37E0FFC3EF
:108BBA0094045027901E34E0FBA3E0FAA3E02404B7
:108BCA00F9E43AFA7E00E92FF9EE3AFA121705FFAC
:108BDA0012C55E901E37E004F080CF901E34E0FB91
:108BEA00A3E0FAA3E0F9E4FDFC12BE39D3EF6480F6
:0F8BFA0094804006901E387401F0901E38E0FF02
:018C09002248
:0BBCF400901DB1EBF0A3EAF0A3E9F013
:10BCFF007B017A1D79B57D587C0212AB887B017A66
:10BD0F001D79B512B794EF701D1286F1901DB4EF27
:10BD1F00F030E5037F0122901DB4E0FF60DF20E3E8
:08BD2F00DC1292A280D77F0014
:01BD370022E9
:0EBF8400441C3CC0A80202441C2AC0A80203B0
:0BC12000901E86EBF0A3EAF0A3E9F00C
:10C12B0090000E121CC8E94A7004FEFF8014901E8A
:10C13B0086E0FBA3E0FAA3E0F99000111218A6FF2A
:02C14B00AEF054
:01C14D0022CF
:09C6D200900019E4F5F002198250
:0BA55D00901E1DEBF0A3EAF0A3E9F054
:10A56800900013121CC8E94A700302A601901E1D30
:10A57800E0FBA3E0FAA3E0F9900013121CC8C003A3
:10A58800C002C001901E1DE0FBA3E0FAA3E0F99011
:10A5980000191218A6D001D002D00329F9EA35F023
:10A5A800FA901E20EBF0A3EAF0A3E9F0901E1DE05C
:10A5B800FBA3E0FAA3E0F9900016121CC8C003C080
:10A5C80002C001901E20A3E0FAA3E0F9D3D082D004
:10A5D80083D0E0E99582EA9583501E901E20E0FB27
:10A5E800EF12177E901E1DE0FBA3E0FAA3E0F9909E
:09A5F8000019E475F001121916B6
:01A601002236
:03C6E5007F0122B0
:10A88A00901E89EBF0A3EAF0A3E9F0901E89E0FBA1
:10A89A00A3E0FAA3E0F99000111218A6FDACF0D3D8
:10A8AA00EF9DEE9C40028004AC06AD07AE04AF05F6
:10A8BA009000111218A6D39400E5F09400401E905F
:10A8CA001E89E0FBA3E0FAA3E02411F9E43AFA12A4
:10A8DA00187BC39FFDE5F09E8DF0121963901E89C7
:10A8EA00E0FBA3E0FAA3E0F99000111218A6D394B2
:10A8FA0000E5F09400400A90000EA3EE8FF00219D2
:10A90A00167B007A007900C003C002C001901E893C
:0FA91A00E0FBA3E0FAA3E0F990000E121CF82274
:03C6E8007F0022AE
:03C6EB007F0022AB
:03C6EE007F0022A8
:0BC6C700C2AF12C6A1D2AF1297E6224C
:10AD3200901E8E74FFF090165DE06078E4901E8D98
:10AD4200F012BA53901E8DE004F0E0C3940640F175
:10AD5200E4901E8DF012BA53901E8DE0242EF582DF
:10AD6200E4341CF583EFF0901E8DE004F0E0C39410
:10AD72000640E212BA53901E8CEFF012BA53901EA4
:10AD82008CE0B40821EF24FA600C24067018901E9F
:10AD92008E7401F08010901663E064016008124B1B
:10ADA20053901E8EEFF0901E8EE0D36480948050FC
:09ADB200031292A2901E8EE0FF34
:01ADBB002275
:0B79C100901D94EBF0A3EAF0A3E9F0A6
:1079CC004A70037F852290165DE070037F9D22AE86
:1079DC0004AF05ED6003027B15EE24F86003027B17
:1079EC0015901D94E0FBA3E0FAA3E0F990001D12A2
:1079FC00171E30E440900008740112179090000993
:107A0C00E412179090000A745E1217909000051201
:107A1C00171E547F90000B12179090000612171E21
:107A2C0090000C12179090000712171E90000D1268
:107A3C001790027AEF901D99E06003027AEF901C88
:107A4C0038E0FFF4601EEF601BE92404F9E43AFA15
:107A5C00901C6B7401F0A3741CF0A3742AF01266D2
:107A6C00C7EF6012901D94E0FBA3E0FAA3E024049E
:107A7C00F9E43AFA80067B017A1C793812962F9039
:107A8C001D9AEBF0A3EAF0A3E9F0901D9AA3E0FA9B
:107A9C00A3E04A604BE4A3F0901D9DE0FFC3940665
:107AAC005041901D9AE0FBA3E0FAA3E02404F9E412
:107ABC003AFA7E00E92FF9EE3AFA121705FD901DFD
:107ACC0094E0FBA3E0FAA3E02408F9E43AFAE92FE6
:107ADC00F9EE3AFAED12177E901D9DE004F080B895
:107AEC007FA12212BDFCEF70037F8F22901D94E0CA
:107AFC00FBA3E0FAA3E0F9901D99E0FD12ADBC7F69
:0B7B0C000812C55EE4FF12C55E7F0199
:017B1700224B
:10C09400E94A602B12ADBC7F0812C55E7F0612C54B
:10C0A4005EE4FF12C55E7F0112C55E7F0812C55EA5
:10C0B400E4FF12C55E7F0612C55E7F0412C55E22D0
:10C4C500900A6DE0FBA3E0FAA3E0F9121705FF90CF
:09C4D5000A6EE475F00112184F23
:01C4DE00223B
:10BC2100900A70E0FBA3E0FAA3E0F9EF12177E900F
:10BC31000A71E475F00112184F900A70A3E0FAA39B
:10BC4100E0D39012779582EA9583400E900A707442
:10BC510001F0A3740EF0A37478F0901279E004F06F
:09BC61007006901278E004F02254
:0BADBC00901E65EBF0A3EAF0A3E9F0A5
:10ADC7004A6075ED6016E4A3F07FFF12C55E901E22
:10ADD70068E004F0E0C3940640EF8036E4901E6814
:10ADE700F0901E68E0FFC394065027901E65E0FBB5
:10ADF700A3E0FAA3E02408F9E43AFA7E00E92FF980
:10AE0700EE3AFA121705FF12C55E901E68E004F0CD
:10AE170080CFE4901E68F0901E68E0FFC394065050
:10AE27001774072FF582E43400F583E0FF12C55E3F
:08AE3700901E68E004F080DFCA
:01AE3F0022F0
:0B66C700901C68EBF0A3EAF0A3E9F0E0
:1066D20090000112171EFFE4FCFDFE7810121AFA58
:1066E200C004C005C006C007901C68E0FBA3E0FA26
:1066F200A3E0F9121705FFE4FCFDFE7818121AFA5E
:10670200D003D002D001D000EF4BFFEE4AFEED499C
:10671200FDEC48FCC004C005C006C007901C68E040
:10672200FBA3E0FAA3E0F990000212171EFFE4FCBB
:10673200FDFE7808121AFAD003D002D001D000EF81
:106742004BFFEE4AFEED49FDEC48FCC004C005C01B
:1067520006C007901C68E0FBA3E0FAA3E0F99000F2
:106762000312171EFFD003D002D001D000EB4FFF5F
:10677200EAFEE9FDE8FC901C6E121BC3901C35E09A
:10678200FFE4FCFDFE7810121AFAC004C005C00630
:10679200C007901C34E0FFE4FCFDFE7818121AFAE0
:1067A200D003D002D001D000EF4BFFEE4AFEED49FC
:1067B200FDEC48FCC004C005C006C007901C36E0D2
:1067C200FFE4FCFDFE7808121AFAD003D002D001D1
:1067D200D000EF4BFBEE4AFAED49F9EC48F8A3E0A2
:1067E200FFEB4FFFEAFEE9FDE8FC901C72121BC3AF
:1067F200901C72E0FCA3E0FDA3E0FEA3E0FF901C6E
:106802006EE0F8A3E0F9A3E0FAA3E05FFFEA5EFE20
:10681200E95DFDE85CFC901C76121BC3901C6BE0EA
:10682200FBA3E0FAA3E0F990000112171EFFE4FCBB
:10683200FDFE7810121AFAC004C005C006C0071285
:106842001705FFE4FCFDFE7818121AFAD003D002F5
:10685200D001D000EF4BFFEE4AFEED49FDEC48FCC3
:10686200C004C005C006C007901C6BE0FBA3E0FAA1
:10687200A3E0F990000212171EFFE4FCFDFE780867
:10688200121AFAD003D002D001D000EF4BFFEE4A29
:10689200FEED49FDEC48FCC004C005C006C00790EF
:1068A2001C6BE0FBA3E0FAA3E0F990000312171EB1
:1068B200FFD003D002D001D000EB4FFFEAFEE9FD8A
:1068C200E8FC901C6E121BC3901C72E0FCA3E0FD5E
:1068D200A3E0FEA3E0FF901C6EE0F8A3E0F9A3E0C2
:1068E200FAA3E05FFFEA5EFEE95DFDE85CFC901C56
:1068F20076E0F8A3E0F9A3E0FAA3E0FBC3121AD60C
:106902007007901C7A04F08005E4901C7AF0901CC9
:036912007AE0FF29
:01691500225F
:1097E60090C00BE0FE90C00AE07C002400FFEC3E37
:1097F600FEEF7003EE64306002803BE4FFFE12C4AD
:10980600DFEF640E7003EE6463600280297F207EC2
:109816000012C4DFEF7003EE64036002801812C208
:109826002BE4FDFC7F22FE12C5D47F227E0012C4EB
:10983600DFEF540F60057EFF7F8B227F0A12C5CFB4
:109846007F0212C5CF7D807C097F047E0112C5D4BC
:10985600E4FDFC7F067E0112C5D4900008E0FE9070
:109866000007E0FDEEFCED7F587E0112C5D49000A6
:109876000AE0FE900009E0FDEEFCED7F5A7E011243
:10988600C5D490000CE0FE90000BE0FDEEFCED7FF1
:109896005C7E0112C5D4E4FDFC7F187E0112C5D49E
:1098A600E4FDFC7F167E0112C5D47DC07C007F12CC
:0A98B6007E0112C5D47E007F01225E
:1057CB00901BB3EBF0A3EAF0A3E9F0A3ECF0A3ED8D
:0157DB00F0DD
:1057DC00E4901BC2F0A3F0A3F0900A6AE0FBA3E0F4
:1057EC00FAA3E0F9C003C002C001900A6DE0FBA36C
:1057FC00E0FAA3E0F9D082D083D0E06B7008E965C1
:10580C00827003EA65837003025A70900A6DA3E0FC
:10581C00FAA3E0AE02FF900A6AA3E0FAA3E0C39FEA
:10582C00FFEA9E901BBEF0A3EFF0901BB6E0FEA328
:10583C00E0FF4E6029901BB3E0FBA3E0FAA3E0F974
:10584C0090000E121CC8E94A6014901BCAEBF0A31E
:10585C00EAF0A3E9F0EF5401901BC4F0801A901BFE
:10586C00BFE030E013E4FF12C55E901BBFE004F014
:10587C007006901BBEE004F0901BBEE0FEA3E0FFA0
:10588C00901BB7E02FFF901BB6E03EFE901BC0F0C4
:10589C00A3EFF0D394EEEE94054002806290C00426
:1058AC0074C0F0A3E4F0901BC0E0FEA3E090C0062F
:1058BC00F0EEA3F07B017A1B79C57D057C0012AB61
:1058CC00887B017A1B79C512B794EF70187F387EEC
:1058DC000112C4DFEE30E0E9901BC0E0FFA3E0A3AF
:1058EC00CFF0A3EFF0901BC2E07002A3E070057E36
:1058FC00FF7F8F227F387E0112C4DFEF30E7057EF9
:10590C00FF7F8C22E4901BB8F0A3F0901BBEE0FE4E
:10591C00A3E0FFC3901BB9E09F901BB8E09E5048DA
:10592C00900A6DE0FBA3E0FAA3E0F912170590C012
:10593C0000F0900A6EE475F00112184F900A6DE0B9
:10594C00FBA3E0FAA3E0F912170590C001F0900A4E
:10595C006EE475F00112184F901BB9E02402F09020
:10596C001BB8E03400F080A3901BC4E0600E901BC9
:10597C00B7E024FFF0901BB6E034FFF0E4901BB8C6
:10598C00F0A3F0901BB6E0FEA3E0FFC3901BB9E0C0
:10599C009F901BB8E09E503E901BCAE0FBA3E475A1
:1059AC00F001121865A9F0FA12170590C000F090DA
:1059BC001BCAE0FBA3E475F001121865A9F0FA12FA
:1059CC00170590C001F0901BB9E02402F0901BB8B1
:1059DC00E03400F080AD901BC4E06015901BCAE071
:1059EC00FBA3E0FAA3E0F912170590C000F0A3E4C2
:1059FC00F0901BBA121BCF000000007F407E0D7D83
:105A0C00037C00901BBAE0F8A3E0F9A3E0FAA3E052
:105A1C00FBC3121AD6504D7F287E0112C4DF901B97
:105A2C00B8EEF0A3EFF0EE5486FEEF54C04E600CCF
:105A3C00901BC274FFF0A3748CF08028901BB8E00C
:105A4C0020E021901BBAE0FCA3E0FDA3E0FEA3E064
:105A5C002401FFE43EFEE43DFDE43CFC901BBA1245
:0C5A6C001BC38097901BC2E0FEA3E0FF6C
:015A7800220B
:106D6800E4901D65F0A3F07F247E0112C4DFEE20BD
:106D7800E03B7B017A1D79607D057C0012AB887B46
:106D8800017A1D796012B794EF70137F247E011287
:106D9800C4DFEE30E0E9901D65E4F0A304F0901D37
:106DA80065E07002A3E070057EFF7F872290C00136
:106DB800E0FE90C000E07C002400FFEC3E901D5CEB
:106DC800F0A3EFF0901D5CE0FEA3E0FF12C6F29086
:106DD800C001E0FE90C000E07C002400FFEC3E9083
:106DE8001D5EF0A3EFF0901D5EE0FCA3E0FD5401F2
:106DF800901D67F0901278E0FEA3E0FFC374FE9F39
:106E0800FF74039EFED3ED9FEC9E4003026F3B9000
:106E18001D5EE0FEA3E0FF901D65EEF0A3EFF0EE2F
:106E2800FF12BC21901D5EA3E0FF12BC21901D67DC
:106E3800E0600E901D5FE024FFF0901D5EE034FFDF
:106E4800F0E4FFFED3901D5FE09F901D5EE09E5032
:106E580003026EEA90C000E0FD900A70E0FBA3E038
:106E6800FAA3E0F9ED12177E900A70A3E475F00119
:106E780012184FFAD3901277E5F09582EA9583407D
:106E88000E900A707401F0A3740EF0A37478F09059
:106E9800C001E0FD900A70E0FBA3E0FAA3E0F9ED81
:106EA80012177E900A70A3E475F00112184FFAD3F6
:106EB800901277E5F09582EA9583400E900A7074F7
:106EC80001F0A3740EF0A37478F0901279E0240214
:106ED800F0901278E03400F074022FFFE43EFE02D6
:106EE8006E4C901D67E0606090C000E0FF900A70F3
:106EF800E0FBA3E0FAA3E0F9EF12177E900A70A373
:106F0800E475F00112184FFAD3901277E5F09582E4
:106F1800EA9583400E900A707401F0A3740EF0A3F2
:106F28007478F0901279E004F07006901278E0041A
:106F3800F080157D407C007F027E0112C5D4901D33
:106F48006574FFF0A3748DF0901D65E0FEA3E0FF6B
:016F58002216
:10C4DF00EF90C00AF0EEA3F090C00DE0FE90C00CFC
:0AC4EF00E07C002400FFEC3EFE227A
:05C5CF00E4FDFC7E010B
:0FC5D400EF90C00AF0EEA3F0EDA3F0ECA3F0227D
:10C22B007D407C007F147E0112C5D47F021E12C498
:10C23B00F97F017E0012C4F97F147E0112C4DF7FE7
:0BC24B00367E0112C4DFEF30E7E7226F
:01C6F2002225
:10C5E3007F347E0112C4DFEF30E7057E007F012236
:03C5F300E4FEFF64
:01C5F6002222
:106B6400901CC1EFF0A3ECF0A3EDF0A3EAF0A3EBCB
:016B7400F030
:106B7500901CC8E0FBA3E0FAA3E0F990000112170E
:106B85001EFD121705FEEDFFE4FCFD901CCE121B49
:106B9500C3901CCEE0F8A3E0F9A3E0FAA3E0FBC0A4
:106BA50000C001C002C003901CC8E0FBA3E0FAA32B
:106BB500E0F990000212171EFE90000312171EFD49
:106BC500EDFFE4FCFDD003D002D001D000EB2FFF98
:106BD500EA3EFEED39FDEC38FC901CCE121BC3904D
:106BE5001CCEE0F8A3E0F9A3E0FAA3E0FBC000C0E7
:106BF50001C002C003901CCBE0FBA3E0FAA3E0F9BF
:106C050090000112171EFD121705FEEDFFE4FCFDB5
:106C1500D003D002D001D000EB2FFFEA3EFEED39C4
:106C2500FDEC38FC901CCE121BC3901CCEE0F8A3E3
:106C3500E0F9A3E0FAA3E0FBC000C001C002C00375
:106C4500901CCBE0FBA3E0FAA3E0F9900002121739
:106C55001EFE90000312171EFDEDFFE4FCFDD003A0
:106C6500D002D001D000EB2FFFEA3EFEED39FDEC5E
:106C750038FC901CCE121BC3901CCEE0F8A3E0F9A3
:106C8500A3E0FAA3E0FB901CC1E0FFE4FCFDFEEBF2
:106C95002FFFEE3AFEED39FDEC38FC901CCE121BB1
:106CA500C3901CCEE0F8A3E0F9A3E0FAA3E0FB90C3
:106CB5001CC2E0FEA3E0FFE4FCFDEB2FFFEA3EFE75
:106CC500ED39FDEC38FC901CCE121BC3901CCEE0B8
:106CD500F8A3E0F9A3E0FAA3E0FB901CC4E0FEA34F
:106CE500E0FFE4FCFDEB2FFFEA3EFEED39FDEC385D
:106CF500FC901CCE121BC3901CCEE0F8A3E0F9A3B8
:106D0500E0FAA3E0FB901CC6E0FEA3E0FFE4FCFD77
:106D1500EB2FFFEA3EFEED39FDEC38FC901CCE1260
:106D25001BC3901CC1E0B4112B901CCEE0F8A3E06E
:106D3500F9A3E0FAA3E0FB901CC2E0FEA3E0FFE4A8
:106D4500FCFDEB2FFFEA3EFEED39FDEC38FC901C17
:106D5500CE121BC3901CCEE0FCA3E0FDA3E0FEA376
:026D6500E0FF4D
:016D67002209
:1085E300901D68121BC3901D6CEBF0A3EAF0A3E986
:0185F300F097
:1085F400A3E07002A3E070030286E2901D6FE0FC2A
:10860400A3E0FD5401901D73F0ECC313FFED139030
:108614001D6FCFF0A3EFF0901D6F74FFF5F01218EB
:108624006545F06068901D6CE0FBA3E475F00112F1
:108634001865A9F0FA121705901D71F0A3E4F090E3
:108644001D6CE0FBA3E475F001121865A9F0FA12A1
:108654001705FF901D72E02FF0901D71E03400F0BB
:10866400901D68E0F8A3E0F9A3E0FAA3E0FB901DF5
:1086740071E0FEA3E0FFE4FCFDEB2FFFEA3EFEED1C
:1086840039FDEC38FC901D68121BC3808A901D7361
:10869400E0604B901D6CE0FBA3E0FAA3E0F9121735
:1086A400057F00FE901D71F0A3EFF0901D71EEF0B8
:1086B400A3EFF0901D68E0F8A3E0F9A3E0FAA3E0CB
:1086C400FB901D71E0FEA3E0FFE4FCFDEB2FFFEA4D
:1086D4003EFEED39FDEC38FC901D68121BC3901D65
:0C86E40068E0FCA3E0FDA3E0FEA3E0FFC3
:0186F0002267
:10B377008052901E69E0FCA3E0FDA3E0FEA3E0FF7E
:10B387007810121AE7EC4D4E4F6041901E69A3A347
:10B39700E0FEA3E0FFE4FDFCC004C005C006C00753
:10B3A700901E69E0FCA3E0FDA3A3E07810121AE762
:10B3B700D003D002D001D000EF2BFFEE3AFEED39DB
:10B3C700FDEC38FC901E69121BC380A6901E69E035
:10B3D700FCA3E0FDA3E0FEA3E0FF121AA5E4FDFC39
:01B3E7002243
:10AB8800901B36EBF0A3EAF0A3E9F0A3ECF0A3EDF9
:10AB9800F012C6AF901B36E0FBA3E0FAA3E0F9EE93
:10ABA8008FF0121963901B36E0FBA3E0FAA3E0F9DB
:10ABB80012187BFF901B3AE02FFF901B39E035F00D
:10ABC8009000028FF01219829000021218A6FFAEB0
:10ABD800F012187BFDACF0D39FEC9E901B36E0FB87
:10ABE800A3E0FAA3E0F95006900004E48020C3E44F
:10ABF8009DFFE49CFEC3901B3AE09FFF901B39E049
:10AC08009E9000028FF012198290000474011217AE
:02AC1800902288
:0BB79400901B36EBF0A3EAF0A3E9F0F5
:10B79F0012C6AF901B36E0FBA3E0FAA3E0F99000CE
:10B7AF000412171E601E12187BFDC3EF9DEE95F05D
:10B7BF0050309000021218A6FDD3EF9DEE95F04089
:10B7CF00217F01229000021218A6FDD3EF9DEE9566
:10B7DF00F0500C12187BFDC3EF9DEE95F050037FD8
:04B7EF0001227F00B4
:01B7F3002233
:0CC6AF00C2AF900A76E0FEA3E0FFD2AF1D
:01C6BB00225C
:10C4F9007B017A1B7931AD07AC0612AB887B017AD7
:09C509001B793112B794EF60F4C4
:01C512002206
:10C55E00900A6AE0FBA3E0FAA3E0F9EF12177E90CF
:09C56E000A6BE475F00102184F9C
:10BA5300900A73E0FBA3E0FAA3E0F9121705FFC213
:10BA6300AF901279E024FFF0901278E034FFF0D227
:10BA7300AF900A74E475F00112184F900A73A3E0B3
:10BA8300FAA3E0D39012779582EA9583400E900A49
:0EBA9300737401F0A3740EF0A37478F07E00BB
:01BAA1002282
:1090CF00901E8FEBF0A3EAF0A3E9F0901E8FA3E0C0
:1090DF00FAA3E04A70030291B9901E8FE0FBA3A39D
:1090EF00E0F9900020743C121790900026740275DE
:1090FF00F00012198212C6AFE4FCFDC004C005C017
:10910F0006C007901E8FE0FBA3E0FAA3E0F99000E2
:10911F001C12171EFFE4FE7810121AFAD003D002A9
:10912F00D001D000EF2BFFEE3AFEED39FDEC38FC0D
:10913F00EF2401FFE43EFEE43DFDE43CFC901E8F76
:10914F00E0FBA3E0FAA3E0F9900034121B57900064
:10915F001FE4121790900022E4121790900021E460
:10916F00121790900024E4F5F0121982900023E476
:10917F00121790900028121C000000000090002C85
:10918F00121C0000000000900030121C00000000B4
:10919F0000900038E4F5F012198290003AE4F5F0EF
:0B91AF0012198290003CE4121790227D
:0E8A1300901DBAEFF0A3EBF0A3EAF0A3E9F098
:108A21004A6023901DBBE0FBA3E0FAA3E0F99000AC
:108A31001C12171E75F03DA42499F582E5F034123D
:108A4100F583E020E0037F8622901DBAE014600EDA
:108A51001460432402705590001F7401803390000C
:108A61001F74021217907D02129FF3D3EF6480945A
:108A710080400F7B017A1D79BE7DA07C8C12AB8872
:108A8100802D901DBBE0FBA3E0FAA3E0F990001F4D
:108A9100E41217908019901DBBE0FBA3E0FAA3E05C
:108AA100F990001F74011217907F01227F0022901C
:108AB1001DBBE0FBA3E0FAA3E0F990001F12171E13
:108AC100FF64046036EF6033901DBAE0B4011C7B93
:108AD100017A1D79BE12B794EF6010901DBBE0FBC7
:108AE100A3E0FAA3E0F912B6D38010901DBBE0FB1E
:108AF100A3E0FAA3E0F912B7F480B4901DBBE0FB48
:0D8B0100A3E0FAA3E0F990001F12171EFF79
:018B0E002244
:0B22CE00901BFDEBF0A3EAF0A3E9F089
:1022D900901B587401F0A3741CF0A37404F0901BB4
:1022E900FDE0F9A3E0FAA3E0901B5BC9F0A3EAF0D3
:1022F900A3E9F07B017A1C7906123671EF70081296
:1023090092A27EFF7FFD22901BFDE0FBA3E0FAA3D2
:10231900E0F9121C59901C0AEBF0A3EAF0A3E9F0CA
:1023290090001F12171EB40A0040030226139023BF
:102339003EF828287302235C0223B10224B3022445
:102349002202262F0225480225B902261302261346
:102359000225F91292A2901C0AE0FBA3E0FAA3E07D
:10236900F990002112171E20E23B12C007901C0AA7
:10237900E0FBA3E0FAA3E0F990001D12171EB44098
:102389002490001C12171EFF12A40F7B007A0079FB
:1023990000C003C002C001901BFDE0FBA3E0FAA34B
:1023A900E0F9121C7902260E1292A2901C0AE0FB97
:1023B900A3E0FAA3E0F990002112171EFF30E2030F
:1023C90002268C30E41212C007901C13EFF0D3647C
:1023D900809480404102296E901C0AE0FBA3E0FA38
:1023E900A3E0F990002C121B0D900028121B577DB9
:1023F90012129FF3901C13EFF0D36480948040165F
:10240900901C0AE0FBA3E0FAA3E0F990001F740313
:1024190012179002268C022AAD901C0AE0FBA3E059
:10242900FAA3E0F990002112171EFF30E4075406C1
:10243900700302262F1292A2901C0AE0FBA3E0FA75
:10244900A3E0F990002112171E30E2181290CF90E4
:102459001C0AE0FBA3E0FAA3E0F990001F74011243
:1024690017908043901C0AE0FBA3E0FAA3E0F990DF
:10247900002112171E30E12C900028121B0DEF24A9
:10248900FFFFEE34FFFEED34FFFDEC34FFFC90005E
:102499002C121B93C3121AD6700A901C0A7D1212B1
:1024A9009FEB800312BFFC02268C1292A2901C0A99
:1024B900E0FBA3E0FAA3E0F990002112171E30E235
:1024C900030226B1901C0AE0FBA3E0FAA3E0F9900D
:1024D900002112171EFF30E40320E12512C00790E6
:1024E9001C13EFF0D3648094804013901C0AE0FB26
:1024F900A3E0FAA3E0F9900020743C0225B3022A74
:10250900AD901C0AE0FBA3E0FAA3E0F990001F7468
:102519000412179012B9581298C0901C13EFF0D3F7
:10252900648094804016901C0AE0FBA3E0FAA3E0C3
:10253900F9900020743C12179002298D022AAD12DD
:1025490092A2901C0AE0FBA3E0FAA3E0F990002212
:1025590012171E30E0447D1112C158D3EF648094E4
:10256900804037901C0AE0FBA3E0FAA3E02438F985
:10257900E43AFA7D327C0012AB88901C0AE0FBA396
:10258900E0FAA3E0F912B9581298C0901C13EFF0C1
:10259900D3648094805003022AB0901C0AE0FBA304
:1025A900E0FAA3E0F990001F74061217900227635E
:1025B900901C0AE0FBA3E0FAA3E0F99000221217AD
:1025C9001E30E00312B9581292A21298C0901C133F
:1025D900EFF0D3648094804014901C0AE0FBA3E0E0
:1025E900FAA3E0F990001FE41217908018022AADAF
:1025F900901C0AE0FBA3E0FAA3E0F990001FE412A3
:1026090017901292A27EFF7FFA22901C0AE0FBA388
:10261900E0FAA3E0F990001F12171ED3940A4006AE
:1026290012B6D3022AA8901C0AE0FBA3E0FAA3E0A1
:10263900F9900028121B0D901C0F121BC390002C3F
:10264900121B0D901C0FE0F8A3E0F9A3E0FAA3E038
:10265900FBC3121AD6602F129DAB1292A2901C0ACC
:10266900E0FBA3E0FAA3E0F990002112171E20E293
:10267900121298CB901C13EFF0D36480948050030E
:10268900022AB0022763901C0AE0FBA3E0FAA3E048
:10269900F990002112171E30E2351292A2901C0AFD
:1026A900E0FBA3E0FAA3E0F990001C12171EFF1249
:1026B900A40F7B007A007900C003C002C001901BFF
:1026C900FDE0FBA3E0FAA3E0F9121C79022AA89025
:1026D9001C0AE0FBA3E0FAA3E0F990002112171EFF
:1026E90030E1171292A212BFFC901C13EFF0D364D1
:1026F90080948040028063022AAD901C0AE0FBA30B
:10270900E0FAA3E0F990002112171E20E4061292C4
:10271900A2022A74901C0AE0FBA3E0FAA3E0F99054
:10272900001F12171E64046008900020743C1217E1
:102739009090001F7404121790D3901AC8E0940067
:10274900901AC7E0940240181292A21298C0901CE5
:1027590013EFF0D3648094804003022A74022AADF7
:10276900E4901C0DF0A3F0901C06E0F8A3E0F9A397
:10277900E0FAA3E0FBC000C001C002C003A3E0FB74
:10278900A3E0FAA3E0F990002312171EFF901AC8DC
:10279900E02FFD901AC7E03400FC12187BFBAAF069
:1027A900C002C003901C0AE0FBA3E0FA90000212E9
:1027B90018A6FF901CC6E5F0F0A3EFF0A37401F092
:1027C900A3741CF0A3742AF0901C0AA3A3E02404A8
:1027D900F9E43AFA901CCBEBF0A3EAF0A3E9F0D0C4
:1027E90003D0027F06126B64D003D002D001D0005F
:1027F900EB2FFFEA3EFEE93DFDE83CFC901C06128A
:102809001BC3901AC7E0FEA3E0FF901C02EEF0A3E1
:10281900EFF04E70030228EBE4901C01F0A3E0FEF8
:10282900A3E0FF901C0AE0FBA3E0FAA3E0F912C6BB
:10283900D212BA53901C00EFF0A3E0901C00700F65
:10284900E0901C0DF0A3E4F0901C0104F0803FE03F
:10285900FF901C0EE02FF0901C0DE03400F0901C4E
:1028690006E0F8A3E0F9A3E0FAA3E0FB901C0DE071
:10287900FEA3E0FFE4FCFDEB2FFFEA3EFEED39FD90
:10288900EC38FC901C06121BC3E4901C01F0901C50
:1028990000E0FF901C0AE0FBA3E0FAA3E0F912A50F
:1028A9005D901AC774FFF5F012184F45F0708290C9
:1028B9001C01E06041901C06E0F8A3E0F9A3E0FAEE
:1028C900A3E0FB901C0DE0FEA3E0FFE4FCFDEB2F71
:1028D900FFEA3EFEED39FDEC38FC901C06121BC3E5
:1028E9008014901C0AE0FBA3E0FAA3E0F990001918
:1028F900E4F5F0121982901C06E0FCA3E0FDA3E0C8
:10290900FEA3E0FF12B377901C06121BC3901C04B0
:10291900E0FEA3E0FFE4FCFDA3E0F8A3E0F9A3E0F7
:10292900FAA3E0FBC3121AD660081292A27EFF7FB7
:10293900FC22129DAB901C02E07002A3E0702812E9
:1029490092A2901C0AE0FBA3E0FAA3E0F990002C04
:10295900121B0D900028121B5790002212171E30CF
:10296900E003022A0E801D901C0AE0FBA3E0FAA3F3
:10297900E0F912C6E5901C13EFF01292A2901C1315
:10298900E0B4A204E4FEFF22901C0AE0FBA3E0FAF3
:10299900A3E0F990002C121B93901C02E0FEA3E027
:1029A900FFEF2BFFEE3AFEE439FDE438FC901C0AF8
:1029B900E0FBA3E0FAA3E0F9900028121B5790006E
:1029C9002212171E20E03E901C0AE0FBA3E0FAA3A6
:1029D900E0F990001D12171EFF30E00A9000111255
:1029E90018A645F06004EF20E0121298CB901C1352
:1029F900EFF0D3648094805003022AB0901C02E067
:102A0900FEA3E0FF22901C0AE0FBA3E0FAA3E0F991
:102A1900900028121B0DEF2401FFE43EFEE43DFD6A
:102A2900E43CFC900028121B571298CB901C13EF22
:102A3900F0D364809480406C901C0AE0FBA3E0FA18
:102A4900A3E0F990001F7409121790E92438F9E4FA
:102A59003AFA7D327C0012AB88901C0A12C14E9062
:102A69001C13EFF0D36480948040057EFF7F892298
:102A7900901C0AE0FBA3E0FAA3E0F990001C1217EE
:102A89001EFF12A40F7B007A007900C003C002C0A8
:102A990001901BFDE0FBA3E0FAA3E0F9121C797E8B
:0D2AA900FF7FFF22901C13E0FF3395E0FE3D
:012AB60022FD
:0B9DAB00901C0AE0FBA3E0FAA3E0F923
:0B9DB600901DC3EBF0A3EAF0A3E9F05E
:109DC1009000241218A6FF901DC6E5F0F0A3EFF055
:109DD100900034121B0D901DC8121BC3901DC6E0CC
:109DE1007002A3E07003029E6C901DC3E0FBA3E030
:109DF100FAA3E0F9900030121B93C000C001C00229
:109E0100901DC6E0FEA3E0FFE4FCFDA3E0F8A3E0A3
:109E1100F9A3E0FAA3E02FFFEA3EFEED39FDEC38AD
:109E2100FCD002D001D000C3121AD6703E901DC6DC
:109E3100E0FEA3E0FF901DC3E0FBA3E0FAA3E0F97D
:109E410012A88A901DC3E0FBA3E0FAA3E0F99000F9
:109E510024E4F5F0121982900020743C12179090BE
:0B9E61000030121B0D900034121B5744
:019E6C0022D3
:0B6F5900901E23EBF0A3EAF0A3E9F088
:106F64004A70057EFF7F8522901E23E0FBA3E0FA92
:106F7400A3E0F990001F12171EFDC3940250057E72
:106F8400FF7FFA2290002012171E6006EDD3940AA8
:106F9400400812B6D37EFF7FFF22901E23E0FBA39E
:106FA400E0FAA3E0F990001F12171E64027027E9AB
:106FB4002438F9E43AFA12B794EF6017901E237D4F
:106FC40002129FEB901E28EFF0D36480948050034C
:106FD40002710C027058901E23E0FBA3E0FAA3E0B8
:106FE400F99000241218A645F06029E92438F9E440
:106FF4003AFA12B794EF7003FEFF22901E23E0FBCF
:10700400A3E0FAA3E02438F9E43AFA7D327C0012D2
:10701400AB888044901E23E0FBA3E0FAA3E0F99040
:10702400001F12171EC39405402EE92438F9E43AD0
:10703400FA12B794EF6021901E23E0FBA3E0FAA3B9
:10704400E02438F9E43AFA7D327C0012AB88901ED1
:107054002312C14EE4FEFF22901E23E0FBA3E0FABC
:10706400A3E0F912C120901E26EEF0A3EFF0901ECB
:1070740023E0FBA3E0FAA3E0F9900024EE8FF012E2
:107084001982EF4E7003FEFF229000261218A6FF0D
:10709400AEF0D3901E27E09F901E26E09E4005EEA2
:1070A400F0A3EFF0D3901E27E09400901E26E09406
:1070B4000240067402F0A3E4F09000241218A6FF24
:1070C400901E26E065F07003A3E06F60057EFF7FED
:1070D400FE229000217418121790123B8B901E28E8
:1070E400EFF0640160028020901E23E0FBA3E0FA2D
:1070F400A3E0F9A3E0FCA3E0FD12BE39901E28EF43
:10710400F0D3648094805007E0FF3395E0FE229032
:107114001E23E0FBA3E0FAA3E02438F9E43AFA7D65
:10712400327C0012AB88901E23E0FBA3E0FAA3E0BC
:0A713400F99000241218A6FFAEF037
:01713E00222E
:10B6D300901E92EBF0A3EAF0A3E9F0901E92A3E090
:10B6E300FAA3E04A604A901E92E0FBA3A3E0F9901C
:10B6F300001FE41217907B007A007900C003C00298
:10B70300C001901E92E0FBA3E0FAA3E0F990000EC3
:10B71300121CF8901E92E0FBA3E0FAA3E0F990005C
:10B7230011E4F5F0121982900024E4F5F012198265
:01B7330022F3
:10A7EA00901E95EBF0A3EAF0A3E9F0901E95A3E082
:10A7FA00FAA3E04A700302A889901E95E0FBA3A37E
:10A80A00E0F9900024E4F5F01219827B007A0079CD
:10A81A0000C003C002C001901E95E0FBA3E0FAA3AA
:10A82A00E0F990000E121CF8901E95E0FBA3E0FAE6
:10A83A00A3E0F9900011E4F5F012198290001F12BA
:10A84A00171EFF64036009EF64046004EFB4072F66
:10A85A00901E95E0FBA3E0FAA3E02438F9E43AFA63
:10A86A007D327C0012AB88901E95E0FBA3E0FAA330
:10A87A00E0F990001F74051217907D1112C1582239
:10BDBD00901E98EBF0A3EAF0A3E9F0901E98E0FB3B
:10BDCD00A3E0FAA3E0F94A602512A7EA901E98E0D5
:10BDDD00FBA3E0FAA3E0F990001F12171EFFD39406
:0FBDED0000400BEFD3940A500512B7F480DE220A
:0BB7F400901E29EBF0A3EAF0A3E9F09F
:10B7FF00E4901E2DF0A3F012C0F2901E2CEFF0304B
:10B80F00E0137B017A1E79291222CE901E2DEEF0C5
:10B81F00A3EFF08010901E2CE030E1097B017A1E1F
:10B82F00792902478D901E2DE0F47004A3E06489FE
:10B83F006011901E29E0FBA3E0FAA3E0F94A600330
:03B84F00126F591C
:01B8520022D3
:0B367100901B55EBF0A3EAF0A3E9F07A
:10367C00E4901B73F012BA53EF901B60F0A3E4F0CC
:10368C0012BA53901B61E02FF0901B60E03EF012D9
:10369C00BA53EF901B5EF0A3E4F012BA53901B5F89
:1036AC00E02FF0901B5EE03EF012BA53901B67EFD8
:1036BC00F012BA53901B68EFF012BA53901B69EFDB
:1036CC00F012BA53901B6AEFF012BA53901B6BEFC7
:1036DC00F012BA53901B6CEFF012BA53901B6DEFB3
:1036EC00F012BA53901B6EEFF0901B67E0FEA3E054
:1036FC00FFE4FCFD901B74121BC3901B74E0F8A339
:10370C00E0F9A3E0FAA3E0FB901B69E0FEA3E0FF65
:10371C00E4FCFDEB2FFFEA3EFEED39FDEC38FC90AE
:10372C001B74121BC3901B74E0F8A3E0F9A3E0FA1E
:10373C00A3E0FB901B6BE0FEA3E0FFE4FCFDEB2F92
:10374C00FFEA3EFEED39FDEC38FC901B74121BC3F6
:10375C00901B74E0F8A3E0F9A3E0FAA3E0FB901B44
:10376C006DE0FEA3E0FFE4FCFDEB2FFFEA3EFEED77
:10377C0039FDEC38FC901B74121BC312BA53901B0E
:10378C0066EFF012BA53901B65EFF0901B74E0F8E3
:10379C00A3E0F9A3E0FAA3E0FB901B66E0FE901B0C
:1037AC0065E0FDEDFFE4FCFDEB2FFFEA3EFEED399D
:1037BC00FDEC38FC901B74121BC3901B66E054F09C
:1037CC00F0E01313543FFFF0C3901AC8E09F901A17
:1037DC00C7E094004008901B66E094125003023A34
:1037EC000C901B66E0FFC3901AC8E09FF0901AC7BC
:1037FC00E09400F012BA53EF901B62F0A3E4F012C5
:10380C00BA53901B63E02FF0901B62E03EF0901BCC
:10381C0074E0F8A3E0F9A3E0FAA3E0FB901B62E0EC
:10382C00FEA3E0FFE4FCFDEB2FFFEA3EFEED39FDCD
:10383C00EC38FC901B74121BC312BA53EFF9901B9B
:10384C0058E0FBA3E0FAA3E0C975F000121963126B
:10385C00BA53901B58E0FBA3E0FAA3E0F9EE8FF00B
:10386C001218DE901B66E0C39412901B64F0901B40
:10387C0074E0F8A3E0F9A3E0FAA3E0FBC000C001F8
:10388C00C002C00312BA53EFFEE4FCFDD003D00219
:10389C00D001D0002BFFEA3EFEED39FDEC38FC9058
:1038AC001B74121BC3901B74E0F8A3E0F9A3E0FA9D
:1038BC00A3E0FBC000C001C002C00312BA53E4FC79
:1038CC00FDD003D002D001D000EB2FFFEA3EFEED7D
:1038DC0039FDEC38FC901B74121BC3901B64E02464
:1038EC00FEF0E07089901B74E0FCA3E0FDA3E0FE09
:1038FC00A3E0FF901B55E0FBA3E0FAA3E0F9121B39
:10390C003D901B5EE0FEA3E0FFA3E0FCA3E0FD7B8B
:10391C00017A1B7925901D3E7406F0128023901BB2
:10392C006FEBF0A3EAF0A3E9F04A6003023AB4901B
:10393C001B5EE0FEA3E0FF7B017A1B7925901D3E08
:10394C007406F0E4FDFC128023901B6FEBF0A3EAED
:10395C00F0A3E9F04A7025901B5EE0FEA3E0FF7B2C
:10396C00017A1A79D0901D3E7406F0E4FDFC1280A9
:10397C0023901B6FEBF0A3EAF0A3E9F0901B6FE030
:10398C00FBA3E0FAA3E0F94A6020901B65E030E16C
:10399C0019901B60E0FFA3E0900002CF8FF012198A
:1039AC0082901B737401F0023AB4901B65E030E214
:1039BC0002804D901B5EE0FEA3E0FF12C1A9901B9C
:1039CC0072EFF0901B5EE0FCA3E0FDA3E0FFA3E030
:1039DC00901C92CFF0A3EFF0A37406F0901B72E052
:1039EC00901C95F0A3E4F0A3F0A3F0A3F0A3F07B5C
:1039FC00017A1B7925124EB3C3EF64809480501D5D
:103A0C007B007A007900C003C002C001901B5BE010
:103A1C00FBA3E0FAA3E0F9121C797F0022EF3395A7
:103A2C00E0FE7C007D3D1217B2747B2FF974123EC0
:103A3C00FA7B01901B6FEBF0A3EAF0A3E9F0900086
:103A4C001FE4121790901AC7E0FEA3E0FF4E601B14
:103A5C00E4FD901B67E0F8A3E0F9A3E0FAA3E02FE4
:103A6C00FFEA3EFEED39FDEC388018901B67E0FC58
:103A7C00A3E0FDA3E0FEA3E02401FFE43EFEE43D51
:103A8C00FDE43CFC901B6FE0FBA3E0FAA3E0F99093
:103A9C000028121B57901B6FE0FBA3E0FAA3E0F980
:103AAC0090001D7440121790901B6FE0FBA3E0FA7E
:103ABC00A3E0F9C003C002C001901B5BE0FBA3E0D4
:103ACC00FAA3E0F9121C79901B65E0FF901B6FE0E4
:103ADC00FBA3E0FAA3E0F9900022EF1217909000FC
:103AEC0021EF121790901B62E0FFA3E0900026CF0D
:103AFC008FF0121982901B66E090002312179090A1
:103B0C001B67E0FCA3E0FDA3E0FEA3E0FF90002C0C
:103B1C00121B57901B6BE0FCA3E0FDA3E0FEA3E09F
:103B2C00FF900030121B57901B73E0B40113901BD5
:103B3C006FE0FBA3E0FAA3E0F990001F74011217E9
:103B4C0090901B6FE0FBA3E0FAA3E0F99000041245
:103B5C00171E7028901B25E0900004121790901BE4
:103B6C0026E0900005121790901B27E0900006129B
:0E3B7C001790901B28E09000071217907F0111
:013B8A002218
:0B3B8B00901D0EEBF0A3EAF0A3E9F0A0
:103B960090002112171EFF901D1BF0900024121892
:103BA600A6FD901D19E5F0F0A3EDF0EF30E13DE044
:103BB6002418F0901D19E03400F0901D187460F080
:103BC600901D12121BCF00000204901D12E0FCA3F0
:103BD600E0FDA3E0FEA3E02400FFEE3402FEE43D98
:103BE600FDE43CFC901D12121BC3801E901D1AE0C2
:103BF6002414F0901D19E03400F0901D187450F054
:103C0600901D12121BCF00000000901D12E0F8A3B9
:103C1600E0F9A3E0FAA3E0FBC000C001C002C003C4
:103C2600901D19E0FCA3E0FD901D0EE0FBA3E0FA59
:103C3600A3E0F912187BFBAAF0C002C003901D0E88
:103C4600E0FBA3E0FA9000021218A6FF901CC6E55E
:103C5600F0F0A3EFF0A37401F0A3741CF0A3742A90
:103C6600F0901D0EA3A3E02404F9E43AFA901CCBCD
:103C7600EBF0A3EAF0A3E9F0D003D0027F06126BC3
:103C860064D003D002D001D000EB2FFFEA3EFEE95C
:103C96003DFDE83CFC901D12121BC3901D12E0F87E
:103CA600A3E0F9A3E0FAA3E0FBC000C001C002C094
:103CB60003901D0EE0FBA3E0FAA3E0F99000341296
:103CC60018A6FFE4FCFDD003D002D001D000EB2FF4
:103CD600FFEA35F0FEED39FDEC38FC901D12121BA3
:103CE600C3901D12E0F8A3E0F9A3E0FAA3E0FBC03D
:103CF60000C001C002C003901D0EE0FBA3E0FAA3C2
:103D0600E0F99000361218A6FFE4FCFDD003D002BD
:103D1600D001D000EB2FFFEA35F0FEED39FDEC388F
:103D2600FC901D12121BC3901D12E0F8A3E0F9A32C
:103D3600E0FAA3E0FBC000C001C002C003901D0E64
:103D4600E0FBA3E0FAA3E0F99000281218A6FFE42E
:103D5600FCFDD003D002D001D000EB2FFFEA35F0F6
:103D6600FEED39FDEC38FC901D12121BC3901D129E
:103D7600E0F8A3E0F9A3E0FAA3E0FBC000C001C0AD
:103D860002C003901D0EE0FBA3E0FAA3E0F9900049
:103D96002A1218A6FFE4FCFDD003D002D001D00001
:103DA600EB2FFFEA35F0FEED39FDEC38FC901D12E5
:103DB600121BC3901D12E0F8A3E0F9A3E0FAA3E0FA
:103DC600FB901D18E0FE901D1BE0FDEDFFE4FCFDE1
:103DD600EB2FFFEA3EFEED39FDEC38FC901D12128A
:103DE6001BC3901D12E0FCA3E0FDA3E0FEA3E024AC
:103DF60000FFEE3402FEE43DFDE43CFC901D121291
:103E06001BC3901D12E0FCA3E0FDA3E0FEA3E0FFB0
:103E1600901D0EE0FBA3E0FAA3E0F990000E121C41
:103E2600C8C003C002C001901D0EE0FBA3E0FAA3C8
:103E3600E0F99000241218A6FB901D6FE5F0F0A3A0
:103E4600EBF0D001D002D0031285E3901D12121BB5
:103E5600C3901D12E0FCA3E0FDA3E0FEA3E0FF1269
:103E6600B377901D12121BC3901D12A3A3E0FFA3EC
:103E7600E0A3CFF0A3EFF0901D0EE0FBA3E0FAA3C2
:103E8600E0F990001B12171EFD901D19E0FFA3E03C
:103E9600901CA3CFF0A3EFF0901D0EA3A3E0126930
:103EA60016EF6401600122901D0EE0FBA3E0FAA369
:103EB600E0F912187BE5F0FF12C55E901D0EE0FBDF
:103EC600A3E0FAA3E0F912187BFF12C55E901D0E5F
:103ED600E0FBA3E0FAA3E0F99000021218A6E5F0D1
:103EE600FF12C55E901D0EE0FBA3E0FAA3E0F99079
:103EF60000021218A6FF12C55EE4901D11F0901D77
:103F060011E0FFC364809484502A901D0EE0FBA349
:103F1600E0FAA3E02434F9E43AFAEF3395E0FEE957
:103F26002FF9EA3EFA121705FF12C55E901D11E041
:103F360004F080CAE4901D11F0901D11E0FFC364E7
:103F4600809484502A901D0EE0FBA3E0FAA3E0249F
:103F560028F9E43AFAEF3395E0FEE92FF9EA3EFA5A
:103F6600121705FF12C55E901D11E004F080CA907D
:103F76001D18E0FF12C55E901D1BE0FF12C55E7F97
:103F86000212C55EE4FF12C55E901D16E0FF12C563
:103F96005E901D16A3E0FF12C55EE4FF12C55EE447
:103FA600FF12C55E901D1BE030E1147F0212C55E54
:103FB6007F0412C55E7F0212C55EE4FF12C55E7FF6
:013FC60001F9
:013FC70022D7
:04B958007F017E00ED
:10B95C00901E39EEF0A3EFF0A3EBF0A3EAF0A3E90D
:10B96C00F0901E3BE0FBA3E0FAA3E0F9900030124C
:10B97C001B0D900034121B5790002C121B93901E21
:10B98C0039E0FEA3E0FFEF2BFFEE3AFEE439FDE4D5
:10B99C0038FCA3E0FBA3E0FAA3E0F9900028021B1B
:01B9AC005743
:10B85300901E9BEBF0A3EAF0A3E9F0901E9BE0FBA4
:10B86300A3E0FAA3E0F9900021ED1217907B007A90
:10B87300007900C003C002C001901E9BE0FBA3E05F
:10B88300FAA3E0F990000E121CF8901E9BE0FBA3B4
:10B89300E0FAA3E0F9900011E4F5F01219829000A8
:0BB8A30024E4F5F0121982123B8B2206
:0AC14E00E0FBA3E0FAA3E0F97D1185
:0BC15800901E9EEBF0A3EAF0A3E9F0BC
:10C1630012B853EFB40111901E9EE0FBA3E0FAA3B3
:08C17300E0F9E4FDFC12BE3905
:01C17B0022A1
:089FEB00E0FBA3E0FAA3E0F99A
:109FF300901E41EDF0901E3EEBF0A3EAF0A3E9F0D2
:10A0030090002012171EB43C24901E3EE0FBA3E0F8
:10A01300FAA3E0F9900028121B0DEF2401FFE43EA0
:10A02300FEE43DFDE43CFC900028121B57901E3ECD
:10A03300E0FBA3E0FAA3E0F9A3E0FD12B853901EFE
:10A0430042EFF064017058901E3EE0FBA3E0FAA3D8
:10A05300E0F9E4FDFC12BE39901E42EFF0D36480B8
:10A063009480403B901E3EE0FBA3E0FAA3E024383B
:10A07300F9E43AFA7D327C0012AB88901E3EE0FB95
:10A08300A3E0FAA3E0F9900034121B0DEF2401FFC3
:10A09300E43EFEE43DFDE43CFC900034121B57908B
:04A0A3001E42E0FF7A
:01A0A7002296
:0B98C000901C0AE0FBA3E0FAA3E0F913
:0B98CB00901D9EEBF0A3EAF0A3E9F073
:1098D600901D9EE0FBA3E0FAA3E0F990000E121C97
:1098E600C8901DA1EBF0A3EAF0A3E9F0901D9EE05D
:1098F600FBA3E0FAA3E0F99000111218A6FF901D51
:10990600A4E5F0F0A3EFF09000241218A6FF901D36
:10991600A6E5F0F0A3EFF07D1012B853EFB40111F5
:10992600901D9EE0FBA3E0FAA3E0F9E4FDFC12BE65
:1099360039901D9EE0FBA3E0FAA3E0F990002074A5
:109946003C121790901DA1E0FBA3E0FAA3E0F9C03A
:1099560003C002C001901D9EE0FBA3E0FAA3E0F95C
:1099660090000E121CF8901DA4E0FCA3E0FD901DD3
:109976009EE0FBA3E0FAA3E0F9900011EC8DF01253
:109986001982901DA6E0FDA3E0900024CD8DF01273
:02999600198234
:0199980022AC
:0BBFFC00901C0AE0FBA3E0FAA3E0F9B0
:10C00700900030121B0D900034121B579000221223
:10C01700171E901EB3B402057414F080037404F065
:08C02700901EB3E0FD12C158A8
:01C02F0022EE
:0FC684007E007F207D007B017A1B79780221D612
:0B828F00901DF1EBF0A3EAF0A3E9F072
:10829A00901DF774A5F0121705FFC394E05003026E
:1082AA0083B7EFD394EF40030283B7901DF1E0FB4D
:1082BA00A3E0FAA3E0F8AC02AD037B017A1B7921B3
:1082CA007E007F041221B2EF70030283B7901DF182
:1082DA0012AC1A901DF4EBF0A3EAF0A3E9F04A609D
:1082EA001B901DF4E0FBA3E0FAA3E0F990000674EA
:1082FA000112174B901DF77402F0806912BF229089
:10830A001DF4EBF0A3EAF0A3E9F04A6058E4FF9009
:10831A001DF1E0FBA3E0FAA3E0F98F827583001256
:10832A00171EFE901DF4E0FBA3E0FAA3E0F98F828A
:10833A00758300EE1217900FEFB404D3901DF4E08A
:10834A00FBA3E0FAA3E0F9900007E412179090006B
:10835A0004E4F5F012198290000674011217909045
:10836A001DF77401F0901DF7E064017040901DF450
:10837A00E0FBA3E0FAA3E0F91287FE901DF7EFF005
:10838A00D364809480901DF4E0FBA3E0FAA3E0F9A3
:10839A00400512BB8A8016E412177E901DF4E0FB9A
:1083AA00A3E0FAA3E0F9900006E4121790901DF7F3
:0283BA00E0FFE2
:0183BC00229E
:0BB4C500901E6DEBF0A3EAF0A3E9F08D
:10B4D000A374A5F0901E6DE0FBA3E0FAA3E0F8AC26
:10B4E00002AD037B017A1B79217E007F041221B219
:10B4F000EF603A901E6D12AC1AE94A603090000677
:10B5000012171E602890000712171EFF64016004C6
:10B51000EFB4021990000674FF12174B9000061248
:10B52000171E700312177E901E707401F0901E702B
:02B53000E0FF3A
:01B5320022F6
:10769500E4901D26F012BA53901D1CEFF0641160A2
:1076A50004E0B4120FC3901AC8E09408901AC7E01A
:1076B50094005006901D267401F0901D26E060038D
:1076C50002778012BA53901D1DEFF012BA53901D28
:1076D5001EEFF012BA53901D1FEFF0E4901D24F039
:1076E500A3F012BA53901D24E0FCA3E02420F582F8
:1076F500741D3CF583EFF0901D25E004F0700690B5
:107705001D24E004F0C3901D25E09404901D24E0A1
:10771500940040CE901D1CE0FFA3E0FD7B017A1D87
:107725007920129B45AD07AC06ECFF901D1EE0B518
:107735000705A3E06D6002803C901D1CE0B41118A4
:1077450078D47C1A7D017B017A1B79217E007F0428
:107755001221B2EF6002801D901D1CE0B4121C784E
:10776500207C1D7D017B017A1A79D47E007F04126D
:1077750021B2EF6006901D267401F0901D26E06091
:1077850003027833901D1CE06411705E901D24F097
:10779500A3F0901D24E0FEA3E0FFC39404EE940043
:1077A5004003027833EF7803C333CE33CED8F924C0
:1077B50078F9741B3EFA7B01901D27EBF0A3EAF0E4
:1077C500A3E9F090000712171EB4020E901D27E0E2
:1077D500FBA3E0FAA3E0F912BB8A901D25E004F0B3
:1077E50070B0901D24E004F080A8901D1CE0641288
:1077F500703C7B017A1D792012AC22901D27EBF09D
:10780500A3EAF0A3E9F04A6025901D27E0FBA3E079
:10781500FAA3E0F990000712171EB40111900007B2
:0E7825007402121790900004E4F5F01219821C
:017833002232
:08AC1A00E0FBA3E0FAA3E0F95E
:0BAC2200901E43EBF0A3EAF0A3E9F062
:10AC2D00E4A3F0A3F0901E46E0FEA3E0FFC394045E
:10AC3D00EE9400505EEF7803C333CE33CED8F924B3
:10AC4D0078F9741B3EFA7B01C003C002901E43E0ED
:10AC5D00FBA3E0FAA3E0F8AC02AD03D002D0037E73
:10AC6D00007F041221B2EF701A901E46E0FEA3E0A1
:10AC7D007803C333CE33CED8F92478F9741B3EFA5A
:10AC8D007B0122901E47E004F0709A901E46E0046E
:09AC9D00F080927B007A0079003E
:01ACA600228B
:10BD7B00E4FDFCEDCEECCE7803C333CE33CED8F955
:10BD8B002478F9741B3EFA7B0190000712171EB43E
:10BD9B0001149000041218A645F0600A9000047478
:10BDAB00FFF5F01219160DBD00010CED64044C707B
:01BDBB00C2C5
:01BDBC002264
:10B04500E4901E4BF0A3F0901E4BE0FEA3E0FFC37F
:10B055009404EE94005065EF7803C333CE33CED815
:10B06500F92478F9741B3EFA7B01901E48EBF0A396
:10B07500EAF0A3E9F090000712171EB4012E901E06
:10B0850048E0FBA3E0FAA3E0F99000041218A645F6
:10B09500F070191287FEEF6013901E48E0FBA3E0E5
:10B0A500FAA3E0F99000077402121790901E4CE085
:0CB0B50004F07093901E4BE004F0808BC0
:01B0C100226C
:1087FE00901DD874A5F0E94A7003028905C001E402
:10880E00901C92F0A3F0A37402F0E4A3F0F9A3C9B4
:10881E00F0A3F0A3E9F0E4A3F0A3F0D001FDFC1265
:10882E004EB3901DD4EFF0C3648094805003028940
:10883E0005E0FF3395E0FE7C007D3D1217B2747BA0
:10884E002FF974123EFA7B01A3EBF0A3EAF0A3E931
:10885E00F02404F9E43AFAE4FD7F12129B45901DD0
:10886E00DAEEF0A3EFF0901DD5E0FBA3E0FAA3E063
:10887E00F9901CA3E4F0A37408F07D02126916EFC0
:10888E00606D7F1212C55EE4FF12C55E901DDAE0C8
:10889E00FF12C55E901DDAA3E0FF12C55EE4901DC7
:1088AE00D9F0901DD9E0FFC364809484502A901DA6
:1088BE00D5E0FBA3E0FAA3E02404F9E43AFAEF339F
:1088CE0095E0FEE92FF9EA3EFA121705FF12C55E92
:1088DE00901DD9E004F080CA901DD5E0FBA3E0FA0C
:1088EE00A3E0F9E4FDFC12BE39901DD87401F0909E
:0C88FE001DD4E0FF12A40F901DD8E0FF75
:01890A00224A
:10BF2200E4FDFCEDAE047803C333CE33CED8F9FF83
:10BF32002478F582741B3EF583E0700B74782FF938
:10BF4200741B3EFA7B01220DBD00010CED64044C12
:08BF520070D17B007A00790038
:01BF5A0022C4
:0B9B4500901DF8EBF0A3EAF0A3E9F09C
:109B5000EFFEEDFFE4FCFDA3121BC3901DFBE0F83C
:109B6000A3E0F9A3E0FAA3E0FBC000C001C002C07B
:109B700003901DF8E0FBA3E0FAA3E0F990000112C6
:109B8000171EFD121705FEEDFFE4FCFDD003D00209
:109B9000D001D000EB2FFFEA3EFEED39FDEC38FCA2
:109BA000901DFB121BC3901DFBE0F8A3E0F9A3E09E
:109BB000FAA3E0FBC000C001C002C003901DF8E0A2
:109BC000FBA3E0FAA3E0F990000212171EFE90003A
:109BD0000312171EFDEDFFE4FCFDD003D002D001FF
:109BE000D000EB2FFFEA3EFEED39FDEC38FC901D76
:109BF000FB121BC3901DFBE0FCA3E0FDA3E0FEA352
:109C0000E0FF12B377901DFB121BC3901DFBE0FC1D
:099C1000A3E0FDA3E0FEA3E0FFC8
:019C19002228
:0BBB8A00901EA1EBF0A3EAF0A3E9F08D
:10BB950012C6AFEE540FFE901C2DE07C002FFFEC7B
:10BBA5003ECF2401CF3400FED3EF94E8EE9403405A
:10BBB500047E037FE8901EA1E0FBA3E0FAA3E0F971
:10BBC5009000077401121790900004EE8FF002198F
:01BBD50082ED
:1012390002154AE86480F8E933E83360110460F084
:10124900ED33EC337009E8FCE9FDEAFEEBFF22041B
:1012590060DED3EB9FEA9EE99DE8C2E78CF0C2F716
:1012690095F0400CE8CCF8E9CDF9EACEFAEBCFFBE2
:1012790012151585D0F05804700320D5B3E8047011
:10128900075002B2D502155492D5EC0460F7E4CCAC
:10129900C0E0C398F8603B94186008400DD0E0FBAB
:1012A90002152CE4FBFAC9FC8028E830E406E4C9FD
:1012B900FBE4CAFCE830E305E4C9CACBFCE85407FF
:1012C9006010F8C3E913F9EA13FAEB13FBEC13FC0A
:1012D900D8F130F52FC3E49CFCEF9BFFEE9AFEEDAD
:1012E90099FDD0E0FBEF4E4D4C701222DB03021545
:1012F90051EC2CFCEF33FFEE33FEED33FDED30E71F
:10130900EB02152CEF2BFFEE3AFEED39FDD0E0FB99
:1013190050130BBB0003021554ED13FDEE13FEEF42
:0813290013FFEC13FC02152C6C
:10133100EC4D6011E8497017ED33EC3304600DE4B6
:10134100FCFFFEFD22E933E8330470F802154A126E
:10135100151558046009E4CC24815006285009026F
:101361001554284003021551C0E0EB4A7044B9807E
:1013710006D0E0FB021540EF4E701CBD8008EBFF6C
:10138100EAFEE9FD80EBE98DF0A4FEE5F002141A16
:10139100E9CDF9EAFEEBFFEF89F0A4FCE5F0CE8997
:1013A100F0A42EFFE435F0CD89F0A42DFEE435F054
:1013B1008067EF4E7005BD80D780C3EF8BF0A4AC82
:1013C100F0EE8BF0A42CFCE435F0F8EF8AF0A42CBD
:1013D100E5F038FCE433CB8DF0A42CFCE5F03BF8D0
:1013E100EE8AF0A42CFCE5F038F8E433CF89F0A4C0
:1013F1002CFCE5F038CF3400CE89F0A42FFFE5F0C6
:101401003EFEE433C98DF0A42EFEE5F039CD8AF01D
:10141100A42FFFE5F03EFEE43DFD33D0E0FB500795
:101421000BBB000F021554EC2CFCEF33FFEE33FE27
:06143100ED33FD02152C55
:10143700021554EC5D046005E85904700302154A6F
:10144700121515580460F6EC4860F2EC7004FDFEC6
:10145700FF22C860DB2481C85009C3986002500688
:101467000215519850CAF582E9294B4A7005AB829B
:1014770002154075F0007C1A7880C3EF9BEE9AED59
:1014870099400DC3EF9BFFEE9AFEED99FDE842F000
:10149700DC23ACF0D0E0FFD0E0FED0E0FDAB822053
:1014A700E7101BEB60BAEC2CFCEF33FFEE33FEEDDD
:1014B70033FD02152CE803F830E705C0F075F0009E
:1014C700EF2FFFEE33FEED33FD40B830E7C280AAC1
:1014D70075F020800E75F010800575F0087D007E90
:1014E700007F003392D530D503121AB2EC33401087
:1014F700EF33FFEE33FEED33FDEC33FCD5F0ED2299
:0E150700E5F0247EA2D513CC92E7CDCEFF22D4
:108EF200901B3E121BC374FFFFFEFDFC901B3EE065
:108F0200F8A3E0F9A3E0FAA3E0FBC3121AD6603893
:108F12007F807E967D187C4B901B3EE0F8A3E0F9A3
:108F2200A3E0FAA3E0FB12155F6002501B7F807E74
:108F3200967D187CCB901B3EE0F8A3E0F9A3E0FA03
:108F4200A3E0FB12155F500F901B3EE0FCA3E0FD77
:108F5200A3E0FEA3E0FF22901B3EE0FCA3E0FDA302
:108F6200E0FEA3E0FF1215D8901B42121BC3901B18
:108F720042E0FCA3E0FDA3E0FEA3E0FFEC1214D765
:108F8200C8ECC8C9EDC9CAEECACBEFCB901B3EE014
:108F9200FCA3E0FDA3E0FEA3E0FF12123CE4FBFA17
:108FA200F9F812155F60264024901B42E0FCA3E012
:108FB200FDA3E0FEA3E0FFEF24FFFFEE34FFFEED92
:108FC20034FFFDEC34FFFC901B42121BC3901B428A
:108FD200E0FCA3E0FDA3E0FEA3E0FFEC1214D72225
:10151500E9D2E7C933E833F892D5EDD2E7CD33EC1C
:0715250033FC5002B2D52295
:10152C00EC30E7100FBF000C0EBE00080DBD000420
:10153C000BEB6014A2D5EB13FCED92E7FD2274FFCC
:10154C00FCFDFEFF22E480F8A2D574FF13FC7D8025
:03155C00E480EF39
:10155F0074F8CC6480CCC86480C8F58204604FC333
:10156F00EB9FF5F0EA9E42F0E99D42F0E89C45F0D2
:10157F00603C501DE5825FFFE582D313CB5BCBF45C
:10158F002B5582FB50280ABA002409B90020088085
:10159F001DE5825BFBE582D313CF5FCFF4C3132F1F
:1015AF005582FF50090EBE00050DBD00010CC3EBA7
:1015BF009FF5F0EA9E42F0E99D42F0E89C45F0600D
:0915CF0007CC4820E701B3EC222F
:1015D800EDD2E7CD33EC3392D524814006E4FFFE0B
:1015E800FDFC22FCE4CFCECDCC24E0501174FF806A
:1015F800EDC3CC13CCCD13CDCE13CECF13CF047007
:07160800F030D5DE021AB23A
:10AB0800028C0AE493A3F8E493A34003F68001F2CD
:10AB180008DFF48029E493A3F85407240CC8C3334E
:10AB2800C4540F4420C8834004F456800146F6DF1D
:10AB3800E4800B010204081020408090BF5BE47E93
:10AB4800019360BCA3FF543F30E509541FFEE49312
:10AB5800A360010ECF54C025E060A840B8E493A3D9
:10AB6800FAE493A3F8E493A3C8C582C8CAC583CA04
:10AB7800F0A3C8C582C8CAC583CADFE9DEE780BEBC
:01BF920000AE
:10160F00E709F608DFFA8046E709F208DFFA803EBD
:10161F0088828C83E709F0A3DFFA8032E309F608AA
:10162F00DFFA8078E309F208DFFA807088828C8312
:10163F00E309F0A3DFFA806489828A83E0A3F608C6
:10164F00DFFA805889828A83E0A3F208DFFA804CA0
:10165F0080D280FA80C680D4806980F28033801077
:10166F0080A680EA809A80A880DA80E280CA8033E0
:10167F0089828A83ECFAE493A3C8C582C8CCC58358
:10168F00CCF0A3C8C582C8CCC583CCDFE9DEE78028
:10169F000D89828A83E493A3F608DFF9ECFAA9F0A7
:1016AF00EDFB2289828A83ECFAE0A3C8C582C8CCFD
:1016BF00C583CCF0A3C8C582C8CCC583CCDFEADE16
:1016CF00E880DB89828A83E493A3F208DFF980CC78
:1016DF0088F0EF60010E4E60C388F0ED2402B40471
:1016EF000050B9F582EB2402B4040050AF23234518
:0616FF00822390165F73C8
:10170500BB010689828A83E0225002E722BBFE02E2
:09171500E32289828A83E4932215
:10171E00BB010CE58229F582E5833AF583E0225080
:10172E0006E92582F8E622BBFE06E92582F8E222CA
:0D173E00E58229F582E5833AF583E49322E4
:10174B00BB010FF8E58229F582E5833AF583E028A2
:10175B00F0225009C58229F8E58226F622BBFE0944
:10176B00C58229F8E22582F222F8EA2583F583E97E
:03177B009328228E
:10177E00BB010689828A83F0225002F722BBFE014A
:02178E00F32244
:10179000F8BB010DE58229F582E5833AF583E8F08F
:1017A000225006E92582C8F622BBFE05E92582C83B
:0217B000F22223
:1017B200EF8DF0A4A8F0CF8CF0A428CE8DF0A42E4B
:0217C200FE2205
:1017C400BC000BBE0029EF8DF084FFADF022E4CC09
:1017D400F875F008EF2FFFEE33FEEC33FCEE9DECD2
:1017E400984005FCEE9DFE0FD5F0E9E4CEFD22ED18
:1017F400F8F5F0EE8420D21CFEADF075F008EF2F62
:10180400FFED33FD4007985006D5F0F222C398FD52
:051814000FD5F0EA22EF
:10181900C2D5EC30E709B2D5E4C39DFDE49CFCEEEA
:1018290030E715B2D5E4C39FFFE49EFE1217C4C387
:10183900E49DFDE49CFC80031217C430D507C3E482
:061849009FFFE49EFE2259
:10184F00C5F0F8A3E028F0C5F0F8E5821582700224
:06185F001583E038F022C1
:10186500A3F8E0C5F025F0F0E58215827002158336
:06187500E0C838F0E82293
:10187B00BB010A89828A83E0F5F0A3E02250068738
:10188B00F009E71922BBFE07E3F5F009E3192289FA
:0B189B00828A83E493F5F0740193222D
:1018A600BB0110E58229F582E5833AF583E0F5F080
:1018B600A3E0225009E92582F886F008E622BBFE5D
:1018C6000AE92582F8E2F5F008E222E5832AF583A3
:0818D600E993F5F0A3E9932268
:1018DE00BB010789828A8302184F500B09C5F02776
:1018EE00F7C5F01937F722BBFE0D09F8E325F0F323
:1018FE00C5F019E338F322F889828A83740193259F
:08190E00F0C5F0F8E493382263
:10191600BB010DC58229C582C5833AC58302184F0E
:101926005011C58229F808E5F026F618F5F0E5828B
:1019360036F622BBFE11C58229F808E225F0F5F03D
:10194600F218E23582F222F8E58229F582E5832A49
:0D195600F58374019325F0F5F0E493382239
:10196300BB010A89828A83F0E5F0A3F0225006F7CF
:0F19730009A7F01922BBFE06F3E5F009F31922CC
:10198200F8BB0111E58229F582E5833AF583E8F097
:10199200E5F0A3F0225009E92582C8F608A6F02254
:0D19A200BBFE09E92582C8F2E5F008F2223B
:0D19AF00EF2BFFEE3AFEED39FDEC38FC2287
:0E19BC00C3EF9BFFEE9AFEED99FDEC98FC2226
:1019CA0075F008758200EF2FFFEE33FECD33CDCCD4
:1019DA0033CCC58233C5829BED9AEC99E582984057
:1019EA000CF582EE9BFEED9AFDEC99FC0FD5F0D634
:1019FA00E4CEFBE4CDFAE4CCF9A88222B800C1B95E
:101A0A000059BA002DEC8BF084CFCECDFCE5F0CB9B
:101A1A00F97818EF2FFFEE33FEED33FDEC33FCEBD4
:101A2A0033FB10D703994004EB99FB0FD8E5E4F98F
:101A3A00FA227818EF2FFFEE33FEED33FDEC33FC7C
:101A4A00C933C910D7059BE99A4007EC9BFCE99A70
:101A5A00F90FD8E0E4C9FAE4CCFB2275F010EF2FB5
:101A6A00FFEE33FEED33FDCC33CCC833C810D707B5
:101A7A009BEC9AE899400AED9BFDEC9AFCE899F8F0
:0E1A8A000FD5F0DAE4CDFBE4CCFAE4C8F92283
:0D1A9800EF4BFFEE4AFEED49FDEC48FC224D
:0D1AA500CFF4CFCEF4CECDF4CDCCF4CC22D6
:0E1AB200C3E49FFFE49EFEE49DFDE49CFC2245
:101AC000EB9FF5F0EA9E42F0E99D42F0EC6480C89D
:061AD00064809845F0223D
:101AD600EB9FF5F0EA9E42F0E99D42F0E89C45F066
:011AE60022DD
:101AE700E8600FECC313FCED13FDEE13FEEF13FFDD
:031AF700D8F12201
:101AFA00E8600FEFC333FFEE33FEED33FDEC33FC4A
:031B0A00D8F122ED
:101B0D00BB010DE58229F582E5833AF583021B7B46
:101B1D005007E92582F8022202BBFE07E92582F86B
:101B2D0002220EE58229F582E5833AF58302221A17
:101B3D00BB010789828A83021BC35005E9F8022283
:0A1B4D0054BBFE05E9F802226022F5
:101B5700BB010DE58229F582E5833AF583021BC3B4
:101B67005007E92582F8022254BBFE07E92582F8CF
:041B770002226022C4
:0C1B7B00E0FCA3E0FDA3E0FEA3E0FF22DD
:0C1B8700E0F8A3E0F9A3E0FAA3E0FB22E1
:101B9300BB010DE58229F582E5833AF583021B87B4
:101BA3005007E92582F802222ABBFE07E92582F8BD
:101BB300022237E58229F582E5833AF5830222443E
:0C1BC300ECF0A3EDF0A3EEF0A3EFF02295
:101BCF00A8828583F0D083D082121BE6121BE61207
:101BDF001BE6121BE6E473E493A3C583C5F0C5832C
:101BEF00C8C582C8F0A3C583C5F0C583C8C582C860
:011BFF0022C3
:101C0000BB010DE58229F582E5833AF583021BCFFE
:101C10005007E92582F802226CBBFE07E92582F80D
:041C200002228522F5
:0C1C2400A42582F582E5F03583F58322CB
:091C3000E0FBA3E0FAA3E0F922B5
:101C3900F8E0FBA3A3E0F925F0F0E5821582700234
:071C49001583E0FA38F022D8
:091C5000EBF0A3EAF0A3E9F02295
:101C5900BB010789828A83021C305005E9F80222F8
:101C69009EBBFE05E9F80222B089828A830222C25C
:101C7900BB011A89828A83D0F0D0E0F8D0E0F9D08C
:101C8900E0FAD0E0FBE8C0E0C0F0021C505016E9D1
:101C9900F8D083D082D0E0F9D0E0FAD0E0FBC0825E
:101CA900C0830222A7BBFE16E9F8D083D082D0E018
:0F1CB900F9D0E0FAD0E0FBC082C0830222B9224A
:101CC800BB010DE58229F582E5833AF583021C30D4
:101CD8005007E92582F802229EBBFE07E92582F813
:101CE8000222B0E58229F582E5833AF5830222C211
:101CF800BB0120E58229F582E5833AF583D0F0D04F
:101D0800E0F8D0E0F9D0E0FAD0E0FBE8C0E0C0F0BD
:101D1800021C505018E92582F8D083D082D0E0F90F
:101D2800D0E0FAD0E0FBC082C0830222A7BBFE1835
:101D3800E92582F8D083D082D0E0F9D0E0FAD0E06B
:091D4800FBC082C0830222B92213
:101D5100D083D082F8E4937012740193700DA3A321
:101D610093F8740193F5828883E473740293686035
:061D7100EFA3A3A380DF35
:101D7700E5132582F582E5123583F583B5120485CF
:101D870082132210AF06858213F51222858213F57E
:041D970012D2AF2293
:0D1D9B00E5132582F582E5123583F58322DC
:101DA800E3F5F009E208B5F06D606B80F3E3F5F058
:101DB80009E608B5F060605E80F387F009E608B5CB
:101DC800F054605280F487F009E208B5F0486046A4
:101DD80080F488828C8387F009E0A3B5F0386036F8
:101DE80080F488828C8387F009E493A3B5F0276098
:101DF8002580F388828C83E3F5F009E0A3B5F0161B
:101E0800601480F388828C83E3F5F009E493A3B52A
:101E1800F004600280F2021ED3808580E7808E8005
:101E2800D2803C8015806C807E809B80B5808B80C2
:101E3800A1804F8070803A021EDF89828A83ECFA83
:101E4800E493F5F0A3C8C582C8CCC583CCE493A3BA
:101E5800C8C582C8CCC583CCB5F070606E80E189F6
:101E6800828A83E493F5F0A3E208B5F05E605C80B3
:101E7800F289828A83E0F5F0A3E608B5F04D604B5D
:101E880080F389828A83E0F5F0A3E208B5F03C602C
:101E98003A80F389828A83E493F5F0A3E608B5F0E3
:101EA8002A602880F2805389828A83ECFAE493F5C9
:101EB800F0A3C8C582C8CCC583CCE0A3C8C582C876
:101EC800CCC583CCB5F004600280E27FFFB5F00298
:101ED8000F2240027F012289828A83ECFAE0F5F022
:101EE800A3C8C582C8CCC583CCE0A3C8C582C8CC6A
:101EF800C583CCB5F0D560D380E389828A83ECFAB8
:101F0800E0F5F0A3C8C582C8CCC583CCE493A3C8C8
:101F1800C582C8CCC583CCB5F0B160AF80E288F08B
:101F2800ED2402B4040050A3F582EB2402B40400AB
:0B1F380050992323458223901E217343
:101F4300E709F60870FA8046E709F20870FA803E5E
:101F530088828C83E709F0A370FA807EE309F60890
:101F630070FA8076E309F20870FA806E88828C83B7
:101F7300E309F0A370FA806289828A83E0A3F608FA
:101F830070FA805689828A83E0A3F20870FA804A45
:101F930080D280FA80C680D4806580F28031801040
:101FA30080A680EA809A80A880DA80E280CA8031A5
:101FB30089828A83ECFAE493A3C8C582C8CCC5831B
:101FC300CCF0A3C8C582C8CCC583CC70E9800D8989
:101FD300828A83E493A3F60870F9ECFAA9F0EDFB87
:101FE3002289828A83ECFAE0A3C8C582C8CCC58360
:101FF300CCF0A3C8C582C8CCC583CC70EA80DD8988
:10200300828A83E493A3F20870F980CE88F0ED24EA
:1020130002B4040050C4F582EB2402B4040050BAA5
:092023002323458223901F9373CF
:10C5BA00E4FFFE121705600C0FEF70010E09E97017
:05C5CA00F20A80EF22DF
:10202C00E3F5F009E208B5F06BDFF58067E3F5F056
:10203C0009E608B5F05EDFF5805A87F009E608B5C9
:10204C00F052DFF6804E87F009E208B5F046DFF675
:10205C00804288828C8387F009E0A3B5F036DFF6E6
:10206C00803288828C8387F009E493A3B5F025DF56
:10207C00F5802188828C83E3F5F009E0A3B5F01498
:10208C00DFF5801088828C83E3F5F009E493A3B527
:10209C00F002DFF402215B808780E9809080D4809D
:1020AC003E8015806E807E809D80B7808D80A38061
:1020BC00518074803C02216789828A83ECFAE49314
:1020CC00F5F0A3C8C582C8CCC583CCE493A3C8C51E
:1020DC0082C8CCC583CCB5F076DFE3DEE1807089B5
:1020EC00828A83E493F5F0A3E208B5F062DFF48012
:1020FC005E89828A83E0F5F0A3E608B5F051DFF53E
:10210C00804D89828A83E0F5F0A3E208B5F040DFC8
:10211C00F5803C89828A83E493F5F0A3E608B5F058
:10212C002EDFF4802A8002805789828A83ECFAE4BD
:10213C0093F5F0A3C8C582C8CCC583CCE0A3C8C5B1
:10214C0082C8CCC583CCB5F006DFE4DEE280007F2C
:10215C00FFB5F0020F2240027F012289828A83ECB4
:10216C00FAE0F5F0A3C8C582C8CCC583CCE0A3C8FF
:10217C00C582C8CCC583CCB5F0D5DFE5DEE380CF16
:10218C0089828A83ECFAE0F5F0A3C8C582C8CCC575
:10219C0083CCE493A3C8C582C8CCC583CCB5F0AFBF
:1021AC00DFE4DEE280A988F0EF60010E4E60ABED5B
:1021BC002402B404005098F582EB2402B4040050BD
:0A21CC008E23234582239020A37385
:1021D600EF4E6012EF60010EEDBB010B89828A8320
:1021E600F0A3DFFCDEFA2289F05007F709DFFCA92D
:0C21F600F022BBFEFCF309DFFCA9F02284
:0C220200E6FC08E6FD08E6FE08E6FF2208
:0C220E00E2FC08E2FD08E2FE08E2FF220C
:10221A00E493FC740193FD740293FE740393FF220A
:0D222A00E6FB08E6F908E6FA08E6CBF82224
:0D223700E2FB08E2F908E2FA08E2CBF82227
:10224400E493F8740193F9740293FA740393FB22F0
:0C225400ECF608EDF608EEF608EFF622B6
:0C226000ECF208EDF208EEF208EFF222BA
:10226C00D083D082E493F608740193F60874029339
:09227C00F608740393F674047370
:10228500D083D082E493F208740193F20874029328
:09229500F208740393F27404735F
:09229E00E6FB08E6FA08E6F92265
:0922A700EBF608EAF608E9F6225C
:0922B000E2FB08E2FA08E2F9225F
:0922B900EBF208EAF208E9F22256
:0C22C200E493FB740193FA740293F92278
:00000001FF
